:020000040000FA
:10000000D8F9012055030000790300007B030000AC
:100010007D0300007F0300008103000083030000D4
:1000200083030000830300008303000083030000B8
:100030008303000083030000EF0200008D380000FE
:1000400069070000730700007D07000087070000B4
:1000500091070000890A0000930A0000AD09000022
:10006000B3080000210900002B0900003509000039
:100070003F09000053090000C5060000CF0600003C
:10008000D9060000E3060000F70A0000E9090000B5
:10009000F3090000FD090000070A0000110A000032
:1000A0001B0A0000A7060000B1060000BB06000006
:1000B000D5090000550700009B070000A5070000B8
:1000C000AF0700009D0A0000B7090000250A0000E4
:1000D0002F0A0000BD0800001F07000029070000CC
:1000E0004B070000A9080000ED0A000049090000C4
:1000F000E30A0000D90A0000ED060000F706000040
:10010000010700000B07000041070000B9070000CD
:10011000C3070000CD070000C1090000CB090000A3
:10012000A70A0000B10A0000BB0A0000C50A0000CF
:10013000CF0A0000C7080000D1080000390A0000FB
:10014000430A00004D0A0000570A00005F07000044
:10015000850900008F090000DB080000E5080000A9
:10016000D7070000E107000099090000DF0900003F
:10017000EB070000F5070000FF070000090800007A
:10018000130800001D0800002708000031080000C7
:100190003B080000450800004F0800005908000017
:1001A000630800006D080000770800008108000067
:1001B0008B08000095080000A30900001507000047
:1001C0003307000017090000610A00006B0A0000F5
:1001D000750A00007F0A0000EF080000F90800001F
:1001E0005D0900009D06000067090000710900001C
:1001F0007B090000030900000D0900009F080000B2
:10020000DFF80CD000F03EF90048004719720000FA
:10021000D8F90120EFF3108072B67047EFF3108029
:100220007047EFF3108062B6704730BF704780F3BD
:1002300011887047EFF31180704700000138FDD13D
:100240007047000072B6704762B67047EFF31080D7
:1002500072B6704780F31088704730BF704720BF78
:100260007047B0FA80F0704790FAA0F0B0FA80F0D2
:10027000704790FAA0F07047EFF3098141B1F1EEB9
:10028000101A40F8041D20ED200A29490A68106060
:100290007047B0EC200A02C8E1EE101A25490A683E
:1002A00010607047EFF3108072B6704780F31088CB
:1002B000704721484FF0FF010170002080F309884A
:1002C0001E48016881F308881D48012101701D48FE
:1002D0004FF08051016062B6FEE71A484FF080513E
:1002E0000160704717484FF080510160704772B647
:1002F000EFF3098028B1203880E8F00F0C49096835
:10030000086000B5104880475DF804EB0F481049BD
:100310000A780270064807490A680260106890E887
:10032000F00F203080F309884EF0F40E62B670476B
:10033000340000203C00002022ED00E06C00002092
:100340002E00002004ED00E0F9330000230000201F
:1003500024000020DFF83000016841F470010160E2
:10036000BFF34F8FDFF82400016821F040410160A6
:10037000BFF36F8F06480047FEE7FEE7FEE7FEE7A4
:10038000FEE7FEE7FEE7000088ED00E034EF00E066
:100390000102000040EA01039B0703D009E008C9FD
:1003A000121F08C0042AFAD203E011F8013B00F83A
:1003B000013B521EF9D27047D2B201E000F8012B86
:1003C000491EFBD270470022F6E710B513460A46D5
:1003D00004461946FFF7F0FF204610BD421E12F8F2
:1003E000013F002BFBD111F8013B02F8013B002B30
:1003F000F9D17047421C10F8011B0029FBD1801A6B
:10040000704710B5002200E0521C835C8C5CA34254
:1004100001D1002BF8D1D8B2E1B2401A10BD30B5ED
:1004200004460020034600E05B1C934203D2E05CDC
:10043000CD5C401BF8D030BD30B5054600200346EA
:1004400000E05B1C934205D2EC5CC85C201A01D131
:10045000002CF6D130BD30B50B46014600202022DD
:10046000012409E021FA02F59D4205D303FA02F5C1
:10047000491B04FA02F52844151EA2F10102F1DC21
:1004800030BD0000064C074D06E0E06840F0010377
:1004900094E8070098471034AC42F6D3FFF7B4FE57
:1004A000F4DF000014E0000070B58C1810F8015B58
:1004B00015F0070301D110F8013B2A1106D110F8FD
:1004C000012B03E010F8016B01F8016B5B1EF9D101
:1004D0002B0705D40023521E0DD401F8013BFAE787
:1004E00010F8013BCB1A921C03E013F8015B01F8F2
:1004F000015B521EF9D5A142D8D3002070BD000087
:1005000000B585B0032000214FF400721E4BCDE9E9
:100510000132CDE90310072003461C4A00901C4815
:1005200002F060FC032000214FF40072194BCDE96A
:100530000132CDE9031006200346174A0090174800
:1005400002F050FC032000214FF48072144BCDE9DF
:100550000132CDE9031008200346124A00901248E8
:1005600002F040FC032000214FF480720F4BCDE9D4
:100570000132CDE90310092003460D4A00900D48D1
:1005800002F030FC05B000BDD4EF0120D0F701200F
:100590009D410000D4E70120D0EF012001160000AA
:1005A000D4DF0120D0E3012059410000D4E3012031
:1005B000D0E701208545000086B000F03FF800F04C
:1005C00035FB04464FF47A70B4FBF0F5284603F08F
:1005D00071F900F0E6FE02F0D9FB01F0DBFD2046E8
:1005E00000F002FD01F048F90C4803C8CDE9000114
:1005F0000B48006805900B48006804900A480068A2
:100600000390DDE9041200F0A3FAFFF779FF03E09D
:100610004FF47A7002F0F4FEFAE70000D0010020F7
:10062000C8010020C4010020C001002070477047AD
:1006300070477047704770477047704710B500F0BB
:100640005FFA00F047FB10BD10B50446702C04D2D1
:1006500004F11001C8B200F0ABFE10BD70B5044645
:10066000002600BF00BFFFF7F1FD064600BF00BF38
:1006700001F0FAFE00BF00BF3046FFF7EBFD00BF00
:1006800000BF702C04D2044850F8245005B1A8478C
:1006900001F004FF70BD00003006002010B5692095
:1006A000FFF7DCFF10BD10B51920FFF7D7FF10BD15
:1006B00010B51A20FFF7D2FF10BD10B51B20FFF7B1
:1006C000CDFF10BD10B50E20FFF7C8FF10BD10B54F
:1006D0000F20FFF7C3FF10BD10B51020FFF7BEFFBE
:1006E00010BD10B51120FFF7B9FF10BD10B52E20B9
:1006F000FFF7B4FF10BD10B52F20FFF7AFFF10BDFF
:1007000010B53020FFF7AAFF10BD10B53120FFF75C
:10071000A5FF10BD10B55F20FFF7A0FF10BD10B5FD
:100720002620FFF79BFF10BD10B52720FFF796FF8F
:1007300010BD10B56020FFF791FF10BD00BFFEE7B0
:1007400010B53220FFF78AFF10BD10B52820FFF743
:1007500085FF10BD10B51D20FFF780FF10BD10B53F
:100760004320FFF77BFF10BD10B50020FFF776FF99
:1007700010BD10B50120FFF771FF10BD10B50220AC
:10078000FFF76CFF10BD10B50320FFF767FF10BD2A
:1007900010B50420FFF762FF10BD10B51E20FFF753
:1007A0005DFF10BD10B51F20FFF758FF10BD10B53D
:1007B0002020FFF753FF10BD10B53320FFF74EFF89
:1007C00010BD10B53420FFF749FF10BD10B535201E
:1007D000FFF744FF10BD10B54820FFF73FFF10BDE5
:1007E00010B54920FFF73AFF10BD10B54C20FFF7B8
:1007F00035FF10BD10B54D20FFF730FF10BD10B50F
:100800004E20FFF72BFF10BD10B54F20FFF726FF3E
:1008100010BD10B55020FFF721FF10BD10B55120BD
:10082000FFF71CFF10BD10B55220FFF717FF10BDDA
:1008300010B55320FFF712FF10BD10B55420FFF77D
:100840000DFF10BD10B55520FFF708FF10BD10B506
:100850005620FFF703FF10BD10B55720FFF7FEFE2F
:1008600010BD10B55820FFF7F9FE10BD10B5592086
:10087000FFF7F4FE10BD10B55A20FFF7EFFE10BDD4
:1008800010B55B20FFF7EAFE10BD10B55C20FFF746
:10089000E5FE10BD10B55D20FFF7E0FE10BD10B500
:1008A0006F20FFF7DBFE10BD10B52920FFF7D6FE45
:1008B00010BD10B50820FFF7D1FE10BD10B52520E2
:1008C000FFF7CCFE10BD10B53D20FFF7C7FE10BDF1
:1008D00010B53E20FFF7C2FE10BD10B54620FFF751
:1008E000BDFE10BD10B54720FFF7B8FE10BD10B516
:1008F0006620FFF7B3FE10BD10B56720FFF7AEFE10
:1009000010BD10B56D20FFF7A9FE10BD10B56E200B
:10091000FFF7A4FE10BD10B56120FFF79FFE10BDCC
:1009200010B50920FFF79AFE10BD10B50A20FFF799
:1009300095FE10BD10B50B20FFF790FE10BD10B551
:100940000C20FFF78BFE10BD10B52B20FFF786FEA5
:1009500010BD10B50D20FFF781FE10BD10B5682049
:10096000FFF77CFE10BD10B56A20FFF777FE10BDC3
:1009700010B56B20FFF772FE10BD10B56C20FFF7AD
:100980006DFE10BD10B54420FFF768FE10BD10B518
:100990004520FFF763FE10BD10B54A20FFF75EFE4D
:1009A00010BD10B55E20FFF759FE10BD10B5072031
:1009B000FFF754FE10BD10B52220FFF74FFE10BD0B
:1009C00010B53620FFF74AFE10BD10B53720FFF7EF
:1009D00045FE10BD10B51C20FFF740FE10BD10B540
:1009E0004B20FFF73BFE10BD10B51320FFF736FE7E
:1009F00010BD10B51420FFF731FE10BD10B5152045
:100A0000FFF72CFE10BD10B51620FFF727FE10BD16
:100A100010B51720FFF722FE10BD10B51820FFF704
:100A20001DFE10BD10B52320FFF718FE10BD10B538
:100A30002420FFF713FE10BD10B53F20FFF70EFE78
:100A400010BD10B54020FFF709FE10BD10B54120C4
:100A5000FFF704FE10BD10B54220FFF7FFFD10BDEB
:100A600010B56220FFF7FAFD10BD10B56320FFF747
:100A7000F5FD10BD10B56420FFF7F0FD10BD10B5F9
:100A80006520FFF7EBFD10BD10B50520FFF7E6FD73
:100A900010BD10B50620FFF7E1FD10BD10B52120F7
:100AA000FFF7DCFD10BD10B53820FFF7D7FD10BDF6
:100AB00010B53920FFF7D2FD10BD10B53A20FFF771
:100AC000CDFD10BD10B53B20FFF7C8FD10BD10B522
:100AD0003C20FFF7C3FD10BD10B52D20FFF7BEFD74
:100AE00010BD10B52C20FFF7B9FD10BD10B52A20A0
:100AF000FFF7B4FD10BD10B51220FFF7AFFD10BD1C
:100B000010B5002404E0E0B2034900F007F8641CCB
:100B1000702CF8D310BD00003D07000070B50446EE
:100B20000D460026702C10D200BF00BFFFF78EFBD1
:100B3000064600BF00BF054840F8245000BF00BF74
:100B40003046FFF787FB00BF00BF70BD30060020B6
:100B50007FB588B0DDE91045E0B28DF818004FF49C
:100B60007F4104EA01000021000A40EA0160C0B2AE
:100B70008DF819004FF47F0104EA01000021000CF8
:100B800040EA0140C0B28DF81A004FF07F4104EAFC
:100B900001000021000E40EA0120C0B28DF81B00C8
:100BA000E8B28DF81C004FF47F402840000A8DF811
:100BB0001D009DF8200000069DF8211040EA01402C
:100BC0009DF8221040EA01209DF82310084305906B
:100BD0009DF8240000069DF8251040EA01409DF88C
:100BE000261040EA01209DF82710084304909DF844
:100BF000280000069DF8291040EA01409DF82A10BF
:100C000040EA01209DF82B100843039000F0C2F841
:100C1000064600210398CDE9000106A93046DDE92A
:100C2000043205F0D1FD0CB070BD00002DE9F04399
:100C3000DFF894C0DCF8B0C0CCF3007CBCF1000F4E
:100C40003ED0DFF884C0DCF860C1CCF38A24DFF842
:100C500078C0DCF860C1CCF30A0303EB9422DFF820
:100C600068C0DCF864C1CCF30425DFF85CC0DCF8B4
:100C700064C10CF01F06DFF850C0DCF8B0C0CCF344
:100C8000036111B1032904D101E0104902E01049C8
:100C900000E000BF00BF01FB02F805F1010C06F106
:100CA00001090CFB09FCB8FBFCF0DFF81CC0DCF808
:100CB000B0C0CCF3090C0CF10107B0FBF7F000E079
:100CC0000020BDE8F083000000E00F400024F400A5
:100CD00040787D012948C06F20F01C002749C86773
:100CE0000846C06F40F01000C8672448C030006854
:100CF000234908402149C1F8C0002048C03000689D
:100D0000204908431D49C031086048061B49B031DD
:100D100008604FF04C70086060201B490860042098
:100D20001649C1F864011848A03800681449084001
:100D30001249C1F8C0001448A0380068134908439C
:100D40000E49C1F8C0000846D0F8600140F4000028
:100D5000C1F8600100BF0C480830006800F00100D5
:100D600080F001000028F6D10448B030006808493E
:100D700008430249C1F8B0007047000000E00F408E
:100D800010FC10FC8100010060E10F40850185012D
:100D90000300009001480068704700005C010020DB
:100DA0002DE9F04104460F4615461E468DB92046F2
:100DB00003F096FE24B93946114806F061FA05E0C1
:100DC000012C03D139460F4806F05AFA0020BDE83D
:100DD000F081012D10D1204603F082FE24B9314666
:100DE000074808F033F905E0012C03D131460548E6
:100DF00008F02CF90020EAE74FF0FF30E7E70000A9
:100E000000000240001002402DE9F04706468946E6
:100E100017461D464FF0000AFFF744FA824635B9DF
:100E20005046FFF743FA4FF0FF30BDE8F08716B9A0
:100E3000DFF8E8800AE0012E02D1DFF8E48005E067
:100E40005046FFF733FA4FF0FF30EEE700BF404661
:100E500001F02CF80028FAD101224946404601F061
:100E600077F8012D1BD10721404601F028F84046B4
:100E700001F031F820B15046FFF718FAA81ED4E768
:100E800000BF404601F012F80028FAD1404601F0B8
:100E900018F838705046FFF709FA0020C5E700241B
:100EA00034E024B90B21404601F009F80BE0681E3C
:100EB000A04204D10521404601F001F803E00921D8
:100EC000404600F0FCFF404601F005F898B1681E6E
:100ED000A0420AD0404600F0FEFF00F010001028AB
:100EE00003D00421404600F0EAFF5046FFF7DEF948
:100EF0004FF0FF3099E700BF404600F0D7FF0028D1
:100F0000FAD1404600F0DDFF3855641CAC42C8D32E
:100F10005046FFF7CBF9002087E7000000000240B1
:100F2000001002402DE9F0470646884617461D4648
:100F30004FF0000AFFF7B6F9824615B146B1012E0F
:100F400006D05046FFF7B2F94FF0FF30BDE8F0870A
:100F50000EB9234800E02348814600BF484600F010
:100F6000A5FF0028FAD100224146484600F0F0FFD4
:100F700000242DE0395D484600F0A6FF24B9032186
:100F8000484600F09CFF0BE0681EA04204D10521FA
:100F9000484600F094FF03E00121484600F08FFF2F
:100FA000484600F098FF60B1681EA04203D00421BB
:100FB000484600F084FF5046FFF778F94FF0FF30C5
:100FC000C4E700BF484600F071FF0028FAD1641C56
:100FD000AC42CFD35046FFF769F90020B6E70000D6
:100FE0000000024000100240014908607047000004
:100FF0005C01002010B54FF48073034A0349044894
:1010000000F0A6F910BD00006001002098D3012077
:1010100000C0004010B54FF48073034A03490448F0
:1010200000F096F910BD00006801002098D401205E
:1010300000D0004010B54FF48073034A03490448C0
:1010400000F086F910BD00007001002098D5012045
:1010500000E0004010B54FF48073034A0349044890
:1010600000F076F910BD00007801002098D601202C
:1010700000F0004010B54FF48073034A0349044860
:1010800000F066F910BD00008001002098D7012013
:101090000000014010B54FF48073034A034904482F
:1010A00000F056F910BD00008801002098D80120FA
:1010B0000010014010B54FF48073034A03490448FF
:1010C00000F046F910BD00009001002098D90120E1
:1010D0000020014010B54FF48073034A03490448CF
:1010E00000F036F910BD00009801002098DA0120C8
:1010F000003001402DE9F0418CB080460C46154689
:101100001E46129FB8F1080F77D2DFE808F00420DE
:101110003C597794AFCA1520714905220223CDE9C5
:101120000967CDE90745CDE90332CDE90510012076
:1011300040F20141CDE900014FF04023694A6A497C
:1011400002906A4803F0DEF90CB0BDE8F081162089
:10115000674906220223CDE90967CDE90745CDE9B4
:101160000332CDE90510012062494FF00112624BB4
:10117000CDE900210290614A5B49491C5B48401C53
:1011800003F0C0F9E0E731205D4921228023CDE959
:101190000967CDE90745CDE90332CDE905104020C7
:1011A00041F6014141F601024FF04023CDE9002113
:1011B0000290544A4C494D48801C03F0A3F9C3E700
:1011C0004820514938222023CDE90967CDE9074558
:1011D000CDE90332CDE90510102041F2014141F281
:1011E00001024FF04023CDE900210290474A3E49D9
:1011F0003E48C01C03F086F9A6E76DE0492044494B
:1012000039220823CDE90967CDE90745CDE9033245
:10121000CDE90510042040F6014140F601024FF0EF
:101220004023CDE9002102903A4A2F492F48001D62
:1012300003F068F988E74A2037493A228023CDE94C
:101240000967CDE90745CDE90332CDE90510402016
:101250003249334A334BCDE900210290324A2249C8
:10126000891C2248401D03F04DF96DE74B202F49A2
:101270003B220223CDE90967CDE90745CDE90332D9
:10128000CDE9051001202A492A4A2B4BCDE900213E
:1012900002902A4A14490D311448801D03F032F996
:1012A00052E74C2026493C222023CDE90967CDE9AD
:1012B0000745CDE90332CDE9051010202149224A26
:1012C000184BCDE900210290204A0749891C0748A4
:1012D000C01D03F017F937E74FF0FF3034E7000087
:1012E000F50F000000C00040000800F0001800F0FA
:1012F00015100000010401000050004000D0004023
:101300003510000000E000405510000000F00040E3
:10131000751000000000014095100000011C020043
:10132000011802000060004000100140B5100000EC
:1013300001040D0001000D00005006400020014096
:10134000D51000000114020001100200003001401D
:101350002DE9F04107460D4614461E460121384648
:1013600003F0CAF880464146384603F0BFF801F062
:101370007BF80DE0384603F061F821686854206876
:10138000401C20602068B0FBF6F106FB11002060D5
:10139000384603F065F80028ECD101F07FF8BDE88D
:1013A000F08110B500F0FAF800F0C0F810BD0000B0
:1013B0002DE9F04104464FF00008102C6BD2DFE815
:1013C00004F0080E0F1014293E090A0B0C11120D1F
:1013D000135300BF00BF00BF00BF00BF89E000BFC4
:1013E00000BF00BF00BF00BF83E000BF00BFFEF72B
:1013F0002DFF804600BF00BF3F48006840F48030AA
:101400003D49086000BF00BF4046FEF723FF00BF14
:1014100000BF6EE000BF00BFFEF718FF804600BFB0
:1014200000BF3548006840F400303349086000BF11
:1014300000BF4046FEF70EFF00BF00BF59E000BFEF
:1014400000BFFEF703FF804600BF00BF2A480068C8
:1014500040F480202849086000BF00BF4046FEF7E6
:10146000F9FE00BF00BF44E000BF00BFFEF7EEFE84
:10147000804600BF00BF4FF0E020006940F001004F
:101480004FF0E021086100BF00BF4046FEF7E2FEDA
:1014900000BF00BF2DE04FF0E0204068401C10214D
:1014A00001EB4010C7B2BC4222DAA4F11000C11710
:1014B00000EBD161C1F34715C11700EBD1614911B0
:1014C000A0EB4111CEB200BF00BFFEF7BFFE8046C9
:1014D00000BF00BF0120B040A90001F1E021C1F828
:1014E000000100BF00BF4046FEF7B4FE00BF00BFD2
:1014F00000BF00BFBDE8F08124ED00E010B500247E
:1015000000BF00BFFEF7A2FE044600BF00BF1021CF
:10151000054800F035FE00BF00BF2046FEF79AFEEA
:1015200000BF00BF10BD0000D801002010B5FFF7BC
:10153000E5FF10BD2DE9F04105460C46002714B922
:1015400000BF00F029F81DB90A202080BDE8F08115
:101550001021284602F0D9FE0646102E15D200BFF3
:1015600000BFFEF773FE074600BF00BF10222946EA
:10157000084802F0A7FE00BF00BF3846FEF76AFE2B
:1015800000BF00BF0020208002E04FF47A7020806E
:1015900000BFDBE7D801002000BFFEE710B5002048
:1015A0000249086000F00AF810BD000000000020A9
:1015B00001490860704700000000002010B50A488B
:1015C000006840F0807008490860002007494860C2
:1015D0000846006840F001000860FFF727FB04465A
:1015E0002046FFF7E5FF10BDFCED00E0001000E035
:1015F0000146002902DA4FF0FF3070470020FCE777
:101600001FB526A502208DF8010041F2D61005F085
:1016100014FBADF8020001A923A004F0E5FF3BE0B4
:1016200000220121022005F07DFD044609E0002290
:101630000121022005F076FD04464FF47A7007F090
:1016400029FE002CF3DB10226946204605F096FAAD
:101650000646002E07DA204605F070FA4FF47A703D
:1016600007F018FE18E011E02846FEF7C3FE074613
:1016700000233A462946204605F072FC0646002E15
:1016800000DA04E04FF47A7007F004FEECE700BFE4
:10169000204605F053FA00BFC2E700004920616D03
:1016A00020636C69656E74003139322E3136382E04
:1016B000312E31313200000070B50446601C00F05C
:1016C000B9F80546FFF794FF002802DA4FF0FF3023
:1016D00070BDA01C00F09EF80546FFF789FF0028AA
:1016E00002DA4FF0FF30F3E7E01C00F08BF805461C
:1016F000FFF77EFF002802DA4FF0FF30E8E7201DF9
:1017000000F078F80546FFF773FF002802DA4FF083
:10171000FF30DDE7601D00F085F80546FFF768FF44
:10172000002802DA4FF0FF30D2E7A01D00F08AF85F
:101730000546FFF75DFF002802DA4FF0FF30C7E7EC
:101740000020C5E770B504460D4614480470002318
:101750001A4629460078FFF723FB06463046FFF776
:1017600047FF002802DA4FF0FF3070BD00F072F83A
:1017700006463046FFF73CFF002802DA4FF0FF3004
:10178000F3E700F00DF806463046FFF731FF00287A
:1017900002DA4FF0FF30E8E70020E6E7B40100206E
:1017A00010B55E21202002F0E5FC0446FFF720FF83
:1017B000002802DA4FF0FF3010BDC721212002F0CF
:1017C000D9FC0446FFF714FF002802DA4FF0FF307F
:1017D000F2E70121222002F0CDFC0446FFF708FFCA
:1017E000002802DA4FF0FF30E6E74021072002F040
:1017F000C1FCE1E710B5044630222146042002F086
:1018000073FC10BD10B5044630222146022002F0C0
:101810006BFC10BD10B5044670222146012002F079
:1018200063FC10BD10B5044610222146052002F0CD
:101830005BFC10BD10B5044670222146002002F06A
:1018400053FC10BD10B50446F0222146062002F0DC
:101850004BFC10BD10B52021082002F08BFC044683
:10186000FFF7C6FE002802DA4FF0FF3010BD452119
:10187000092002F07FFCF9E710B505490120FFF7C8
:1018800061FF4FF4E131012000F004F810BD0000C9
:10189000801A060038B504460D4600200346602233
:1018A000294600902046FFF725FC38BD10B50346B9
:1018B000CC00443418591070040A5470040C94700D
:1018C000040ED470CC00403418591071040A5471BD
:1018D00010BD10B5CB004033C3586FF30F0314791C
:1018E0002343547943EA0424CB004033C450137893
:1018F000547843EA0423947843EA0443D47843EACF
:101900000464CB004433C45010BD000070B5D0F85F
:10191000185C156005680C4E35400D60D0F8DC4051
:1019200004F480351DB1C4F30D051D600AE005689F
:1019300005F480151DB14FF420551D6002E04FF4F1
:1019400000651D6070BD0000FF7E5F7A30B50468E1
:101950000A4D2C400C4344F40044046023B143F48A
:101960008034C0F8DC4005E0D0F8DC4024F480345A
:10197000C0F8DC40C0F8182C30BD00000C81A085F8
:101980004268024B1A400A434260704700F8FE7FEB
:10199000F0B50446DDE9055700BFDFF894C0DCF878
:1019A00000C00CF0010CBCF1000FF6D142EA870C2C
:1019B0004CF08000202D01D8202B03D940F08070FE
:1019C000ED08DB08AB4202D140EA052007E04FF406
:1019D000000C4CEA052C4CEA434C4CEA0000C4F8DD
:1019E000000CDFF850C0DCF8146000200DE0DFF8D8
:1019F00044C05CF830C08C4506D3DFF838C00CEB2F
:101A0000C00CDCF8046002E0401C0328EFD300BFE8
:101A1000D4F810C02CF03C0C4CEA060CC4F810C0F2
:101A20004FF0FF3CC4F80CC1C4F810C1F0BD000079
:101A300000CC0E40F0D8000044F245020A400AB142
:101A400041F4803142F2BA720A400AB141F40041D5
:101A500021F000421AB121F00042C0F8142C01F02C
:101A600000422AB1D0F8D82F42F00102C0F8D82F96
:101A7000704744F245020A400AB141F4803142F213
:101A8000BA720A400AB141F4004121F0004232B179
:101A9000D0F81C2C21F000431A43C0F81C2C01F094
:101AA00000422AB1D0F8D42F42F00102C0F8D42F5E
:101AB0007047000010B50246D2F8140C094C2040C3
:101AC00021B1D2F81C4C44F0F044204011B1D2F8BE
:101AD000D83F01E0D2F8D03F03F001040CB140F050
:101AE000004010BDFFFF01FC70B505460C46C5F86F
:101AF000C44F04F0404060B9134802F067FC00BFD7
:101B0000114802F047FC0028FAD042F21070FEF7AC
:101B100095FB04F04040B0F1404F06D10B480068FF
:101B200040F480300949086005E00848006820F466
:101B3000803006490860064800F042F84FF47A7099
:101B4000FEF77CFB70BD0000003000F0C8CF0E40F7
:101B500000C00E40034600BF186900F001000028D5
:101B6000FAD1186900F03C0040EA821040EAC12036
:101B7000401C186100BF186900F001000028FAD16C
:101B8000586980B2704710B500BF046904F00104C1
:101B9000002CFAD14361046904F03C0444EA821445
:101BA00044EAC124E41C046100BF046904F0010498
:101BB000002CFAD110BD0146C86A00F061007047E0
:101BC000D0F8001C41F00101C0F8001C00BFD0F8A3
:101BD000001C01F001010029F9D17047C0F80C1C6C
:101BE0007047D0F8181C41F00201C0F8181C0168B9
:101BF00041F00401016070470146D1F828077047A1
:101C0000C0F8101C70470021C0F8041C7047D0F8C1
:101C1000181C41F40051C0F8181C016841F008017B
:101C20000160704702F001031BB1D0F800340B4390
:101C300002E0D0F800348B43C0F8003402F0020315
:101C40001BB1D0F820340B4302E0D0F820348B4392
:101C5000C0F8203470470000F0B55F4D2D685F4E2E
:101C600035405F4EB5421AD0002416E00125A5404C
:101C70000D4085B1D0F8C45F67000326BE40B54370
:101C8000C0F8C45FD0F8C45F6700C2F34116BE401D
:101C90003543C0F8C45F651CECB2082CE6DB02F0EB
:101CA00001051DB1D0F800550D4302E0D0F80055F4
:101CB0008D43C0F8005502F002051DB1D0F804555F
:101CC0000D4302E0D0F804558D43C0F8045502F0EE
:101CD00004051DB1D0F808550D4302E0D0F80855B1
:101CE0008D43C0F8085502F008051DB1D0F818550D
:101CF0000D4302E0D0F818558D43C0F81855364D05
:101D00002D68364E3540364EB5420BD002F01005E8
:101D10001DB1D0F83C550D4302E0D0F83C558D4341
:101D2000C0F83C5503F001051DB1D0F80C550D432A
:101D300002E0D0F80C558D43C0F80C5503F00205B5
:101D40001DB1D0F810550D4302E0D0F810558D4369
:101D5000C0F8105503F004051DB1D0F814550D431B
:101D600002E0D0F814558D43C0F8145503F008056F
:101D70001DB1D0F81C550D4302E0D0F81C558D4321
:101D8000C0F81C55144D2D68144E3540144EB54204
:101D900017D003F400751DB1D0F844550D4302E08F
:101DA000D0F844558D43C0F8445503F440751DB137
:101DB000D0F840550D4302E0D0F840558D43C0F8AF
:101DC00040551BB9D0F828550D4302E0D0F82855EE
:101DD0008D43C0F82855F0BD00E00F400000FF70B3
:101DE0000000051010B50146C1F307400F4BDB6E34
:101DF00001248440234033B1012303EB40030C4C06
:101E000054F8230003E04300094C54F82300C1F3C5
:101E10000722D0F82C350F249440A34301F00F047F
:101E200094402343C0F82C3510BD000000E00F4063
:101E3000A0DA000030B504460D46022229462046AD
:101E4000FFF7F0FE0823662229462046FFF704FF2D
:101E500030BD30B504460D46022229462046FFF724
:101E6000E1FE0923012229462046FFF7F5FE30BD99
:101E700030B504460D46022229462046FFF7D2FE21
:101E80000823012229462046FFF7E6FE30BD30B583
:101E900004460D46022229462046FFF7C3FE0823CA
:101EA000012229462046FFF7D7FE30BD014648688B
:101EB00000F0010008B1012070470020FCE74160FC
:101EC000704701468868704781607047016A41F039
:101ED0001001016270470246516801F0010008B12B
:101EE0000020704701F0120010B101F01C00F8E76B
:101EF0000020F6E770B503460C4616461846FFF775
:101F0000E5FF012E01D10F4A00E00F4A142000FB2B
:101F10000240401E02EB82018900B0FBF1F0451E39
:101F2000DD60D3F8C00F00F0010048B1074820443D
:101F3000401E0649B0FBF1F0451E45F08000D86018
:101F400070BD0000801A0600A0860100804737019E
:101F500042EA410303607047016A41F020010162D7
:101F60000121C0F80418704700B502460B46104620
:101F7000FFF7F2FFC2F8003800BD000010B50024E2
:101F800026E0002004EBC4014A4A02EB810108620A
:101F900004EBC40102EB8101486004EBC40102EBD5
:101FA00081018860172C01D1104605E0601C00EB10
:101FB000C000404901EB800004EBC4013D4A02EB44
:101FC0008101C8603C4804EBC40142F82100641C54
:101FD000182CD6D3002039498860C860002459E005
:101FE000032240F2EC51104606F036FA04EBC4012D
:101FF000334A02EB810108624FF4804004EBC401D4
:1020000002EB8101486004EBC400114601EB800043
:10201000006A18B304EBC40001EB8000006A40685A
:1020200004EBC40102EB8101886004EBC40011469B
:1020300001EB8000406804EBC40102EB8101096AF6
:102040004989084304EBC40102EB810148604FF069
:10205000004004EBC40142F821000AE0002004EB38
:10206000C401174A02EB8101886004EBC40142F805
:102070002100072C01D1124805E0601C00EBC000D4
:102080000F4901EB800004EBC4010D4A02EB810112
:10209000C860641C082CA3D3002008498860C8606D
:1020A00007490848FFF79AFD02490648FFF7A8FDCF
:1020B00010BD000018CF01200000D04020010020FA
:1020C00078D2012000C00E40042806D119490968C1
:1020D00041F48031174A11602BE0052806D11549DB
:1020E000096841F40031134A116022E0062806D144
:1020F0001049096841F480210E4A116019E00F2847
:1021000008D14FF0E021096941F002014FF0E022CF
:1021100011610EE010280CD3A0F1100101F01F0294
:1021200001219140A0F110025209034B53F82220E3
:102130001160704724ED00E0ECDB000010B5FEF705
:1021400070F808B1012010BD0020FCE710B50A4668
:1021500083080A4C54F8233019688307DC0EFF23E8
:10216000A34099438307DB0E02FA03F31943830864
:10217000024C54F82330196010BD000050DB000001
:1021800030B505460C4622460021284600F026F8C8
:1021900030BD00000D480E4901600146416000213C
:1021A0008160C160016141618161C161016201635E
:1021B000C162416207498163C1634FF48061016478
:1021C00041640146044A116070470000E8010020A4
:1021D0004845415030020020040000202DE9F04124
:1021E00003460C4617460FB9BDE8F08103B9FBE77B
:1021F0000025002202E02D022543521C042AFAD3B6
:10220000384603F0030C1946BCF1000F08D06246B3
:1022100003E001F8014B401E521C08B1042AF8D318
:102220000E4601E020C6001F0428FBD2314602E022
:1022300001F8014B401E0028FAD100BFD4E700008E
:102240001D481E481E481F481F4820482048214856
:102250002148224822482348234824482448254826
:1022600025482648264827482748284828482948F6
:1022700029482A482A482B482B482C482C482D48C6
:102280002D482E482E482F482F4830483048314896
:102290003148324832483348334834483448354866
:1022A0003548364836483748374838483848394836
:1022B000394800BF704700003CDD000040DD0000F1
:1022C00046DD000048DD000044DD00004ADD00007E
:1022D0004CDD00004EDD000050DD000052DD00004E
:1022E00054DD000056DD000058DD00005ADD00001E
:1022F0005CDD00005EDD000060DD000062DD0000EE
:1023000064DD000066DD000068DD00006ADD0000BD
:102310006CDD00006EDD000070DD000072DD00008D
:1023200074DD000076DD000078DD00007ADD00005D
:102330007CDD00007EDD000080DD000082DD00002D
:1023400084DD000086DD000088DD00008ADD0000FD
:102350008CDD00008EDD000092DD000094DD0000C9
:1023600096DD000098DD0000F81B0020782000209A
:102370009CDD00009EDD0000A0DD0000A2DD00006D
:10238000A4DD0000A6DD0000A8DD0000AADD00003D
:10239000ACDD00009ADD0000AEDD00002DE9F0416B
:1023A00005460E46144600271148007818B1122041
:1023B0002070BDE8F0812878012808D0022807D0D5
:1023C000032802D0042804D100E000BF00BF00BFF2
:1023D00002E001202070ECE700BFFDF763FF074635
:1023E0006E613846FDF762FF0020207000BFE0E715
:1023F0002100002010B500F019F801F0ABFB01F04E
:10240000D7FB01F0F7FB01F075FB01F035FB01F0A4
:102410008BFC01F0B5FC01F02DFC01F053FC01F048
:10242000FBF800F01FF8FFF70BFF10BD09488021F3
:1024300002E0491E002204C00029FAD1064A074BD7
:102440001A601A46126822F007021A600022044B32
:102450001A807047B8200020B82200206C000020AD
:10246000700000207047000010B50024FDF71AFF2F
:10247000044608480078012808D107480078FF285A
:1024800004D205480078401C034908702046FDF737
:102490000DFF10BD2E0000202100002010B50024EB
:1024A0001A480078012830D1FDF7FCFE0446184890
:1024B000007820B116480078401E1549087014486D
:1024C0000078F8B913480078E0B901F0BBFC124875
:1024D0001249097850F82100114908600F48007826
:1024E0001049097888420DD00D480068C06B401C27
:1024F0000B490968C8630C480068401C0A49086019
:10250000FDF7F0FE2046FDF7D1FE10BD2E000020A5
:102510002100002022000020901200202400002032
:102520003C00002023000020080000202DE9FC5F73
:1025300005460F4691469A4600200090FDF7B2FEF0
:10254000009018480468006820B116480068406888
:10255000144908600098FDF7A9FE2CB95A208AF8A2
:1025600000000020BDE8FC9FA8462E46781E019082
:102570004FF0000B05E04E44C8F80060B0460BF188
:10258000010B01988345F6D30020C8F800002560B0
:1025900065602761E760C4F808908AF8000020466B
:1025A000E0E70000480000202DE9F04104460D4618
:1025B0000027FDF777FE0746206968B16668306836
:1025C00060602069401E20613846FDF76FFE0020E4
:1025D00028703046BDE8F0813846FDF767FE5D2083
:1025E00028700020F6E770B504460D460026FDF77A
:1025F00059FE0646D4E90310884204D33046FDF75D
:1026000055FE5E2070BD6068286065602069401CD2
:1026100020613046FDF74AFE0020F3E72DE9F04146
:1026200006460F464FF000082048007810B1002001
:10263000BDE8F081FDF736FE80461D48046800685D
:1026400020B11B4800684068194908604046FDF702
:102650002DFEFCB1FDF726FE804616480568D5B173
:1026600000680068134908604046FDF71FFE6E6071
:1026700006EB8700A860EE602E61AF820020E88242
:10268000022020700020208165600BA06061204640
:1026900001F0E4F908E0064800686060044804605E
:1026A0004046FDF703FE00242046C1E7210000203C
:1026B0000C0000204C0000203F0000002DE9F047F6
:1026C0000446894615464FF0000A2078022804D0B7
:1026D000012028702046BDE8F0873548007818B101
:1026E0000F2028702046F6E7FDF7DCFD8246A07A31
:1026F00010B14FF0010801E04FF00008B9F1000FF0
:1027000003D0B9F1010F49D121E0B8F1000F17D181
:1027100028A0606166682848006830602648066026
:102720000020207025480068606000202081234838
:1027300004605046FDF7BAFD00202870002705E030
:102740005046FDF7B3FD4920287027462DE005E0EF
:10275000022304220021204601F0C6F8A07A0028B6
:10276000F6D114A0606166681348006830601248B2
:102770000660002020701148006860600020208101
:102780000E4804605046FDF791FDB8F1010F01D1EC
:1027900001F01EFB00202870002706E05046FDF7E0
:1027A00085FD07202870274600BF00BF384692E706
:1027B000210000203F0000004C0000200C00002001
:1027C00070B505460026FDF76DFD06466C6860682D
:1027D000E060606820610020E0823046FDF766FD21
:1027E000002070BD2DE9F0470746884615464FF09A
:1027F00000093878022804D0012028700020BDE8A4
:10280000F0873E48007818B1022028700020F6E7D3
:102810003B48007818B10D2028700020EFE7FDF745
:1028200041FD81467C68E08A98B12169081D2061DC
:102830000E68E08A401EE082A1682069884201D1CA
:10284000606820614846FDF731FD00202870304661
:10285000D5E72C48006890F8340040F0040029497E
:10286000096881F8340000202649096881F835009C
:1028700024480068C0F83080384601F0B1F8484676
:10288000FDF714FD01F0A4FAFDF70CFD81461D488B
:10289000006890F8350020B101280DD002280AD137
:1028A00005E018480068466A002028700DE0002600
:1028B0000E20287009E000BF39461248006801F078
:1028C0005BF800260A20287000BF00BF00200D49D9
:1028D000096881F834000B49096881F83500094915
:1028E0000968C861074909680862064909684862B9
:1028F0004846FDF7DBFC304681E700002100002060
:1029000022000020340000202DE9F04105460E464B
:1029100000272878022802D00120BDE8F081FDF7C9
:10292000C1FC0746A87A60B100230422314628463C
:1029300000F0DAFF3846FDF7B9FC01F049FA002053
:10294000EBE76C68E08AA18A884204DB3846FDF731
:10295000ADFC1E20E1E7E168081DE0600E60E08A42
:10296000401CE082D4E90210884201D16068E06036
:102970003846FDF79BFC0020CFE72DE9F0470546E0
:102980000C464FF0000A2878022802D00120BDE84A
:10299000F087FDF787FC8246A87A207405F10B08C2
:1029A00004F10809002705E018F8010B09F8010BEC
:1029B000781CC7B2082FF7D36E68F08A18B1306957
:1029C0000068206001E000202060F08AA080B08ACA
:1029D000E0805046FDF76AFC0020D8E710B50024DF
:1029E0000B480078012811D1FDF75CFC044609482A
:1029F000007840B908480078FF2804D206480078DB
:102A0000401C054908702046FDF750FC10BD000031
:102A10002E000020210000202200002010B50024FC
:102A200013480078012821D1FDF73CFC04461148E9
:102A30000078C0B91048007888B10F480078401E6F
:102A40000D4908700846007828B92046FDF72EFC8D
:102A500001F0BEF90AE02046FDF728FC06E020461A
:102A6000FDF724FC02E02046FDF720FC10BD00002D
:102A70002E000020210000202200002070B5054615
:102A800000261048007808B1002070BDFDF70AFC50
:102A900006460D480468006820B10B48006840688D
:102AA000094908603046FDF701FC4CB10320207055
:102AB00025810020606005A06061204600F0CEFF07
:102AC0002046E2E7210000200C0000203F0000002B
:102AD0002DE9F0470446884615464FF00009207856
:102AE000032804D0012028702046BDE8F0872D4837
:102AF000007818B10F2028702046F6E7FDF7D2FBCA
:102B00008146A07A08B1012700E00027B8F1000F44
:102B100003D0B8F1010F3AD119E08FB922A060615A
:102B200000202070214800686060002020811F483C
:102B300004604846FDF7BAFB00202870002605E037
:102B40004846FDF7B3FB49202870264626E005E0FD
:102B5000022301220021204600F0C6FEA07A0028B0
:102B6000F6D111A0606100202070104800686060FC
:102B7000002020810D4804604846FDF797FB012F97
:102B800001D101F025F900202870002606E0484612
:102B9000FDF78CFB07202870264600BF00BF30469B
:102BA000A3E70000210000203F0000000C000020EF
:102BB0002DE9F04105460E461446002728780328E3
:102BC00003D001202070BDE8F0813248007810B1B8
:102BD00002202070F7E73048007810B10D202070F7
:102BE000F1E7FDF75FFB0746288940B12889401EC1
:102BF00028813846FDF75AFB00202070E3E727487C
:102C0000006890F8340040F001002449096881F818
:102C1000340000202149096881F835001F48006808
:102C20000663284600F0DCFE3846FDF73FFB01F066
:102C3000CFF8FDF737FB07461848006890F83500D5
:102C400020B1012809D0022806D102E0002020701E
:102C50000BE00E20207008E000BF29460F480068F6
:102C600000F08AFE0A20207000BF00BF00200B4940
:102C7000096881F834000949096881F83500074975
:102C80000968C8610549096808623846FDF70EFB06
:102C900000BF98E72100002022000020340000201F
:102CA00070B5044600252078032801D0012070BDAE
:102CB000FDF7F8FA0546A07A60B100230122194613
:102CC000204600F011FE2846FDF7F0FA01F080F8EA
:102CD0000020ECE720894FF6FF71884207D2208957
:102CE000401C20812846FDF7E1FA0020DFE7284656
:102CF000FDF7DCFA3320DAE72DE9F04704460D460C
:102D00004FF000092078032802D00120BDE8F087A9
:102D1000FDF7C8FA8146A07AA87204F10B0705F105
:102D20000208002605E017F8010B08F8010B701CDB
:102D3000C6B2082EF7D3208928804846FDF7B6FA98
:102D40000020E3E710B50B48007890B901F07AF85D
:102D5000094800780949087009480749097850F876
:102D60002100084908600846006807490860FDF727
:102D7000A0FA10BD2E000020240000202300002017
:102D8000901200203C0000203400002010B50024E8
:102D9000022000F035FBFDF785FA044600200B49C0
:102DA00008602046FDF782FA642000F029FBFDF759
:102DB00079FA04460548006805490860012005497C
:102DC00008702046FDF772FA10BD000030000020A8
:102DD000180000202000002010B504462046FDF712
:102DE00025FC10BD2DE9F04F85B081468A469346FB
:102DF0001C46DDE90F78129D00200390FDF752FA82
:102E000003902348007830B10398FDF74FFA3C2037
:102E100005B0BDE8F08F1F4850F8240088BB0120A2
:102E20001C4941F824000398FDF740FA2A46414620
:102E3000384601F04BF92B465A465146484600F0B9
:102E400073F904901198CDE9008002953A46204626
:102E50000E9B049901F00CF8064636B90E4800782E
:102E600001280CD100F0B4FF09E0FDF71BFA039034
:102E70000020084941F824000398FDF717FA30466E
:102E8000C6E7FFE70398FDF711FA2820C0E7000026
:102E900021000020901200202E00002010B50446D2
:102EA0002046FDF7C4FB10BD2DE9F0410546002783
:102EB0004A48007810B14020BDE8F0813F2D01D193
:102EC0003E20F9E7FDF7EEF90746FF2D03D1444810
:102ED000006890F83650434850F8254024B93846E9
:102EE000FDF7E4F94320E7E7012C04D13846FDF76C
:102EF000DDF93D20E0E714F8380F3B49085C6178C4
:102F000088432178384A505414F838091146085C2F
:102F100030B994F83A10354800788843334908703E
:102F2000E06918B12046E16900F026FD206A18B179
:102F30002046216A00F037FDA66A16B1304600F03F
:102F4000C7FD0020206384F8340084F83500284849
:102F50000078FF2804D226480078401C24490870D5
:102F60003846FDF7A3F900F0BDFCFDF79BF90746D5
:102F70001F48007820B11E480078401E1C49087088
:102F8000204600F041F81B480078401E194908709F
:102F90000020144941F82500A06930B9002061697A
:102FA000886115496069086005E0D4E90501486158
:102FB000D4E9051088611148006860610F48046019
:102FC0000FA020653846FDF771F90E4800780128FA
:102FD00001D100F0FDFE00206EE70000210000207E
:102FE0003400002090120020260000202500002040
:102FF000220000202F000020400000203800002088
:103000003F0000002E00002010B504462046FDF7CA
:103010000FFB10BD10B5FDF70CFB10BD2DE9F04105
:1030200006460F4614464FF000081548007818B1C0
:1030300012202070BDE8F081FDF734F98046FF2EA4
:1030400003D11048006890F836600F4850F82650B9
:103050002DB94046FDF72AF943202070EAE7012DFB
:1030600005D14046FDF722F943202070E2E72F65A5
:103070004046FDF71BF90020207000BFDAE7000092
:1030800021000020340000209012002010B50446DA
:103090002046FDF7CFFA10BD10B5FDF7CCFA10BDF4
:1030A0002DE9F04707460D464FF0000A0020286042
:1030B0006860FDF7F7F88246FF2F03D118480068D3
:1030C00090F83670174850F827402CB95046FDF755
:1030D000EDF84320BDE8F087012C04D15046FDF700
:1030E000E5F84320F6E7207C00F0010020B95046C7
:1030F000FDF7DCF84520EDE70026D4F80C90D4F875
:1031000008805046FDF7D2F800E0761C58F8041B02
:103110000029FAD02E60A9EB060068600020D9E7EC
:10312000340000209012002070B50446101D20F0DD
:1031300007004FF08076051F28462E60051F2846A1
:103140002C60684E051F28462E604FF01236051F72
:1031500028462E604FF00336051F28462E604FF09C
:103160000236051F28462E607610051F28462E6061
:10317000051F284629604FF01136051F28462E608E
:103180004FF01036051F28462E604FF00936051FF8
:1031900028462E604FF00836051F28462E604FF057
:1031A0000736051F28462E604FF00636051F2846B5
:1031B0002E604FF00536051F28462E604FF004366E
:1031C000051F28462E6003F00405002D7ED0F6056D
:1031D000051F28462E60444E051F28462E60434E8C
:1031E000051F28462E60424E051F28462E60414E80
:1031F000051F28462E60404E051F28462E603F4E74
:10320000051F28462E603E4E051F28462E603D4E67
:10321000051F28462E603C4E051F28462E603B4E5B
:10322000051F28462E603A4E051F28462E60394E4F
:10323000051F28462E60384E051F28462E60374E43
:10324000051F28462E60364E051F28462E604FF07B
:103250008346051F28462E60324E051F28462E60E5
:10326000314E051F28462E60304E051F28462E6021
:103270002F4E051F28462E602E4E051F28462E6015
:103280002D4E051F28462E602C4E051F28462E6009
:103290004FF08246051F28462E60294E051F2846FE
:1032A0002E60284E051F28462E60274E051F2846F3
:1032B0002E604FF08146051F28462E60234E051FC5
:1032C00028462E603602051F284600E009E02E60E1
:1032D0004FF07E56051F28462E600026051F284603
:1032E0002E6070BDD93F00000000F8410000F041A1
:1032F0000000E8410000E0410000D8410000D0415A
:103300000000C8410000C0410000B8410000B041C9
:103310000000A8410000A041000098410000904139
:1033200000008841000070410000604100005041F1
:1033300000004041000030410000204100001041E9
:103340000000E0400000C0400000A04000004040FD
:103350002DE9F04105464FF00008FCF7A3FF804639
:10336000FF2D05D12048006890F83650012608E06E
:103370001D48006890F83600A84201D1012600E0FF
:1033800000261A4850F825402CB94046FCF78EFF1D
:103390004820BDE8F081012C04D14046FCF786FFAF
:1033A0004320F6E794F838701148C05D94F839105E
:1033B00088430F49C8550846C05D30B994F83A10A3
:1033C0000C48007888430B49087094F8340040F0AA
:1033D000080084F834004046FCF768FF012E01D154
:1033E00000F0F6FC0020D4E734000020901200200A
:1033F000260000202500002010B5FDF71DF910BDA6
:1034000070B5054600261748007800B170BD164813
:10341000007800B1FAE71DB3FCF744FF06461348F5
:10342000006890F838401248005D1049096891F82A
:10343000391088430E4908550846005D40B90B48CD
:10344000006890F83A100B480078884309490870E2
:103450000648006805633046FCF728FF00F0B8FC1A
:1034600000BFD3E72100002022000020340000200C
:1034700026000020250000202DE9F04105460E46DB
:1034800017461C461248007810B15520BDE8F0815F
:103490001048007808B13220F8E74FF47A706043A2
:1034A0004FF47A71B0FBF1F14FF461606843C6EB01
:1034B000061200EB8200384400EB4002C2EBC01061
:1034C00001EBC0084046FFF79BFF0020DEE700004D
:1034D000210000202200002070B50025FCF7E2FE4C
:1034E0000546034804682846FCF7E0FE204670BD08
:1034F0005400002070B5002600F072F8FCF7D2FEF0
:10350000064631480068401C2F4908603046FCF7E9
:10351000CDFE2E480078012853D12D48007820B1E7
:10352000012804D0022809D103E001250BE0002581
:1035300009E0012501202649087004E0012500204A
:103540002349087000BF00BF05B970BD2148046859
:1035500033E0FCF7A7FE0646206B50B3206B401EFD
:103560002063206B28BB94F8340000F0370040B192
:1035700014F8340F00F0C800207001206070343C53
:1035800002E0002084F8350094F8340000F00800D0
:1035900078B93834A0781049097808430E49087082
:1035A00020780E49085C6178084314F838190B4AF2
:1035B000505464693046FCF779FE94F836003F2891
:1035C000C7D100BFC1E70000540000202E0000203A
:1035D000440000204000002025000020260000209C
:1035E00010B5FDF72AF806480088401C04490880F9
:1035F0000846008818B10020088000F003F810BDCC
:103600007000002010B503480068FFF749FB04462E
:10361000204610BD64000020F8B54FF42071284802
:1036200000F078FB4021274800F074FB002514E0EF
:10363000681C86B205EB8500214901EBC00406EB4E
:10364000860001EBC00764202070002084F825006C
:10365000E7601DA02062681C85B20F2DE8D305EB42
:103660008500174901EBC00464202070002084F815
:103670002500E06014A0206200201449086014496D
:1036800008801020134908800D4813490860012064
:10369000FFF7F4F9114908600020FFF7EFF910492E
:1036A00008606A460FA10D480068FEF777FE6A467B
:1036B00011A10B480068FEF771FE00F027F8F8BD75
:1036C000F81B0020782000203F0000005C00002054
:1036D0005A000020580000206800002060000020F0
:1036E0006400002075432F4F532D494920546D72BB
:1036F0004C6F636B0000000075432F4F532D4949F9
:1037000020546D725369676E616C000000B587B01C
:103710000320002180220A4BCDE90132CDE90310BC
:103720004FF6FD703D23074A00900748FFF75AFB0C
:1037300006AA06A13D20FFF771FC07B000BD0000FE
:10374000781E002074200020C937000075432F4FD9
:10375000532D494920546D720000000070B50B468E
:10376000032580F82550012B05D1154EC569366813
:10377000354445610CE085692DB9114EC56936683F
:103780003544456104E00E4E85693668354445612F
:10379000057D05F007040B4D05EBC4010D682DB93F
:1037A00008600025C56001258D8006E00A68086074
:1037B000C26010618D886D1C8D800025056170BD13
:1037C0005C0000207820002008B500BF00BF6A46DA
:1037D00000211A480068FFF7EBF9FFF7FFF81848D7
:1037E0000068401C164908600846007800F0070889
:1037F000144800EBC8073C681AE0E66810496069A5
:103800000968884213D1204600F01EF894F824007D
:10381000022804D101212046FFF7A0FF02E0022088
:1038200084F82500656815B12046A168A84734468C
:10383000002CE2D1FFF7F2F8C9E700006400002095
:103840005C0000207820002030B5057D05F00704DD
:103850000D4D05EBC4031D68854205D1C168196093
:1038600039B100250D6104E00169C268CA6002B186
:103870001161012580F825500025C56005619D88EE
:103880006D1E9D8030BD00007820002010B5FCF733
:1038900009FD044606480078401C0549087020468A
:1038A000FCF704FDFFF726FEFEF7F8FD10BD000053
:1038B0002100002001464A1E4FF0E0235A61084AC9
:1038C000106820F07F4000BF10601A46126942F075
:1038D00005021A611A46126942F002021A61704723
:1038E00020ED00E0704700002DE9F04F05460F463F
:1038F00090469946A87A1C490E5C05F10B00805D44
:1039000011F800B00BEBC60000F0FF0A174850F8A2
:103910002A4000202434E0602760207C20EA080050
:10392000207484F81190207C243C00F0080068B9D1
:1039300094F83A000E49097808430D4908700D487B
:10394000805D94F8391008430A4988552946204675
:1039500000F012F8206A20B12046216A00F023F816
:10396000E5615046BDE8F08F3CDC0000901200207D
:10397000250000202600002010B590F8382001F125
:103980000B039B5C90F83940A34301F10B04A35453
:1039900023469B5C23B98B7A90F83A40A3438B7201
:1039A0000023C36110BDF0B5024612F8384F957878
:1039B0005678383A0B4618680FE000F10B073F5D68
:1039C000B74300F10B0C0CF8047067463F5D17B964
:1039D000877AAF4387721B1D18680028EDD1F0BDB0
:1039E00010B51B4A1268D061194A126892F8383033
:1039F00000F10B02D25C164B1B6893F839301A4366
:103A0000134B1B6893F8384000F10B031A55827A68
:103A10000F4B1B6893F83A301A4382720C4A1268B3
:103A200092F838100B4A525C094B1B6893F83930F6
:103A30009A43084B5A541A46525C42B9044A1268D7
:103A400092F83A30044A12789A43034B1A7010BD28
:103A5000340000202600002025000020014600221E
:103A60008A72002005E0002301F10B021354421C6E
:103A7000D0B20828F7D370472DE9F041A0211148B2
:103A800000F048F900250DE0681C86B20D4800EBF7
:103A9000051400EB06170020207067600AA0E060A4
:103AA000681C85B2092DEFD3064800EB05140020F1
:103AB0002070606004A0E060024804490860BDE82E
:103AC000F0810000F00D00203F00000010000020F9
:103AD00030B501464A6808682AB9CC68606028B1E8
:103AE0000025456002E0106000B142608B6800254F
:103AF0009D6230BD70B54FF4C061134800F00AF903
:103B0000002411E0601C85B204EB44000E4901EB77
:103B1000C00305EB450001EBC006002018705E6095
:103B20000AA05861601C84B23F2CEBD304EB440024
:103B3000054901EBC00300201870586003A05861CC
:103B400008460349086070BDF00700203F000000F0
:103B50000C00002000200B4908600B4908700B493D
:103B600008700B4908700B4908700B4908600B4935
:103B700008600B4908600B4908600B4908700B4945
:103B8000087070475400002021000020220000200F
:103B90002F0000202E000020080000203000002010
:103BA0001C000020180000202000002050000020F1
:103BB00000210A4A1170002004E00021084A115433
:103BC000411CC8B20828F8D30021064A1170064AE1
:103BD0001170064A1160064A1160704725000020E6
:103BE0002600002023000020240000203C000020AC
:103BF0003400002070B54FF4F261194800F08AF8E3
:103C00004FF48071174800F085F8002413E0601C21
:103C1000C5B204EB440000EBC400114901EBC00342
:103C200005EB450000EBC50001EBC0065E610EA090
:103C30001865601CC4B2152CE9D304EB440000EBFA
:103C4000C400074901EBC0030020586106A01865B5
:103C500000200649086002480549086070BD000060
:103C600090130020901200203F0000004000002030
:103C70003800002000B587B00320002180220A4BC5
:103C8000CDE90132CDE903104FF6FF703F23074A1B
:103C900000900748FFF7A6F806AA06A13F20FFF705
:103CA000BDF907B000BD0000901000208C1200206C
:103CB000B13F000075432F4F532D49492049646C93
:103CC0006500000000B587B00320002180220A4B68
:103CD000CDE90132CDE903104FF6FE703E23074ACD
:103CE00000900748FFF77EF806AA06A13E20FFF7DE
:103CF00095F907B000BD0000900E00208C10002048
:103D0000F13F000075432F4F532D494920537461F3
:103D10007400000004E0002200F8012B4A1E91B25A
:103D20000029F8D17047000070B578211148FFF7DD
:103D3000F1FF00240EE004EB44000E4901EBC00546
:103D4000601C00EB400001EBC00068600AA06861E5
:103D5000601C84B2042CEED304EB4400054901EB53
:103D6000C0050020686004A0686108460349086037
:103D700070BD0000201B00203F0000004800002014
:103D80002DE9F04160211048FFF7C4FF00240DE049
:103D9000601C86B204EB44000B4901EBC00506EB46
:103DA000460001EBC0072F60601C84B2032CEFD3E8
:103DB00004EB4400044901EBC005002028600846DC
:103DC00002490860BDE8F081981B00204C000020EB
:103DD00010B50024FCF766FA044613480078F8B9D9
:103DE00012480078E0B900F02DF81148114909781F
:103DF00050F82100104908600E4800780F490978F2
:103E000088420DD00C480068C06B401C0A49096804
:103E1000C8630B480068401C09490860FCF75DFA5C
:103E20002046FCF743FA10BD2100002022000020AC
:103E300090120020240000203C00002023000020DD
:103E4000080000200649074A1278885C0649095C88
:103E5000034A515C01EBC001044A11707047000035
:103E60003CDC00002500002026000020240000206B
:103E70002DE9F84F05460F4690469946DDE90AAB15
:103E800000200090FCF70EFA009042480468002CD5
:103E90007BD01C3454F8080C3E4908600098FCF7AD
:103EA00005FA44F81C7CA5760020207660766061D7
:103EB00044F818BC44F810AC44F8148C0C9824F85E
:103EC0000C0C24F80A9C0020E077E810207705F01D
:103ED0000700E076217F01208840A077E17E012065
:103EE00088406077002020606060E060A060206211
:103EF000A0626062E062206327A060631C3C002631
:103F000006E0002104F1540040F82610701CC6B2EF
:103F1000002EF6D02046FEF75FFFFCF7C3F90090B5
:103F20001E4840F825400098FCF7C0F92046FEF7EF
:103F3000B5FFFCF7B7F900901948006860610020F0
:103F4000A0611748006810B11548006884611448E2
:103F500004603834A078134909780843114908707F
:103F600020781149085C6178084314F838190E4A22
:103F700050540E480078401C0C4908700098FCF71B
:103F800095F90020BDE8F88FFFE70098FCF78EF95F
:103F90004220F7E7380000203F0000009012002088
:103FA0004000002025000020260000202F000020D7
:103FB000002400BF00BFFCF775F9044605480068FF
:103FC000401C044908602046FCF770F9FFF722F80E
:103FD000F1E700003000002010B504480068FFF74A
:103FE00055F8FF20FEF760FF10BD000034000020F0
:103FF00000BF00BF02E0C820FFF702FA1F480078A8
:104000000028F8D01E4800686421B0FBF1F01C497C
:1040100008600846006828B900201A490870FF2087
:10402000FFF796F9FCF73EF904461548006864214D
:104030004843154908602046FCF738F900BFFCF7F3
:1040400031F90446104800681049086000200E4904
:1040500008602046FCF72AF90C48006808490968FE
:10406000B0FBF1F0C0F1640006490870FFF714F8E6
:1040700000F00EF86420FFF7C3F9E0E7200000200D
:104080001800002014000020300000201C00002038
:104090007CB5002514E069462846FFF701F806467E
:1040A00066B9094850F8254044B1012C06D0D4E93E
:1040B000020100EB8100A0640198E064681CC5B2B5
:1040C0003F2DE8D97CBD00009012002002F00103D2
:1040D00043B102F002032BB102E0491E002308C0E5
:1040E0000029FAD1704700002DE9FC4104460D4635
:1040F0001646019400200090012301AA682115486A
:104100000078FCF70FFF07463846FDF771FA0028E4
:1041100003DA4FF0FF30BDE8FC8101236A466821D5
:104120000C480078FCF770FE07463846FDF760FA49
:10413000002802DA4FF0FF30EDE79DF8000000F0B4
:104140000F013040001100EB800001EB40002870AF
:104150000020E0E7B401002008E00548FDF7ACFAD4
:104160000023012219461846FFF786F9F5E70000FB
:10417000B5010020F8B504460D468DF800408DF8D5
:10418000015002236A46682103480078FCF7CAFE02
:104190000646FDF72DFAF8BDB40100202DE9F041E7
:1041A000AEB0804600220121022002F0BBFF06468D
:1041B00009E000220121022002F0B4FF06464FF47C
:1041C0007A7005F067F8002EF3DB00202A902B9020
:1041D0002C902D9002208DF8A900002002F020FDE7
:1041E0002B9041F2D71002F028FDADF8AA00102262
:1041F0002AA9304602F058FC002805DA304602F0C1
:104200009DFC2EB0BDE8F0810521304602F030FD66
:10421000002803DA304602F091FCF2E743E0102078
:10422000259025AA26A9304602F07EFB0546002DE2
:1042300000DA38E02AE0002005A90855072C1CD137
:10424000072219A105A8FCF7F7F8B0B9184840787B
:10425000009017488378C27816A102A800F0BEF932
:1042600002A8FCF7C7F8074600233A4602A92846E9
:1042700002F076FE002809DA10E00023224605A9A4
:10428000284602F06DFE002800DA07E000237F22B6
:1042900005A9284602F03AFD041ECCDC00BF2846E2
:1042A00002F04CFC00BFBAE747455420525443008B
:1042B000B5010020253032753A253032753A253067
:1042C0003275000070B504460D4616460CB9002044
:1042D00070BD0DB90020FBE721462A46002304E00B
:1042E00010780870491C521C5B1C21B11AB110785F
:1042F00008B1B342F4D301B10AB90020E8E7B342F0
:1043000001D2002008702046E2E710B502460B46B5
:104310001146002001E0491C401C19B10C780CB179
:104320009842F8D310BD000010B50121C0F3072258
:10433000094B1A4402F0704242F00072C0F30723A6
:10434000054C2344C3F3130342EA4312C3B242EAC7
:104350008302116010BD000000E60F400146C1F36A
:1043600007200B4A104400F0704040F00070C1F389
:104370000722074B1A44C2F3130240EA4210CAB2A2
:1043800040EA8200006808B1012070470020FCE785
:1043900000E30F400146C1F307200B4A104400F030
:1043A000704040F00070C1F30722074B1A44C2F37B
:1043B000130240EA4210CAB240EA8200006808B123
:1043C000012070470020FCE700EA0F4018B50121EA
:1043D000C0F30722184B1A4402F0704242F00072F8
:1043E000C0F30723144C2344C3F3130342EA4312DC
:1043F000C3B242EA830211600021009102E00099F9
:10440000491C009100991029F9D30021C0F307221B
:10441000094B1A4402F0704242F00072C0F30723C5
:10442000054C2344C3F3130342EA4312C3B242EAE6
:104430008302116018BD000000E50F400146886945
:1044400000F0100008B9086870474FF0FF30FBE734
:1044500000BF826902F02002002AFAD10160704791
:1044600001468869012222EA10107047F0B504461F
:104470000E4615461F46204600F01EF8B6EB051FF7
:1044800005D2206B40F0200020636D0803E0206B14
:1044900020F020002063F000B0FBF5F0401C430842
:1044A0009809606203F03F00A062E7620020A0610B
:1044B000204600F011F8F0BD00BF816901F008014D
:1044C0000029FAD1C16A21F01001C162016B40F2EA
:1044D0000132914301637047C16A41F01001C1622A
:1044E000016B40F201321143016370474164704730
:1044F000826B0A4382637047024609B1106C7047B1
:10450000D06BFCE72DE9F84F80460C4615461E4659
:10451000DDF84CB0DDE90C9A0E9F4046FFF704FF32
:104520002046FFF701FF0A98FDF75CFC0B98FDF7AA
:1045300059FC49EA0A00C1B23046FDF7A8FCFCF775
:1045400029FC0090129840EA0B00149940EA0103FC
:104550002846119A0099FFF789FFF8B20F99FCF7E6
:10456000DDFAF8B2FCF770F81098FDF7ADFD6021A8
:104570001098FDF7EBFD50212846FFF7B9FF00200A
:10458000BDE8F88F1FB51BE00E48407800900D483D
:104590008378C2780CA101A800F020F8002405E07F
:1045A00001A8015D0C48FFF753FF641C01A8005DE2
:1045B0000028F5D10023012219461846FEF75CFFBA
:1045C000E2E70000B5010020253032753A2530328F
:1045D000753A25303275000000D000400FB4084B0A
:1045E00010B504A902AA039800F01CF8044602A919
:1045F000002000F0B8F9204610BC5DF814FB000064
:104600006749000002E008C8121F08C1002AFAD159
:1046100070477047002001E001C1121F002AFBD142
:10462000704700002DE9FF4F8BB0884605460026F5
:1046300006E025280BD0DDE90D1290476D1C761C95
:1046400028780028F5D10FB03046BDE8F08F00245F
:10465000A146A2460122AE4900E0044315F8013FFD
:10466000203B02FA03F00842F7D128782A2810D01C
:104670006FF02F022878A0F13001092915D809EB35
:10468000890102EB410144F0020400EB01096D1CB9
:10469000F0E758F8041B5FEA010903D544F400541D
:1046A000C9F1000944F002046D1C28782E2817D1A6
:1046B00015F8010F44F004042A280ED06FF02F02E1
:1046C0002878A0F1300109290AD80AEB8A0102EB07
:1046D000410100EB010A6D1CF2E758F804AB6D1CB8
:1046E00028786C280FD006DC4C2817D068280DD00D
:1046F0006A2814D104E0742810D07A280FD10DE074
:1047000044F400140AE044F4801401E044F440143A
:104710006978814202D104F580146D1C6D1C2878E3
:10472000692865D006DC00288DD0632827D064284E
:1047300006D15DE06E2808D073282AD0752877D07E
:10474000DDE90D129047761CE0E0C4F30250022828
:1047500009D003280DD0D8F8001004280DD00E6021
:1047600008F10408D2E0D8F80010F217C1E900629D
:10477000F6E7D8F800100E80F2E70E70F0E718F8B0
:10478000041B8DF8001000208DF80100EB4601207D
:1047900003E058F804BB4FF0FF3061074FF000070B
:1047A00001D40AE07F1C57450DDA8742FADB1BF87B
:1047B00007100029F6D106E07F1C8742FCDB1BF8BE
:1047C00007100029F8D1DDE90D23A9EB0700814688
:1047D000214600F0B1F83044C61904E0DDE90D12BD
:1047E0001BF8010B90477F1EF8D22146484688E00F
:1047F00058F8040BC4F302514FF00A0B032900D1FF
:1048000000B2042900D140B2002802DA40422D2132
:1048100002E0210505D52B218DF82410012104E0AB
:1048200006E0E10710D02021F6E708AF089113E079
:1048300058F8040BC4F302514FF00A0B032900D1BE
:1048400080B2042900D1C0B20021EEE75946FBF73F
:1048500002FE303107F8011D0028F7D1ADEB07004B
:1048600000F1200B600702D524F4803401E04FF002
:10487000010ADA4502DDAAEB0B0000E000208246C7
:1048800000EB0B0108980144A9EB01000A90E0033A
:1048900006D4DDE90D2321460A9800F04DF80644C0
:1048A0004FF0000908E009A911F80900DDE90D122F
:1048B000904709F10109761C08998945F3DBE0036B
:1048C0000CD5DDE90D2321460A9800F035F80644A1
:1048D00004E0DDE90D1230209047761CBAF10001AA
:1048E000AAF1010AF5DC05E0DDE90D1217F8010B6C
:1048F0009047761CBBF10001ABF1010BF4DC0A9888
:104900002146DDE90D2300F005F806446D1C97E60D
:10491000092801002DE9F041044600251E461746EE
:10492000880404D405E039462020B0476D1C641E7D
:10493000F9D52846BDE8F0812DE9F041044600256F
:104940001E469046C80301D5302700E02027880482
:1049500004D505E041463846B0476D1C641EF9D5C4
:104960002846BDE8F0810A68531C0B601070704740
:104970002DE9F04706460F469046354605F11400EE
:1049800004F06CFC18B96FF00500BDE8F0872878DA
:10499000E96A03F0EDF8044614B94FF0FF30F4E78C
:1049A0006760204604F030FB84F80880214605F15A
:1049B000140004F03FFC30B3D4F8049000214846C2
:1049C00004F0D6FE0021484607F092F9002148463F
:1049D00007F02BFB04220021484606F081F9002154
:1049E000484605F0EDF90020606004F1100004F085
:1049F000D1FB04F1100004F019FC204603F0F5F996
:104A00004FF0FF30C1E7E86A20B100221146284686
:104A1000EB6A98470020B8E72DE9F04105460E46BD
:104A20000027002447E004F06AFB074604EB44003B
:104A3000234951F83000C8BB04EB440041F8305022
:104A4000384604F092FB002004EB44011C4A02EBC0
:104A5000C101486004EB440102EBC101088104EB91
:104A6000440102EBC10148812878102804D10EB11D
:104A7000012002E0002000E0012004EB4401104A84
:104A800002EBC1018881002004EB440102EBC1016B
:104A9000C88104EB440102EBC101086104EB44014D
:104AA00002EBC10148612046BDE8F081FFE73846CE
:104AB00004F05BFB641C082CB5DB4FF0FF30F3E720
:104AC000B822002010B5044601F036F80022034950
:104AD00041F2883004F062FC10BD0000C54A0000BD
:104AE00010B50446A4B91748FFF71EFC1648FFF797
:104AF0001BFC1648FDF776F91548FDF773F90421FC
:104B00001448FDF7B5F908211248FDF7A2F917E09E
:104B1000012C15D10B48401CFFF706FC0A48401D2C
:104B2000FFF702FC0C48FDF75DF90C48FDF75AF958
:104B300001210B48FDF79CF902210948FDF789F98D
:104B400010BD0000002000F0010800F00208010084
:104B5000020C0100005000400200060002040600A2
:104B60000060024010B50446206890F9080010F17A
:104B7000090F03DA2068007A207127E0FA202071FB
:104B80002068406810B32068007800F0F00010281A
:104B900012D0202808D0402816D12268A168506879
:104BA00003F0FDFF207110E0A2892368A168586816
:104BB00008F012FC207108E0A2892368A1685868F7
:104BC00004F0D8FD207100E000BF00BF10BD000060
:104BD0002DE9F047044600BF00BF00BF00BF00BF83
:104BE00000BF00BF00BF00BF00BFA06A067A06F08A
:104BF000010706F00208032E01D1012000E0002089
:104C00008146B9F1000F03D00021606804F0B0FDC7
:104C10006068007E012804D10021606804F009FD6D
:104C20001BE03FB10021606807F062F80021606876
:104C300004F0FFFCB8F1000F03D00021606807F01A
:104C4000F4F9B9F1000F08D004220021606806F0E1
:104C500047F80021606805F0B3F8B9F1000F04D0FF
:104C6000606804F0D3FD054605E0424639466068B9
:104C700007F0DFF9054635BB0020A16A0871A06284
:104C80006070B9F1000F07D06060E06A20B10022C7
:104C900004212046E36A984737B1E06A20B1002238
:104CA00011462046E36A9847B8F1000F06D0E06A43
:104CB00020B1002202212046E36A984704F10C004B
:104CC00004F021FB12E000BF00BF0949606807F053
:104CD000ACF904220749606806F002F806496068EA
:104CE00005F06EF82146606804F042FDBDE8F087EB
:104CF000A18F0000358B00001553000010B504464D
:104D00002068406810B9F420207158E020680078CD
:104D100000F0F000102812D0202808D0402846D1FA
:104D20002268A168506803F042FF207146E0A28922
:104D30002368A168586808F08FFB20713EE0206866
:104D4000407810B1F720207130E0206804F05CF961
:104D5000A2892368A16858681C4B04F049FE2071A1
:104D6000207918BB216891F82010C1F3400003217D
:104D70002268517000BF40B1216891F8201041F0C5
:104D80000401226882F8201007E0216891F82010C1
:104D900021F00401226882F8201000BF10B1FB212D
:104DA000217102E021688C6210BD00BF06E000BFE7
:104DB00000BFFA20207100BF00BF00BF00BF216804
:104DC00001F10C0004F09FFA00BFEDE7D14D0000A7
:104DD0002DE9F0470546894616462C461CB96FF06A
:104DE0000500BDE8F08700BF00BF00BF00BFA06A9C
:104DF00008B1A06A06712078102803D116B92046A0
:104E000004F002F994F82000012121EA900700BF84
:104E100094F8200020F0040084F8200000BF002057
:104E2000A06260707FB900BF804604F068F98046D8
:104E300094F9080010F1090F01DB002020724046B0
:104E400004F093F900BFE06A20B10022022120465D
:104E5000E36A98471FB104F10C0004F054FA0020F3
:104E6000BFE710B504462068407860B120684078FC
:104E7000022808D020684078032804D000BF00BF73
:104E8000FB20207141E000BF00BF206802F058FF06
:104E90002068406848B32068007800F0F0001028CF
:104EA00011D0202806D040281AD12168486803F084
:104EB000F7FE16E0002021684968C861216848684B
:104EC00008F064FC0DE000BF00BF042021684870BA
:104ED00003202072206884622068FFF779FE10BDED
:104EE00000BF00BF0020216848602068C06A20B170
:104EF000206800221146C36A98472068C06A20B122
:104F0000206800220221C36A9847216801F10C0041
:104F100004F0FFF920B1216801F10C0004F0F3F96D
:104F200000BFDCE710B504462068007800F0F00010
:104F3000202806D12168486808F0C0FA00202071B6
:104F400001E0FA20207110BD0168496800294AD0AB
:104F5000017C29B102688168526812680A6004E025
:104F600002688168526852680A6000210171016814
:104F7000097801F0F001102925D020290CD0402912
:104F80002DD1017C29B1016849680A7CC1680A8079
:104F900001E0F321017125E0017C29B10168496834
:104FA0004A8AC1680A800DE001684968097C01F0FD
:104FB000040111B9F321017104E0016849688A8A8A
:104FC000C1680A800EE0017C19B101684968498B0B
:104FD00002E001684968898BC268118002E000BF65
:104FE00000BF00BF01E0F3210171704770B50446B6
:104FF000206890F9080010F1090F03DA2068007AA0
:10500000207150E0F32020712068406800284AD0C9
:1050100020680078102844D120684078002842D1C8
:1050200021684868012105F0B3FA054615B9FF204B
:10503000207135E0216801F1100004F00FF948B14A
:10504000216801F1100004F0A5F8216801F11000B9
:1050500004F0ECF800202071216801F1140004F044
:10506000FDF830B9216801F11400042104F0A8F81A
:105070002071207970B9022021684870206845604D
:105080002168486804F074FB21684868064904F008
:10509000D0FA05E0284604F0B9FB002021684860FA
:1050A00001E0F220207170BD7149000010B5044686
:1050B000002020712068406810B9204603F0A8FC49
:1050C00010BD70B504460020207120684068B0B162
:1050D00020680078102812D1A56800BFB5F5803F80
:1050E00002D34FF6FF7000E0A8B206462168486878
:1050F000314606F019FEAD1B002DEFD100BF70BD8B
:1051000010B50446206890F9080010F1090F03DA81
:105110002068007A20713BE020680078102835D1A3
:105120002068407810B1FB20207131E02068406891
:1051300048B301202168487000BF00BF00BF00BF16
:1051400020688462002021684862206890F820006E
:1051500020F00100216881F82000206800F01CF890
:1051600080B100BF00BF0B4804F0CDF8216801F109
:105170000C00002103F0C7FF0021064803F0C3FF25
:1051800000BF00BF10BDF320207101E0FA202071A4
:1051900000BFF7E7880000202DE9F84F0446002003
:1051A000009094F8200000F0020020B9A06A007C72
:1051B00000F0040008B1012000E000200746A06ACA
:1051C00090F8108000BF00BF00BF00BF00BF00BF4D
:1051D00000BF00BF00BF00BFA06A8068616A00EB2B
:1051E000010BA06AC068616AA0EB010ABAF5803FB2
:1051F0000AD34FF6FF7694F8200040F0010084F8BF
:10520000200048F0020801E01FFA8AF66068B0F852
:105210006690B1450DDA4E461FB156B96FF00605DE
:1052200014E094F8200040F0010084F8200048F0D9
:10523000020800BF00BF434632465946606807F087
:105240007DF905460DB1681C30BB00BF8FB1A06A67
:10525000C068B0420DD9E06A20B132460321204631
:10526000E36A984794F8200040F0100084F820008A
:1052700012E06068B0F8660040F66931884204DDEB
:105280006068B0F86800082806DBE06A20B13246A2
:1052900003212046E36A98479DB9606A3044606202
:1052A000D4E90910C068814200D037B1D4E90910AF
:1052B000C1600120009000206062606805F07EFA05
:1052C00011E0681C50B94FB9606805F077FA94F89E
:1052D000200040F0010084F8200004E0012000904C
:1052E0000021A06AC160009870B1A06A0571002019
:1052F000A062607094F8200000F0010040B104F159
:105300000C0004F000F803E04FF0FF30BDE8F88F28
:105310000020FBE72DE9F04707460E464FF0000856
:105320003C4600BF00BF0020606003F0E8FE8046FE
:105330002672404603F019FF657800206070E06A2D
:1053400020B1002204212046E36A9847E06A20B198
:10535000002211462046E36A9847E06A20B1002205
:1053600002212046E36A984704F1100003F076FF1B
:1053700020B1002104F1100003F05CFF04F11400DF
:1053800003F06CFF20B1002104F1140003F052FF80
:10539000012D03D0042D01D0032D19D194F8200044
:1053A000C0F3800900BF94F8200020F0040084F8C6
:1053B000200000BFB9F1000F09D100BF00BFA06AF3
:1053C00006710020A06204F10C0003F09CFF01E0D4
:1053D00000BF00BFBDE8F0872DE9FC4705468846C1
:1053E000164600BF0DB9BDE8FC8700BF70892A28AA
:1053F0000EDA4B48408C401C81B249484184C08B36
:10540000401C81B24648C183304603F0F0F9EAE718
:10541000776807F10E042088B0F5807F08D12079E5
:10542000062805D16079042802D1608808280ED0AA
:105430003B48008D401C81B239480185C08B401C1F
:1054400081B23748C183304603F0D1F9CBE7344805
:10545000408B401C81B232484183D4F80E00019049
:10546000A0690090281D08B1686810B94FF00009C4
:1054700007E000986968884201D1012000E000201F
:105480008146B9F1000F01D0012000E0022003465F
:1054900004F1080201A9284600F094FBE088B0F569
:1054A000807F03D0B0F5007F2DD12BE0B9F1000F44
:1054B00026D0022001F0C1FBE080D4F80E00A061EC
:1054C0006868C4F80E0000BF00BFA068C4F81200EE
:1054D000A089E082A0683860A089B880D8F8000070
:1054E000A060B8F80400A081D8F80000C7F8060052
:1054F000B8F80400788131462846AA69904700E050
:1055000000BF07E006E00648808D401C81B20448D9
:10551000818500BF00BF304603F069F900BF62E734
:1055200060A601202DE9FC5F05460F464FF00A08F2
:10553000C1460A260024A34600200190B2460090EE
:1055400000BF5CE004EB84004D4A02EB8000817CEC
:105550000A2E02D109B966B24FE000294DD000BF32
:1055600000BF5DB104EB8402454B03EB8202286867
:105570005268904202D160B2BDE8FC9F012928D157
:1055800004EB84003E4A52F8200088B104EB84000A
:1055900002EB8000C27C009882422EDB4FFA84FA34
:1055A00004EB8400364A02EB8000C07C009024E0CB
:1055B00004EB8400324A02EB8000C07C58451CDBBF
:1055C0004FFA84F804EB840002EB800090F813B0EB
:1055D00013E0022911DB04EB8400294A02EB80006E
:1055E000C27C0198824208DB4FFA84F904EB840004
:1055F000234A02EB8000C07C0190601CC4B20A2CDC
:10560000A0DB07F0020020B90A2E05D107F0010047
:1056100010B94FF0FF30AFE70A2E01DAF4B21AE00A
:10562000B9F10A0F03DA09F0FF0400BF0EE0B8F188
:105630000A0F02DA08F0FF0408E0BAF10A0F02DAF2
:105640000AF0FF0402E04FF0FF3095E700BF00BF13
:10565000204600F017F800BF00BF00BF00BF35B103
:1056600004EB8401064A02EB8101286848600020AF
:1056700004EB8401024A02EB8101C87460B27BE74B
:1056800094A7012010B5044604EB84000C4951F89E
:10569000200060B104EB8401094A52F8210003F0B4
:1056A000A6F8002004EB8401054A42F821000020FE
:1056B00004EB8401024A02EB8101887410BD0000F2
:1056C00094A701202DE9FC4704460F461546A9463C
:1056D00000BF00BF00BF00BF00BF00BF0E213846A3
:1056E00003F0E9F840B14B484089401C49494881E2
:1056F0006FF00100BDE8FC872146286800F08DFDB1
:1057000010B1DFF814817DE0287800F0F000E02887
:1057100015D101208DF8000000208DF801005E20D9
:105720008DF80200687800F07F008DF80300A878FB
:105730008DF80400E8788DF80500E84661E02868F7
:10574000A1680840D4E901121140884210D028888D
:1057500080B24FF6A96188420AD004F10C0020B152
:10576000E06810B104F10C0902E06FF00300C1E73A
:105770002A48007800EB8000294901EB8000807CFA
:10578000022818DB2549097801EB8101244A02EB44
:105790008101D9F80000496888420CD11D48C08DAC
:1057A000401C81B21B48C1851C48027839462046FE
:1057B00000F038F89EE700261BE006EB860018494B
:1057C00001EB8000807C022811DB06EB8601144A85
:1057D00002EB8101D9F800004968884207D10F49DE
:1057E0000E70F2B23946204600F01CF882E7701CB9
:1057F00046B20A2EE1DB3A464946204600F048F818
:1058000078E700BF434604F12F023946204600F0F6
:1058100077F96FE760A6012070DF00001201002019
:1058200094A7012070B505460E46144600BF00BF80
:1058300004EB8400154901EB8000807C022817D11D
:1058400004EB840001EB8000C07CE42810DB04EB57
:1058500084000A4602EB8000011D284600F03AF958
:1058600030B9032004EB8401084A02EB81018874FB
:1058700004EB8400054901EB800000F10C0305F105
:105880002F023146284600F03BF970BD94A7012055
:105890002DE9F05F80460F46164608F12F094FF0BC
:1058A000FF3A4146386800F0B8FC38B9387800F063
:1058B000F000E02802D00FB1386818B96FF00D0081
:1058C000BDE8F09F01213846FFF72CFE0446002C6E
:1058D00008DA2EB14948808C401C81B24748818447
:1058E0002046EDE704EB8400454901EB8000807C15
:1058F00030B9012004EB8401414A02EB8101887434
:1059000000BF00BF04EB84003D4901EB8000807CB8
:10591000012800D03EB93946404600F0DBF8824607
:105920000EB95046CCE700BF00BF04EB84003449F9
:1059300001EB8000807C02280FDB32490C7004EB05
:1059400084002F4901EB800000F10C034A463146E8
:10595000404600F0D5F882464EE004EB840028492A
:1059600001EB8000807C012846D14FF0000B3546CA
:1059700008E000BF00BF287B012802D04FF0010BD8
:1059800002E02D68002DF4D100BFBBF1000F10D054
:1059900029890022032002F05FFD05466DB13146E2
:1059A000284602F07BFE40B1284602F020FF002589
:1059B00003E03546284603F01DF8A5B104EB84004A
:1059C0000F4951F8200030B104EB84010C4A52F821
:1059D000210002F00CFF04EB8400094941F820503B
:1059E0004FF0000A07E00548808C401C81B2034854
:1059F00081844FF0FF3A00BF504661E760A6012066
:105A000094A70120120100202DE9F84F074688468F
:105A100091469A46DDF828B00020009000BF00BFF4
:105A200000222A21032002F017FD05464DB928481F
:105A3000808C401C81B2264881844FF0FF30BDE845
:105A4000F88F00BF00BF6E6806F10E040D9801F0DC
:105A5000F4F8E08000BF00BFDAF80000A060BAF8F8
:105A60000400A0810B980168C4F812108088E082BD
:105A7000D9F800003060B9F80400B080D8F8000010
:105A8000C6F80600B8F804007081DBF80000C4F81E
:105A90000E000C980068A0614FF4807020800820F0
:105AA000608006202071042060714FF4C160B081D5
:105AB00029463846BA69904700900548008B401C3B
:105AC00003490883284602F092FE00250098B6E7B5
:105AD00060A601207FB504460D460121064A201D1F
:105AE00004F12F038DE825000391044A194620464E
:105AF000FFF78AFF04B070BD76DF000070DF0000A2
:105B00002DE9F04105460E4617469846746800BFD9
:105B100000BFD8F800002060B8F80400A080386802
:105B2000C4F80600B88860810820A0813146284664
:105B3000AA699047BDE8F08170B500243DE004EB10
:105B400084001F4901EB8000857C25B304EB8400B1
:105B500001EB8000C07C401C04EB8401184A02EB7E
:105B60008101C87404EB8400114601EB8000C07C05
:105B7000F0280DDA04EB840001EB8000807C012822
:105B80000AD104EB840001EB8000C07C022803DB17
:105B90002046FFF777FD0EE004EB8400084901EB97
:105BA0008000807C032806D1022004EB8401044A93
:105BB00002EB81018874601CC4B20A2CBFDB70BD8B
:105BC00094A701202DE9F04706460D461746984652
:105BD00000BF00BF5DB1286848B13146286800F0B9
:105BE0001CFB20B9287800F0F000E02803D16FF00A
:105BF0000D00BDE8F08741462846FFF793FC0446B8
:105C0000002C01DA2046F4E7022004EB84011A4A52
:105C100002EB8101887404EB8400114601EB8000E3
:105C2000866004EB840001EB80003968C160B988AC
:105C30000182002004EB840102EB8101C87404EBB3
:105C40008400114651F8200098B104EB840051F80B
:105C50002090002004EB840142F821003B4606F12D
:105C60002F0249463046FFF74BFF484602F0BFFD82
:105C700000BF0020BDE7000094A701202DE9F041FE
:105C800004460E464FF00E0860890E280BDC3348A0
:105C9000008D401C81B231480185C08B401C81B20F
:105CA0002E48C18354E06568AF89287800F0010070
:105CB000B0B12878012809D1687888B9A8785E2819
:105CC0000ED1607B40F01000607309E00622244989
:105CD0002846FAF7A4FB18B9607B40F0080060730F
:105CE000082F03D0B7F5C16F22D114E096F8350024
:105CF00000F0200000B92BE0C8F1000001B22046FE
:105D000002F0D9FD10B100BF00BF21E031462046AE
:105D100000F0AAFA18E096F8350000F0200000B96B
:105D200016E0224606F12F013046FFF755FB0BE047
:105D30000A48008D401C81B208480185C08B401C78
:105D400081B20648C18303E000BF0020BDE8F081B6
:105D5000204602F04CFD0020F8E7000060A601207C
:105D600070DF00002DE9F05F074688464FF0000B1A
:105D7000EFB1BC69002C14DA03F0C1F98346B869AD
:105D800000280ADAB8F1000F02D1B869401EB861E4
:105D9000584603F0EAF9BDE8F09FBC69584603F0A5
:105DA000E4F9204600F0B4F805460DB9F3E7F2E750
:105DB00003F0A5F98346B8F1050F17D2DFE808F024
:105DC00003080D1013006889401C00B2688110E0C0
:105DD0006889401E00B268810BE00120A88108E0BC
:105DE0000020A88105E00120E88102E000BF00BF9B
:105DF00000BF00BF686918B9584603F0B6F9CAE792
:105E000000BF324806685AE07069002848D18146D0
:105E1000B5F90A0000280FDDB16869B1E11704EB9C
:105E20005171C910B268515C04F0070301229A4015
:105E3000114009B14FF00109A88990B1B9F1000FE3
:105E40000FD1F16869B1E11704EB5171C910F26823
:105E5000515C04F0070301229A40114009B14FF050
:105E60000109E88990B1B9F1000F0FD1316969B129
:105E7000E11704EB5171C9103269515C04F007035A
:105E800001229A40114009B14FF00109B9F1000F08
:105E900005D00120706106F1180003F034FA00BF4C
:105EA0000B48D0F800A0584603F05FF903F027F93B
:105EB000834607480068824500D0A2E73668002E76
:105EC000A2D1584603F051F900BF64E774000020E6
:105ED000780000202DE9F04104460D460027666851
:105EE000002060602081206103F009F9074600204E
:105EF0002060384603F039F93EB11DB1304602F05A
:105F000076FC02E0304601F0C5FDBDE8F0810000FE
:105F10000146002901DB082901DB0020704701EB65
:105F20004100044B03EBC002106808B90020F5E7FC
:105F30001046F3E7B822002070B505460C4622460D
:105F40000321284600F0F2F870BD00002DE9FE4F55
:105F5000044689467248B0F84A00401C81B2704835
:105F6000A0F84A106568287800074FEA9068C8F1E1
:105F70000001204602F09FFC10B92089042800D2BD
:105F8000B4E0606890F800A0BAF1000F03D0BAF155
:105F9000080F7DD100E0A4E001266248007800F0FF
:105FA000F000E02800D100265E490868494600F06C
:105FB00034F900B1002666B95948B0F85C00401CBD
:105FC00081B25748A0F85C10204602F010FCBDE8F2
:105FD000FE8F2089082800D288E0204600F0F2F8E1
:105FE00058B1204602F003FC4D48B0F85000401C68
:105FF00081B24B48A0F85010E9E72421204602F076
:106000005AFC48B34146204602F055FC10B100BF8F
:1060100000BF77E021890022022002F01DFA064627
:1060200006B96FE000BF00BF2146304602F036FBE4
:1060300010B100BF00BF65E07568C8F1000001B293
:10604000304602F038FC10B100BF00BF5AE02046D5
:1060500002F0CDFB344608E06FF02301204602F049
:106060002AFC10B100BF00BF4CE067682D480068F3
:10607000E8602D4800682861002038707880FF2093
:106080002872002068812648B0F84800401C00E0D3
:1060900017E02349A1F848004146204602F00BFCD6
:1060A00008B100BF0CE001200021FF230A46CDE922
:1060B000010900911B49204600F0FEF9064600BF89
:1060C0000FE01748B0F85800401C81B21448A0F8FF
:1060D0005810B0F84E00401C81B21148A0F84E1084
:1060E00000BF00BF204602F082FB70E7204602F0AE
:1060F0007EFB0B48B0F85200401C81B20848A0F863
:10610000521064E7204602F072FB0548B0F85C00CC
:10611000401C81B20248A0F85C1000BF57E70000A5
:1061200060A601200C010020080100202DE9FE439B
:1061300006460F46904600222421012002F08CF9E9
:1061400005460DB9BDE8FE8300BF00BFD6F8049038
:106150006C68277084F801800020A080E08071685E
:106160006A6802F108001C22FAF714F90020608026
:106170006989204600F01CF860800C48B0F848009F
:10618000401C0A49A1F84800D9F80C0002900120EF
:106190000021FF2302AACDE90010284600F068F98B
:1061A000284602F024FB00BFCCE7000060A60120D7
:1061B00070B504460D462946204600F0FEFFC04358
:1061C00080B270BD2DE9F041064600240027354617
:1061D00017E06989686800F0F0FF0444A0B200EBA2
:1061E0001444688900EBD0714910A0EB410139B12A
:1061F000C7F10100C7B2E0B2C4F3072141EA0024AD
:106200002D68002DE5D127B1E0B2C4F3072141EAA2
:106210000024E04380B2BDE8F08118B50246009248
:10622000D04300B10AB9012018BD91F8350000F043
:10623000020008B90020F7E74868904201D1002029
:10624000F2E700988B681840D1E901342340984266
:1062500008D1886822EA00008C68E343984201D1A3
:106260000120E1E70020DFE72DE9F04706460F4671
:106270007948408E401C81B27748418675682878FD
:106280000421B1EB201F12D0304602F0B0FA724860
:10629000B0F84400401C81B26F48A0F84410C08E92
:1062A000401C81B26C48C1860020BDE8F087287888
:1062B00000F00F094FF6FF7000EA8909688800F0C6
:1062C0001FFD80467089484502DB308940450FDA62
:1062D000304602F08CFA6048408F401C81B25E4824
:1062E0004187C08E401C81B25B48C1860020DCE73C
:1062F0004146304602F042FB286958490860E86888
:10630000574908604FF0010A3C4600BF94F8350039
:1063100000F0010078B1201D68B1606858B14F48A5
:1063200000686168884205D04C4908682146FFF73B
:1063300074FF00B10DE0BAF1000F04D04FF0000A75
:106340004848046800E02468BC4200D12468002C5E
:10635000DCD100BF424908683946FFF75EFF28B923
:106360003F48007800F0F000E0280AD1304602F003
:106370003EFA3948C08E401C81B23748C1860020A1
:1063800093E724B9304602F032FA00208DE7E8881E
:106390004FF63F71084088B1304602F028FA2E4887
:1063A000B0F84200401C81B22B48A0F84210C08EC9
:1063B000401C81B22848C186002076E72A48076041
:1063C0002A4805603946304602F0FAFBC0BB687ABD
:1063D00001280DD0062806D011280ED139463046A6
:1063E00007F076F82BE03946304603F02FFD26E023
:1063F00039463046FFF7AAFD21E0184908683946BA
:10640000FFF70BFF50B91548007800F0F000E028C6
:1064100004D0756002213046FFF78EFD304602F051
:10642000E6F90D48B0F84000401C81B20A48A0F8D7
:106430004010C08E401C81B20748C18600BF00BF1B
:1064400000200949086009490860054908600349B6
:10645000086000BF29E7000060A601200C010020B1
:10646000080100209C000020000100200401002001
:106470002DE9FE4F06460F4615469846DDE90C9A73
:1064800000BF00BF284600F07DF8041E08D109486F
:10649000C08F401C81B20748C187201FBDE8FE8F16
:1064A00043462A4639463046CDE9009A029400F028
:1064B00003F8F3E760A601202DE9F84F05460E46E4
:1064C00017469A46DDF828B0DDF8308000BF00BFDF
:1064D000002F43D04FF014091421284602F0EBF9A5
:1064E00058B12648B0F84400401C81B22348A0F8B7
:1064F00044106FF00100BDE8F88F6C6800BF00BF6A
:1065000084F808A00B9860723868206148464FEA0A
:10651000E97109EB9171C1F3870141F040012170EC
:1065200084F801B0288900F088FB60800020E080BA
:106530001348008800F081FBA08011480088401CAF
:106540000F4908800EB1306818B9D8F80400E0602F
:1065500001E03068E0600020608103E06C68206941
:1065600000906F460548008E401C044908863A4654
:1065700029464046D8F814309847BCE760A6012069
:106580001001002010B50246144801680FE091F890
:10659000350000F0010048B110688B681840D1E95F
:1065A00001342340984201D1084610BD09680029F2
:1065B000EDD10B48006830B10948006890F835000B
:1065C00000F0010038B90748C08F401C83B205486D
:1065D000C3870020E9E702480068E6E79C00002046
:1065E000A000002060A601202DE9FF47064688464E
:1065F0006F46347800BF302C01DB392C03DD0020DE
:1066000004B0BDE8F08700254FF00A09302C0ED108
:10661000701C06460478782C01D0582C05D14FF018
:106620001009701C0646047801E04FF0080900BF0D
:10663000302C09DB392C07DCA4F1300005FB0905FF
:10664000701C06460478F3E7B9F1100F1BD1302C0B
:1066500001DB392C07DD612C01DB662C03DD412CCD
:1066600011DB462C0FDC612C03DB7A2C01DC612171
:1066700000E0412104F10A00401A40EA0515701CAF
:1066800006460478D4E700BF00BF2E2C09D103A82A
:10669000874201D30020B3E720C7701C0646047868
:1066A000A9E700BF00BF6CB1202C0BD00C2C09D087
:1066B0000A2C07D00D2C05D0092C03D00B2C01D0AF
:1066C00000209DE76846381A012101EBA00005284B
:1066D0002AD2DFE800F00305060F1B0000208FE739
:1066E00025E0B5F1807F01D3002089E7009845EAD5
:1066F00000651CE0B5F5803F01D3002080E70098DD
:106700000006019940EA0140054310E0FF2D01D940
:10671000002075E700980006019940EA01400299BF
:1067200040EA0120054302E000BF00BF00BF00BFF8
:10673000B8F1000F04D0284600F072FAC8F8000043
:1067400001205DE770B50025FBF78EFEF9F7AAFD85
:10675000054601211848FBF7ADF9044604F08050C6
:1067600050B11548FBF753FA1348FBF73AFA1248B1
:10677000FBF721FA24F080541CB121460E48FBF7A8
:106780005BF904F0005058B10B48FBF735FA0646A8
:106790000A48006820B131460748084A1268904705
:1067A0001CB12146064806F085FB2846F9F77EFD18
:1067B000FBF774FE70BD000000C00E40A001002079
:1067C00098DB0120704700002DE9FC4704460D4688
:1067D00016461F46DDE90A892248FDF7A5FD214836
:1067E000FDF7F4FD2048FDF7B9FD30B11E48FDF777
:1067F0009BFD1D48FDF7EAFD01E000BFFEE700BF7D
:106800001848FDF7C7FD0028FAD040F20E4117489E
:10681000FBF76AF9002004210B46154ACDE9001068
:1068200021461248FBF7B4F800234FF008724FF4EA
:1068300040610E48FBF78AF82A4600210B48FBF717
:1068400048F80C48C0F800900B4806600B480760F9
:106850000B48C0F8008000210A4806F053F9BDE853
:10686000FC870000009C00F0003000F000C00E40EB
:1068700002000004A4010020A8010020AC010020B7
:10688000B0010020A168000010B50446FFF79AFF90
:10689000002202490A2002F081FD10BD8968000033
:1068A00010B586B004461848006878B917480068E3
:1068B00000F0B6F905901648006800F0B1F90490B0
:1068C0001448006800F0ACF9039003E00020059044
:1068D0000490039010481149002203ABCDE9002138
:1068E000029004AA05A90E4801F0C0FC0C4801F072
:1068F0000BFD0B4801F08DFD00220A490A2002F031
:106900004DFD06B010BD0000A4010020A80100202C
:10691000AC010020B00100206DCB000075CE00005E
:1069200098DB0120896800002DE9F04F87B082468E
:10693000884617464FF0000B5046FFF7E9FA044629
:1069400024B94FF0FF3007B0BDE8F08F206890F811
:10695000200000F0020050B1B4F90A00002806DC63
:1069600000BF0B20206100BF4FF0FF30EBE706A90E
:10697000206801F09FF80546BDB120680078102816
:1069800004D000BF5F20206100BFDCE700BF684289
:10699000102804D24248694250F8210000E0052046
:1069A000206100BF4FF0FF30CDE700BF00BF00BF48
:1069B000069890F8200040F00800069981F8200021
:1069C00000BF002304AA05A9069801F02BFA05468A
:1069D0008DB1069801F07CF900BF6842102804D2FE
:1069E0002F48694250F8210000E00520206100BFD7
:1069F0004FF0FF30A7E7B8F1000F1ED000BF00BF77
:106A00000020009001900290039010208DF800006B
:106A100002208DF80100BDF8100000F00EF9ADF86D
:106A20000200059801903868102801D910203860BC
:106A3000694640463A68F9F7ADFC01210698FDF732
:106A4000EBFF0646701C48B9069801F041F900BFFB
:106A50001720206100BF4FF0FF3074E700BF00BF78
:106A600000BF00BF06EB46000E4901EBC00902F073
:106A700046FB8346B9F80A1006988069C0F1FF30DA
:106A8000084400B2A9F80A0006988661584602F048
:106A90006CFB00BF0020206100BF304653E70000C0
:106AA000B0DD0000B82200202DE9F84F82460C46E8
:106AB00090465046FFF72CFA05461DB94FF0FF30BF
:106AC000BDE8F88F00BFB8F1100F05D1607802283B
:106AD00002D104F0030038B100BF1748806B286171
:106AE00000BF4FF0FF30EBE700BF27463C46786819
:106AF0000090B7F80290484600F002F983465A46E3
:106B00006946286801F08CF8064676B100BF7042ED
:106B1000102804D20848714250F8210000E00520F6
:106B2000286100BF4FF0FF30CAE700BF0020286196
:106B300000BF00BFC4E70000B0DD000070B505462F
:106B400000262846FFF7E4F904460CB9701E70BD14
:106B5000206840B120680078102801D1012000E0B1
:106B60000020064601E000BF00BF206801F0B0F839
:106B700031462046FFF7AEF90020E8E72DE9F84F4F
:106B800081460E4690464846FFF7C2F904461CB9B6
:106B90004FF0FF30BDE8F88F00BFB8F1100F05D1FE
:106BA0007078022802D106F0030038B100BF1B48FC
:106BB000806B206100BF4FF0FF30EBE700BF37462E
:106BC0003E46787820B9206801F096F805460EE038
:106BD00078680090B7F802A0504600F091F883461C
:106BE0005A466946206801F047F8054600BF75B16E
:106BF00000BF6842102804D20848694250F82100BA
:106C000000E00520206100BF4FF0FF30C2E700BF69
:106C10000020206100BF00BFBCE70000B0DD000025
:106C20000146080601F47F4240EA022001F47F0297
:106C300040EA122040EA1160704701460806000C45
:106C400040EA1120704710B502F008FA02F094FAF9
:106C500000F086FB00F06AFD01F040FB00F0ACFAAA
:106C600006F034FC03F0F0F802F004FC10BD000064
:106C70002DE9F04107460E463846FFF749F904462C
:106C80001CB94FF0FF30BDE8F081002E01DD304629
:106C900000E00020FF2805DA002E01DD304602E08A
:106CA000002000E0FF200646F1B2206801F0F4F871
:106CB0000546BDB120680078102804D000BF5F20D1
:106CC000206100BFDFE700BF6842102804D20848F7
:106CD000694250F8210000E00520206100BF4FF01C
:106CE000FF30D0E700BF0020206100BF00BFCAE72F
:106CF000B0DD000000B503461846FFF791FF00BD68
:106D000000B502461046FFF798FF00BD2DE9FC4193
:106D100004460D4616461F46002000903B4632466C
:106D200029460190204600F003F8BDE8FC810000F0
:106D30002DE9FF4F8BB016469846DDF86490002091
:106D40000A90002506900B98FFF7E2F804461CB95C
:106D5000681E0FB0BDE8F08F00BF606810B16068BA
:106D60000A9057E008F0080028B9206890F8200041
:106D700000F00200B0B1B4F90A00002812DC002DC6
:106D800009DD2946206801F0FFF900BF00202061DD
:106D900000BF2846DDE700BF0B20206100BF4FF099
:106DA000FF30D6E720680078102805D10AA92068AE
:106DB00001F0D8F9834604E00AA9206801F0CEF872
:106DC0008346BBF1000F21D0002D09DD2946206844
:106DD00001F0DAF900BF0020206100BF2846B8E7C3
:106DE00000BFCBF10000102805D25C48CBF10001B8
:106DF00050F8210000E00520206100BF0BF10C00DD
:106E000008B90020A5E74FF0FF30A2E700BF00BFA0
:106E10000A98606020680078102802D10A980990CA
:106E200002E00A98006809900998B0F808A0208943
:106E3000AAEB00001FFA80FA564501D9574600E038
:106E4000B7B223890C9841193A46099801F086FC9B
:106E50003D4420680078102812D100BF00BFF61B07
:106E60005EB10998407B00F0010030B9B4F90A0026
:106E7000002802DD08F0010020B10120069001E0A9
:106E8000012006900698D0B31898B8B3B9F1000F56
:106E900034D020680078102808D105A80890002375
:106EA00007AA2068089900F0BDFF05E00A9808309D
:106EB00008900A9880890790002001900290039022
:106EC000049010208DF8040002208DF80500BDF814
:106ED0001C00FFF7B2FEADF80600089800680290AB
:106EE000D9F80000102802D91020C9F8000001A923
:106EF000D9F800201898F9F74DFA00BF00BF08F044
:106F00000100D8B920680078102809D1AAEB070041
:106F1000002805DD0A9860602089384420810DE052
:106F200000206060208120680078102803D10A9832
:106F300001F05DFC02E00A9800F0ACFD0698002824
:106F40003FF40BAF002D03DD2946206801F01CF94A
:106F500000BF0020206100BF2846FAE6B0DD000037
:106F60002DE9FE4F8046894692461E464046FEF772
:106F7000CFFF05461DB94FF0FF30BDE8FE8F2868F2
:106F80000078102809D00020009033465246494628
:106F90000190404600F030F8EFE706F0100008B12D
:106FA000022000E0002040F0010006F0080109B1D5
:106FB000042100E0002140EA01070020029002A81D
:106FC00000903B4652464946286801F0F7F80446CF
:106FD00000BF6042102804D20648614250F82100E8
:106FE00000E00520286100BF0CB90298C5E74FF00A
:106FF000FF30C2E7B0DD00002DE9FF4F81B08B46C6
:107000000E9F0198FEF784FF044624B94FF0FF302D
:1070100005B0BDE8F08F20680078102806D15946E9
:10702000DDE903230198FFF79BFFF1E700BF00BFF5
:10703000039880B2009000BF0FB90F9880B10F98ED
:10704000102805D17878022802D107F0030038B162
:1070500000BF3248806B206100BF4FF0FF30D7E7A0
:1070600000BFB84602220020009901F0F5F98146E0
:10707000B9F1000F3ED0C9F804B0B8F1000F07D045
:1070800008F1040AB8F80200FFF73AFE06460EE0DF
:107090002068406800F1040A2068007800F0F000E1
:1070A000202803D120684068868A00E0002600215D
:1070B0001B4802F028F820680078402809D1216890
:1070C00052464868494601F00BFE216808720546A1
:1070D00009E02168334652464868494606F076FB87
:1070E0002168087205460E4802F00DF9484601F085
:1070F0007EFB01E04FF0FF3500BF6842102804D24C
:107100000648694250F8210000E00520206100BFD8
:107110000DB900987CE74FF0FF3079E7B0DD000053
:10712000880000202DE9F04180460F461646012FC9
:1071300016D0022F08D0032F22D1F1B21D4A4020D1
:1071400000F0D0FE04461FE0882E01D1212100E08E
:1071500020210846174A002100F0C4FE044613E02F
:10716000144A0021102000F0BDFE04463CB100BFCF
:1071700094F8200040F0080084F8200000BF03E0ED
:107180004FF0FF30BDE8F08100BF14B94FF0FF3081
:10719000F8E700212046FDF73FFC0546681C28B9AA
:1071A000204600F095FD4FF0FF30EBE7A561284643
:1071B000E8E70000655D00007047F8B505460A463F
:1071C0002B4600200090002103F0010636B1002A72
:1071D00004DD13F8010B8DF80100521E1C4603E07C
:1071E00034F8027B3944921E012AF9DC002A02DDC0
:1071F00020788DF80000BDF80000014488B200EB53
:10720000114188B200EB114126B1C8B2C1F3072782
:1072100047EA002188B2F8BD88B006A90FA0FAF7A6
:1072200089F9F9F70FF8FBF7E5F8032000214FF48F
:1072300080720E4BCDE90132CDE9031004200346E4
:107240000B4A00900B48FBF7CDFD07AA0AA10420CA
:10725000FBF7E4FEFBF776FD00BFFEE7544D344339
:10726000313239344E43504454000000D4DB012005
:10727000D0DF0120B9050000537461727400000072
:1072800070B505460C460C48844208D1F9F782FDDA
:107290000646012231462846FAF72CFE0AE0074846
:1072A000844207D1F9F776FD06460022314628468A
:1072B000FAF720FE70BD0000801A0600A0860100CB
:1072C00070B5054605B970BD00BF00BF00BF00BF67
:1072D0001E480068854203D31D48006885420FD3CD
:1072E000002601F00CFF06461A48B0F89800401C32
:1072F00081B21848A0F89810304601F036FFE2E756
:107300000021154801F0FFFEA5F1080400BF00BFF1
:107310000020207111480068844201D20F480460A7
:1073200020880A490988611A411A0A48B0F892006F
:10733000401A81B20748A0F89210204601F0B6FB2F
:10734000054801F0E0FF00BFBDE700008C00002011
:107350009000002060A601209800002094000020EA
:1073600010B500BF00BF174820F0030016490860A1
:10737000084604684FF4205020800020608020716F
:107380000846006800F5205010490860012009688F
:1073900008714FF420500D49096808800B490968AD
:1073A0004880094800680A4908604FF4205009499C
:1073B000A1F890000121084801F088FF08B100BF42
:1073C00000BF10BD7B2300208C0000209000002017
:1073D0009400002060A60120980000202DE9F041D3
:1073E000054615B90020BDE8F081E81C20F0030037
:1073F00085B20C2D00DA0C25B5F5205F01DD0020EB
:10740000F1E70021524801F07EFE524800885249BF
:107410000988401A86B289E04F48006884192079AB
:1074200000287CD1218806F10800081AA8427AD3E6
:10743000218806F10800091A05F11400814232D3AF
:1074400006F1080028441FFA80F84348006800EB62
:10745000080700203871208838807E80A4F80080DA
:10746000012020713888B0F5205F05D038883A496E
:1074700009680844A0F8028000BF3848B0F89210AC
:1074800005F10800084481B23448A0F89210B0F821
:107490009410B0F89200814204DA3048B0F89210AB
:1074A000A0F894101BE00120207100BF20882A4919
:1074B0000988611A411A2948B0F89200084481B23B
:1074C0002648A0F89210B0F89410B0F892008142CB
:1074D00004DA2248B0F89210A0F8941000BF1D48BA
:1074E0000068844211D11B49086803E001881A4AE8
:1074F00012688818017919B1194909688842F5D1CB
:107500001449086000BF00BF00BF114801F0FBFE36
:1075100000BF00BF00BF00BF00BF00BF00E002E02F
:1075200004F108005FE70C480068865BC5F5205051
:10753000B0423FF771AF0948B0F89600401C81B2E5
:107540000648A0F89610024801F0DDFE00204AE748
:1075500098000020940000208C00002060A60120EC
:10756000900000202DE9F05F82460D46E81C20F0D7
:10757000030085B20C2D00DA0C25B5F5205F02DD85
:107580000020BDE8F09F00BF00BF4B480068824567
:1075900003D34A480068824511D34FF0000B01F035
:1075A000AEFD83464648B0F89800401C81B244487E
:1075B000A0F89810584601F0D8FD5046E1E7AAF12E
:1075C00008073D480088381A1FFA80F93888A0EB70
:1075D000090008381FFA80F800BF00BF454501DDEB
:1075E0000020CEE7454501D15046CAE70021354885
:1075F00001F089FD3888304909684418207950BB6A
:10760000208809F1080129448EB22F490968A14256
:1076100004D12949096831442B4A11602649096877
:107620008C19002121712080A4F802903E802188CD
:10763000B1F5205F04D021881F4A126811444E80A2
:107640001F49B1F89210A8EB0502891A8AB21C49A9
:10765000A1F892202AE005F11400404526D809F14E
:107660000800284486B21448006884191648006847
:10767000844201D2144804600020207138882080A0
:10768000A4F802903E802088B0F5205F04D02088C6
:1076900009490968084446800948B0F89200A8EBF7
:1076A0000501401A81B20648A0F89210054801F081
:1076B0002AFE504665E700008C0000209000002064
:1076C00060A6012098000020940000202DE9F041E0
:1076D00004460D4600270DB9BDE8F08100BF00BF8C
:1076E000A5F11C0601F00BFD074600F0DBF804EBEA
:1076F00084010C4800EB41004088401E81B204EB3D
:107700008402084800EB42004180074850F82400FA
:107710003060054840F82460384601F026FD00BF7F
:10772000DAE70000FAA601208C4B002070B5002497
:107730001CE0002104EB8402224800EB420041805F
:1077400004EB84021F4800EB4200818004EB8402BA
:107750001C4800EB4200C1801B4830F8141004EBB9
:107760008402184820F81210601C84B20C2CE0DB54
:10777000164820F0030500241DE00020144941F8BC
:107780002400002610E0124850F824002860104819
:1077900040F824500F4830F8141005F11C0008443C
:1077A00000F11005701C86B2074830F81400B04292
:1077B000E9DC601C84B20C2CDFDB00F033F900F054
:1077C00071F870BDFAA6012008DE0000BF4B002052
:1077D0008C4B0020F0DD00002DE9F04104460E4600
:1077E00017464FF0000800BF0C2C02DB0020BDE85C
:1077F000F08100BF01F083FC804600F053F8274879
:1078000050F82450ADB32549286841F824000020E1
:1078100028606E60AF6000BF04EB8401204800EB7D
:1078200041004088401C81B204EB84021C4800EBFC
:107830004200418004EB8401194800EB410081883B
:1078400004EB8402164800EB4200408881420BDAC8
:1078500004EB8401124800EB4100418804EB8402F0
:107860000F4800EB4200818000BF00BF00BF1C3505
:107870000EE0FFE704EB8401094800EB4100C088FB
:10788000401C81B204EB8402054800EB4200C18039
:10789000404601F06AFC2846A9E700008C4B002016
:1078A000FAA6012070B51F4820F00305002417E058
:1078B00000BF00260DE02146284600F039F81A489E
:1078C00030F8141005F11C00084400F11005701C7C
:1078D00086B2164830F81400B042ECDC601C84B26A
:1078E0000C2CE5DB0F4820F00305002417E000BF57
:1078F00000260DE02146284600F05AF80A4830F8E4
:10790000141005F11C00084400F11005701C86B22B
:10791000064830F81400B042ECDC601C84B20C2C39
:10792000E5DB70BDBF4B0020F0DD000008DE00008D
:10793000F0B5A1B006460C461A4830F8141006F10E
:107940001C000F18002529E0785DCD2824D0802266
:10795000154901A8F8F71EFD14A0006800900A2C34
:107960000ADB0A2094FBF0F03030C0B28DF8000042
:10797000694601A8F8F732FD0A2094FBF0F100FBFC
:1079800011403030C0B28DF80000694601A8F8F708
:1079900025FD00BF00BF00BF681C85B2102DD3DBE2
:1079A00021B0F0BDF0DD000020DE0000300000005E
:1079B000F0B5A1B006460C4606F10C07002529E0FB
:1079C000785DCD2824D08022144901A8F8F7E2FC84
:1079D00013A0006800900A2C0ADB0A2094FBF0F048
:1079E0003030C0B28DF80000694601A8F8F7F6FC07
:1079F0000A2094FBF0F100FB11403030C0B28DF84A
:107A00000000694601A8F8F7E9FC00BF00BF00BF0D
:107A1000681C85B2102DD3DB21B0F0BDA0DE0000C4
:107A2000300000002DE9F041174820F00305002444
:107A300025E000BF00261BE005F10C07CD22102138
:107A40003846F8F7B9FC114830F8141005F11C005D
:107A50000F18CD2210213846F8F7AEFC0B4830F84D
:107A6000141005F11C00084400F11005701C86B2CA
:107A7000074830F81400B042DEDC601C84B20C2CE5
:107A8000D7DBBDE8F0810000BF4B0020F0DD000037
:107A900008DE000010B504465CB1206828B12068FB
:107AA00000F0A5FE00206060206021460520FFF761
:107AB0000DFE10BDF8B504460D4600BF15B96FF0B8
:107AC0000D00F8BD00BF0020286000BF14B96FF0A2
:107AD0000D00F6E700BF00BF04F1140001F0BEFB8B
:107AE00010B96FF00D00ECE700BF94F9086016F1D3
:107AF000090F01DA3046E4E7694604F11400E2694F
:107B000001F0AEFA401C90B900BF002701F0F7FA6F
:107B1000074694F9080010F1090F01DBFD202072DF
:107B2000384601F022FB00BF6FF00200C9E7E06AAF
:107B300020B1002201212046E36A9847009890B9BD
:107B400000BF002701F0DBFA074694F9080010F1A6
:107B5000090F01DBF6202072384601F006FB00BF5A
:107B60006FF00900ADE7009828600020A9E7000049
:107B70002DE9F04105460E4640F241221BA10620A8
:107B8000FFF72AFE044614B90020BDE8F08100206A
:107B90002072257060600427002104F10C0001F0C0
:107BA00095FB00B11BE0394604F1100001F008FB21
:107BB00020B104F10C0001F07FFB10E004F114008F
:107BC00001F034FB00206070401EA061E6620020DE
:107BD000A0626062E06184F820002046D5E721467B
:107BE0000620FFF773FD0020CFE700002E2E5C2E4D
:107BF0002E5C5372635C5573725C44726976657275
:107C00005C55704472697665725C6C7769705C6112
:107C100070695C6170695F6D73672E6300000000BE
:107C20002DE9F04186B004460E46174600BF24B940
:107C30006FF00D0006B0BDE8F08100BF0D48009068
:107C400001940396ADF81070684604F0FFFE0546F7
:107C500000BF4FF0000801F052FA804694F9080086
:107C600010F1090F00DB2572404601F07EFA00BFDB
:107C70002846DFE7654B00002DE9F04186B0044659
:107C80000E46174600BF24B96FF00D0006B0BDE8E0
:107C9000F08100BF0D48009001940396ADF810707C
:107CA000684604F0B5FE054600BF4FF0000801F03D
:107CB00026FA804694F9080010F1090F00DB2572BE
:107CC000404601F052FA00BF2846DFE7FD4C0000B5
:107CD00010B586B0044614B9002006B010BD0548A2
:107CE00000900194684604F093FE204600F07DF871
:107CF0000020F2E7634E000070B586B0044600BF76
:107D00001CB96FF00D0006B070BD00BF0B480090AD
:107D10000194684604F09AFE054600BF002601F073
:107D2000EEF9064694F9080010F1090F00DB257200
:107D3000304601F01AFA00BF2846E4E7254F00005C
:107D4000F8B5044604F1100001F088FA18B312E007
:107D5000207810280CD1009868B1009E606818B196
:107D60003189606803F0E0FF304600F040FD02E03A
:107D70000098FFF78FFE694604F1100001F0B6F994
:107D8000401C0028E4D104F1100001F003FA04F1D2
:107D9000100001F04BFA04F1140001F05FFA18B37F
:107DA00012E0009D606808B100BF00BF2846FFF7E1
:107DB000C7FF686820B1686801F034FC0020686083
:107DC000284600F012F800BF694604F1140001F0E3
:107DD0008DF9401C0028E4D104F1140001F0DAF917
:107DE00004F1140001F022FAF8BD10B5044600BFFA
:107DF00000BF00BF04F1100001F030FA00BF00BF67
:107E000004F1140001F02AFA00BF04F10C0001F0A3
:107E100053FA04F10C0001F073FA21460620FFF733
:107E200055FC10BD2DE9F04387B004460D461646BB
:107E3000984600BF24B96FF00D0007B0BDE8F0838D
:107E400000BF00BF15B96FF00D00F6E700BF00BF1F
:107E500016B96FF00D00F0E700BF0E4801900294D4
:107E6000049505968DF8188001A804F0EFFD0746EB
:107E700000BF4FF0000901F042F9814694F9080073
:107E800010F1090F00DB2772484601F06EF900BFC0
:107E90003846D2E7494F0000F0B587B004460F4698
:107EA00000BF1CB96FF00D0007B0F0BD00BF0C485B
:107EB0000190029401A804F0C9FD054600BF002608
:107EC00001F01DF9064694F9080010F1090F00DBD6
:107ED0002572304601F049F900BF2846E4E700006A
:107EE000ED4F0000F0B587B007460D461646314607
:107EF0003846FFF73DFE04465CB3174801908DF805
:107F00001050029401A804F0A1FD10B300BF00BFFF
:107F100000BF04F10C0001F0FCF900BF00BF04F148
:107F2000100001F09BF900BF00BF04F1140001F044
:107F300095F900BF04F10C0001F0BEF904F1100046
:107F400001F028F921460620FFF7C0FB002007B00A
:107F5000F0BD2046FBE70000AD5000002DE9F843DE
:107F600005460E46002400BF1EB96FF00D00BDE8A7
:107F7000F88300BF0020306000BF15B96FF00D001E
:107F8000F5E700BF00BF05F1100001F067F910B977
:107F90006FF00C00EBE700BF2878102834D10020E8
:107FA00000904FF4ED721BA10520FFF715FC04466D
:107FB0009CB900BF4FF0000801F0A1F8804695F988
:107FC000080010F1090F01DBFF202872404601F084
:107FD000CCF800BF4FF0FF30C9E76946284600F0F3
:107FE00033F807462FB121460520FFF76FFB3846CF
:107FF000BDE700BF00BF00982060009860600020CF
:10800000A081A0603460B2E73146284600F01CF839
:10801000ADE700002E2E5C2E2E5C5372635C557310
:10802000725C4472697665725C55704472697665FB
:10803000725C6C7769705C6170695C6170695F6CBF
:1080400069622E63000000002DE9F04188B004460B
:108050000D460020079000BF25B96FF00D0008B055
:10806000BDE8F08100BF0020286000BF14B96FF0A8
:108070000D00F4E700BF00BF04F1100001F0EEF8BE
:1080800010B96FF00C00EAE700BF94F9087017F11F
:10809000090F01DA3846E2E707A904F11000E269A6
:1080A00000F0DEFF401C98B900BF4FF0000801F05F
:1080B00026F8804694F9080010F1090F01DBFD2035
:1080C0002072404601F051F800BF6FF00200C6E791
:1080D0002078102834D194F8200000F0080008B16E
:1080E000079868B91E4801900294079818B107983C
:1080F0000189049101E00121049101A804F0A6FC8A
:108100000798D0B9E06A20B1002201212046E36A35
:10811000984700BF4FF0000800F0F1FF804694F947
:10812000080010F1090F01DBF4202072404601F035
:108130001CF800BF6FF00B0091E70798068904E078
:1081400000BF00BF079800680689E06A20B1324688
:1081500001212046E36A98470798286000207EE7BF
:10816000C350000070B504460D4600BF14B120781E
:10817000102802D06FF00D0070BD00BF29462046C8
:10818000FFF762FFF8E7000030B587B004460D4600
:108190007CB1207810280CD194F8200000F0080061
:1081A00038B1054801900294049501A804F04EFCF2
:1081B00000BF07B030BD0000C35000002DE9F04FF4
:1081C00087B00446894615469846109E00BF24B9DC
:1081D0006FF00D0007B0BDE8F08F00BF00BF207842
:1081E000102802D06FF00500F4E700BF0DB90020A1
:1081F000F0E794F8200000F0020010B908F0040045
:1082000008B1012000E000208246BAF1000F03D03F
:1082100016B96FF00500DDE7134801900294CDF820
:1082200010908DF81880059501A804F00FFC074602
:108230003FB936B1BAF1000F02D00598306000E0C6
:10824000356000BF4FF0000B00F059FF834694F9F2
:10825000080010F1090F00DB2772584600F085FF77
:1082600000BF3846B6E70000015100002DE9F04795
:1082700004460D4616461F46DDE909A9DDF82080B3
:1082800000BF00BF00206060A060E06084F835009F
:10829000E0612062C4F828800E48007884F8380035
:1082A0000C480078401C0B490870C4F810903B46FD
:1082B00032462946204600F012F82046D04710B139
:1082C0000020BDE8F0870448006820600248046090
:1082D0002046F6E7A40000209C00002070472DE90E
:1082E000F04106460F4614461D463946304600F01A
:1082F00017F82146304600F086F82946304600F04F
:1083000009F8BDE8F08100000149086070470000ED
:10831000A000002009B9002200E00A68C26070478E
:108320002DE9F04107460C4654B32068796888422D
:1083300001D1012000E0002010BB154806680BE0C9
:1083400030687968884206D1D6F80C80304601F052
:1083500069F9464600E0F668002EF1D10D4805683F
:108360000CE055B1286840B128687968884204D18A
:108370000CB9002000E020682860ED68002DF0D1E5
:108380000CB9002000E020687860BDE8F0810000B2
:10839000BC000020B800002010B5044694F8350059
:1083A00000F0100060B194F8350020F0100084F85F
:1083B000350000BF206A10B12046216A884700BFFF
:1083C00010BD10B5044694F8350000F01000C8B98F
:1083D00014F8350F40F01000207014F8350900F043
:1083E000010040B194F8350000F0200018B1211DC3
:1083F0002046FDF76FFB00BF206A10B12046216ABE
:10840000884700BF10BD09B9002200E00A688260F9
:10841000704710B5044694F8350000F00100D0B95B
:1084200094F8350040F0010084F8350000BFE069A1
:1084300010B12046E169884700BF94F8350000F08C
:10844000100040B194F8350000F0200018B1211D53
:108450002046FDF73FFB10BD2DE9F05F83460F4638
:108460009046BBF1000F09D0BBF1010F08D0BBF162
:10847000020F07D0BBF1030F08D105E038260AE050
:10848000242608E0102606E0002604E000BF00BF16
:108490000020BDE8F09F00BFB8F1000F78D0B8F120
:1084A000010F72D0B8F1020F70D0B8F1030F6ED186
:1084B000EF2256A10B20FFF78FF904461CB900F0FC
:1084C00039FA0020E5E784F80C800020206006F1EE
:1084D00010002044C01C20F00300606000BF00BFFB
:1084E0002781F01C20F0030040F2EC51081AB8423A
:1084F00001DD384605E0F01C20F0030040F2EC51AD
:10850000081A608100BF00BF00BF00BF0120E081EA
:10851000A2466089A7EB000932E04FF488723BA1C4
:108520000B20FFF759F9054635B900F003FA20464C
:1085300000F05DF90020ACE785F80C80002068733E
:108540002860CAF8005000BF00BFA5F808901FFAC5
:1085500089F040F2EC51884202DA1FFA89F001E01A
:1085600040F2EC50688105F11000686000BF00BF68
:1085700000BF00BF0120E8816889A9EB0009AA4675
:10858000B9F1000FC9DC39E002E020E020E031E081
:1085900006F1130121F00302F91C21F0030111443B
:1085A00088B2FEF71BFF04460CB9002071E704F106
:1085B00010003044C01C20F00300606027816781F8
:1085C0000020206084F80C8000BF00BF16E000BFD0
:1085D0004FF4A3720DA10A20FFF7FEF804460CB970
:1085E000002056E70020606027816781206084F8C2
:1085F0000C8003E000BF00BF00204AE700BF01205D
:10860000E08100206073204643E700002E2E5C2EA0
:108610002E5C5372635C5573725C4472697665724A
:108620005C55704472697665725C6C7769705C63E6
:108630006F72655C706275662E63000010B502464D
:1086400000BF02B101B910BD00BF104604E00389AC
:108650000C892344038100680368002BF7D100BF15
:1086600000BF00BF00BF03890C8923440381016060
:1086700000BFE8E770B505460C4621462846FFF7DF
:10868000DDFF204600F0B6F970BD0146002002E093
:10869000421CD0B209680029FAD170472DE9F04197
:1086A00005460C460026002700BF25B11CB12889CD
:1086B0002189884203DA6FF00D00BDE8F08100BF28
:1086C00000BF6889801B6189C91B884204DB6089FF
:1086D000C01B1FFA80F803E06889801B1FFA80F82E
:1086E0006268D1196A6890194246F7F753FE06EBA3
:1086F000080086B207EB080087B200BF00BF00BFCA
:1087000000BF6089B84201DC002724686889B04254
:1087100008D100262D6800BF1DB914B16FF00D00FF
:10872000CBE700BF54B160892189884206D100BFE0
:10873000206810B16FF00500BFE700BF55B1688930
:108740002989884206D100BF286810B16FF0050062
:10875000B3E700BF002CB4D10020AEE72DE9F05FF5
:108760008046894616461D464FF0000B00BFB8F103
:10877000000F02D10020BDE8F09F00BF00BFB9F19B
:10878000000F01D10020F6E700BF4FF0000AB8F15A
:10879000000F02D0B9F1000F01D10020EBE74446F1
:1087A00020E035B16089A84203DC6089281A85B2CF
:1087B00017E06089401B87B2B74200DD3746626828
:1087C000511909EB0A003A46F7F7E4FD0BEB0700F5
:1087D0001FFA80FB0AEB07001FFA80FAF01B86B233
:1087E000002524680EB1002CDBD15846C3E72DE9E3
:1087F000F047044624B900BF00BF0020BDE8F08761
:1088000000BF00BF00262DE04FF0000900F077FC0C
:10881000814600BF00BFE089401E1FFA80F8A4F81F
:108820000E80484600F0A1FCB8F1000F18D127686F
:10883000257B032D04D121460B20FEF747FF0BE0DB
:10884000012D01D0022D04D121460A20FEF73EFF62
:1088500002E02046FEF734FD701CC6B23C4600E044
:10886000002400BF002CCFD13046C7E770B50025EB
:1088700000F045FC054600200A490870284600F033
:1088800074FC0948046808E0606F28B1606F03F069
:1088900074FB0020606770BDE468002CF4D100BF59
:1088A000F9E70000A5000020BC00002010B5044638
:1088B000FFF7DCFF10BD70B5024600BF00BF01B17D
:1088C0000AB9002070BD002908DA484284B200BF0E
:1088D0005089A04201DA0120F4E700E08CB2137B5A
:1088E00055680BB1032B0AD15068401A506002F151
:1088F00010005668864215D255600120E2E7022B2F
:1089000001D0012B0AD1002906DA5089A04203DBED
:108910005068401A506005E00120D3E700BF00BF57
:108920000120CFE750890844508110890844108104
:108930000020C7E770B5002500F0E1FB05460D48B3
:10894000047801200B490870284600F00EFC84B919
:1089500000BF00221146084804F08AF840B100F038
:10896000CEFB0546002003490870284600F0FDFBB9
:1089700000BF70BDA5000020AD8800002DE9F041CA
:1089800006460F4600BF00BF00BF00BF3089B84297
:1089900001DCBDE8F0813089A7EB00083D46344694
:1089A0000AE06089281A85B200BF00BF20894044D0
:1089B0002081246800BF00BF6089A842F1DB207BD2
:1089C00060B96089A84209D0A088001B284481B200
:1089D0002046FEF7C7FD044600BF00BF65816089E1
:1089E0002081206810B12068FFF701FF002020607F
:1089F00000BFCEE770B50446002544B100F07FFB10
:108A00000546E089401CE081284600F0AEFB70BDC1
:108A100010B5044600BF00BF2068007800F0F000E9
:108A200010282CD0202812D0402836D1207A00F0EF
:108A300001F9216848602068406810B9FF20207162
:108A40002EE022681749506800F026F928E004F06B
:108A500043FE216848602068406810B9FF202071FB
:108A60001EE020680078222803D10120216849688F
:108A7000087422680C49506804F084FE10E001F08C
:108A80000DFE216848602068406810B9FF20207101
:108A900006E0206800F0B8FA02E0FA20207100BF7A
:108AA00000BF10BD818D0000E58E000030B500BF15
:108AB00000BF00BF00BF00BF00BF00BF00BF0388F2
:108AC000194C24681919884215D00B799BB9174B9A
:108AD0001B6899420FD0164B1B688B4201D1144B77
:108AE00018600B880380104B1B88C31A0C880E4D2E
:108AF0002D682C44638043880B4C24681A198242E9
:108B000011D013797BB90A4B1B68834201D1084B02
:108B10001A6003881380044B1B88D31A0488024D03
:108B20002D682C44638030BD8C0000209000002014
:108B30009400002070B505460E462C4600BF00BFCD
:108B40006078012803D12046FCF726FB05E0607819
:108B5000042802D12046FCF73BF894F8200000F0EE
:108B60001000D0B16068C0B16068B0F8660040F62F
:108B70006931884211DD6068B0F8680008280CDAB5
:108B800094F8200020F0100084F82000E06A20B162
:108B9000002202212046E36A9847002070BD024669
:108BA00009B9002000E00868106000207047024604
:108BB00009B9002000E008685060002070470000FC
:108BC0002DE9F04705468A460027D5F8048098F835
:108BD00009900026144804681FE0207C48451AD1FB
:108BE00034B1206820B1114920680968884212D147
:108BF000606980B10E4B2A462146D4E905C0E047A2
:108C000048B10025012736B1E068F06006480068E9
:108C1000E060054804602646E4680FB9002CDCD10A
:108C20003846BDE8F0870000A80000200C010020B5
:108C30000801002070B5054640F2511209A100203C
:108C4000FEF7CAFD04465CB11C212046F7F7BBFBCA
:108C50002574FF20A0720F480068E0600D48046092
:108C6000204670BD2E2E5C2E2E5C5372635C5573B5
:108C7000725C4472697665725C557044726976659F
:108C8000725C6C7769705C636F72655C7261772E81
:108C900063000000A800002041618261704700006D
:108CA00070B505460D480068A84205D10B4800681C
:108CB000C0680A4908600CE00848046807E0E068FA
:108CC00020B1E068A84201D1E868E060E468002CC7
:108CD000F5D129460020FEF7F9FC70BDA800002060
:108CE0002DE9FE4F04460D46914614212846FFF714
:108CF000E2FD88B1002211460120FFF7ADFB0646D8
:108D00001EB94FF0FF30BDE8FE8F288980B129469B
:108D10003046FFF7AFFC0BE02E466FF013013046F4
:108D2000FFF7C9FD20B100BF00BF4FF0FF30EAE7F9
:108D30004846FDF727FC071E07D1AE4202D0304659
:108D4000FFF755FD6FF00300DDE70CB1206810B9A7
:108D500007F1040800E0A046207C617ACDE9010714
:108D60000091A37A4A4641463046FDF7A5FB82466C
:108D7000AE4202D03046FFF73AFD5046C3E700004E
:108D80002DE9F05F0746894690469B463E46002EF9
:108D900042D006F1100000F061FA00283CD0B8F88B
:108DA000081000220320FFF757FB054645B1414656
:108DB0002846FFF773FC18B12846FFF718FD002579
:108DC000002D29D06B2215A10520FEF705FD0446D4
:108DD0002CB92846FFF70BFD0020BDE8F09F256069
:108DE00065601B480068A06099F81000A081B5F884
:108DF00008A0214606F1100000F01CFA20B1204620
:108E0000FEF748FE0020E8E7F06A20B15246002154
:108E10003046F36A984700BF0020DEE72E2E5C2E16
:108E20002E5C5372635C5573725C44726976657232
:108E30005C55704472697665725C6C7769705C61D0
:108E400070695C6170695F6D73672E63000000007C
:108E5000080100202DE9F047074688461546994647
:108E600000BF00BF00BF00BF3C4600BF00BF1CB931
:108E70006FF00500BDE8F08704F1100000F0EEF996
:108E800048B935B12989404602F04EFF2846FFF720
:108E9000AEFC0020EEE700BF4FF0000A00F02FF913
:108EA000824694F9080010F1090F01DB84F808905C
:108EB000504600F05AF900BF0DB12E8900E000269F
:108EC000294604F1100000F0B5F910B14FF0FF3061
:108ED000D0E7E06A20B1324600212046E36A984795
:108EE0000020C7E72DE9F05F80468B4616461F46F7
:108EF000DDF828A000BF00BF00BF00BF454600BF8F
:108F000000BF25B105F1100000F0A8F920B93046E6
:108F1000FFF76DFCBDE8F09FAB2214A10520FEF722
:108F20005BFC04461CB93046FFF761FCF2E72660A3
:108F300066600FB9002000E03868A060A4F80CA0BB
:108F4000B6F80890214605F1100000F073F918B149
:108F50002046FEF79FFDDDE7E86A20B14A46002182
:108F60002846EB6A984700BFD4E700002E2E5C2EFF
:108F70002E5C5372635C5573725C447269766572E1
:108F80005C55704472697665725C6C7769705C617F
:108F900070695C6170695F6D73672E63000000002B
:108FA0002DE9F04105460F4616462C4600BF00BF8E
:108FB0006078012803D12046FCF7EEF805E06078E0
:108FC000042802D12046FBF703FED4B16068C0B18B
:108FD0006068B0F8660040F66931884211DD60686B
:108FE000B0F8680008280CDA94F8200020F010008F
:108FF00084F82000E06A20B1324602212046E36A6C
:1090000098470020BDE8F08170B5044665682146A8
:10901000284600F0ADFB0949284602F069FE0849E0
:10902000284603F002F804220649284601F058FEBB
:109030000549284600F0C4FE70BD0000558E0000B2
:10904000A18F0000358B00001553000070B5044659
:109050000D4629462046F8F787FF70BD704700008F
:109060002DE9F84F81460E461446D9F800A04CB1C0
:109070004FF47A7060434FF47A71B0FBF1F717B98F
:10908000012700E00027FAF727FA0446B9B26A463A
:10909000DAF80000F9F7A6FB80463EB11248804599
:1090A00002D10020306001E0C6F800809DF8000089
:1090B0000A2802D14FF0FF3413E000BF00BFFAF7D7
:1090C0000BFA0546A54201D92D1B02E0C4F1FF3081
:1090D00005444FF47A7068434FF47A71B0FBF1F0B5
:1090E000441C2046BDE8F88F1C01002070B50446E2
:1090F0000D46012229462046FFF7B2FF70BD10B58C
:10910000F7F7D0F810BDF8B507460C464CB14FF450
:109110007A7060434FF47A71B0FBF1F616B901260C
:1091200000E00026FAF7D8F90446B1B26A4638687A
:10913000F9F73EFD9DF800000A2802D14FF0FF34F8
:1091400011E0FAF7C9F90546A54201D32D1B02E04B
:10915000C4F1FF3005444FF47A7068434FF47A71DC
:10916000B0FBF1F0441C2046F8BD10B50446204683
:10917000F7F79CF810BD000008B56B465422142187
:109180000248F9F7D3F90249086008BD5CA801203C
:109190001401002038B5044621680868F9F710FB6F
:1091A00021686A4608680121F9F788FA03482168AE
:1091B0000068F9F718FA0020206038BD140100207B
:1091C00038B504460D46142D00DD142569460E48B9
:1091D0000068F9F7E9F920609DF8000080B9A9B2AC
:1091E0002268101DF9F71AFA2168086020680068E3
:1091F00008B1002038BD214603480068F9F7F3F9AB
:109200004FF0FF30F6E700001401002070B504466F
:109210000D4605B9044D00BF216808682946F9F7D5
:1092200073FB0028F8D170BD1C01002000210160F3
:109230007047000070B505460E4606B9064E29680F
:1092400008683146F9F760FB04460CB9002070BD90
:109250004FF0FF30FBE700001C010020F0B585B0A7
:109260000446256814216846F7F7ADF86946286872
:10927000F9F783FB0646022E07DABDF80400BDF8B5
:109280000610884201DA012000E000200746384637
:1092900005B0F0BD38B504466CB10021684600F059
:1092A00015F8054635B921466846FFF72CFF684694
:1092B00000F002F800BF38BD38B504466A46012107
:1092C0002068F9F705FC0020206038BD38B5044659
:1092D0000D462846F9F7D2FB2060206810B94FF000
:1092E000FF3038BD6A4603A12068F9F757F800201F
:1092F000F7E700004C5749502053656D000000000F
:1093000000210160704710B504462068F9F7C8FCD9
:1093100010BD3EB5044669462068F9F7EDFC08B972
:1093200001203EBD0020FCE72DE9F04385B08046DA
:109330000D4616461F460C9C4FF0000900BF00BFAB
:1093400010A14046F7F75DF8B0B9F6F7ABFF8146DC
:10935000032000214FF400620E4BCDE90132CDE92C
:109360000310A0B2E3B20C4A00902846F9F73AFD88
:109370004846F6F79BFF00E00024E0B205B0BDE8E8
:10938000F083000074637069705F74687265616473
:1093900000000000ECAE0120E8CE01202DE9F041F4
:1093A00006460F46904640F20F1224A10920FEF710
:1093B00013FA04461CB900BF00BFBDE8F0810020CD
:1093C0002060A760C4F80C8066602948006810B966
:1093D00027480460F1E7264800684068B0420CD98D
:1093E000234800684068801B21490968486020487C
:1093F000006820601E4804601DE01D48056817E0F5
:1094000060686968401A6060286820B12868406810
:10941000616888420BD9286828B12868406861686B
:10942000401A29684860286820602C6002E02D6896
:10943000002DE5D100BF00BFBFE700002E2E5C2E3F
:109440002E5C5372635C5573725C4472697665720C
:109450005C55704472697665725C6C7769705C63A8
:109460006F72655C74696D6572732E630000000035
:10947000F000002010B50022024941F28830FFF7C9
:109480008DFF10BDC54A00002DE9F0478046894692
:1094900000BF2248006830B9002249464046FFF725
:1094A000DFFD054637E01D480068406840B11B48B5
:1094B0000068494642684046FFF7D2FD054601E094
:1094C0004FF0FF35681CA8B9144804681349206898
:1094D0000860A668E76821460920FEF7F7F846B15C
:1094E00000210F48FFF70FFE3846B0470C48FFF742
:1094F0000AFFCEE7094800684068A84207D9074834
:1095000000684068401B05490968486003E0002086
:10951000024909684860BDE8F0870000F0000020BB
:10952000880000202DE9F04106460F4614480068E7
:1095300008B9BDE8F0811248046800251BE0A06866
:10954000B04216D1E068B84213D11DB90C49206869
:10955000086001E020682860206828B12068406821
:10956000616808442168486021460920FEF7AEF88A
:10957000DFE725462468002CE1D100BFD9E70000D1
:10958000F00000202DE9FC4704460E4600BF00BF56
:10959000207E0A2808D121461F4801F057FB2146AA
:1095A0000220FEF793F834E0276DD4F82880D4F831
:1095B0008C50D4F8109000BF2146184801F046FBAB
:1095C00001201749087000BF206F10B1206F02F012
:1095D000D4FCE06E10B1E06E02F0CFFC606F10B111
:1095E000606F02F0CAFC4EB1A08B618B231D224636
:1095F000CDE900104146384602F03CFC21460220ED
:10960000FEF764F800BF1DB16FF009014846A84796
:1096100000BFBDE8FC870000C0000020BC000020A7
:10962000C800002010B5044601212046FFF7AAFF1C
:1096300010BD4161704703466FF00900704700009C
:1096400070B5064640F2035239A10220FEF7C4F875
:109650000446002C25D100F0DBFE40F2095234A173
:109660000220FEF7B9F8044694B9304600F0A6FE91
:1096700040F20F522EA10220FEF7AEF804463CB194
:109680003748B0F8B400401E81B23548A0F8B41095
:109690003CB13348B0F8B400401E81B23048A0F865
:1096A000B410002C41D0A0212046F6F78CFE1834CF
:1096B000667041F2D060A4F84E000020A4F850007B
:1096C00042F23820A082E082002004F80F0CFF2034
:1096D00004F80E0C4FF40670E0830620A0850020ED
:1096E000208506206085C01FA0830120A08601F090
:1096F0000FF805462564A56325636564194800686D
:10970000E0601948007860720020E0711748A06698
:1097100040F6B830A0674FF4FA60E0670620C4F85E
:109720008000002084F88600183C204670BD0000B0
:109730002E2E5C2E2E5C5372635C5573725C4472E9
:10974000697665725C55704472697665725C6C7797
:1097500069705C636F72655C7463702E63000000F7
:1097600060A60120B0000020CA000020FBBC000061
:10977000016170472DE9F04705460C4617464FF04A
:10978000040900BF287E18B16FF00500BDE8F0871E
:1097900000BF37B900F088FF074617B96FF0010026
:1097A000F4E74FF0000819E0164850F82800066862
:1097B00010E0708BB8420CD146B1306830B12CB19A
:1097C000206818B130682168884202D16FF0070024
:1097D000DCE7F668002EECD108F10108C845E3DBB0
:1097E0001CB1206808B1206828606F8300BF06485C
:1097F0000068E8600448056002F0F4FD00BF002046
:10980000C4E7000060DF0000B400002010B504468B
:10981000207E012803D0A07F40F01000A077012116
:10982000204600F001F810BD7CB504460E46002E1F
:109830005BD0207E042802D0207E072855D1A06F5F
:1098400020B9A08D42F2382188424ED000BF00BF1F
:10985000A08B618BCDE90010231D2246A16A206DEB
:1098600002F008FB204601F0CDF900BF00BF5A48C6
:109870000068A04205D158480068C0685649086091
:1098800018E055480068554908600EE053480068E4
:10989000C068A04204D15149E0680968C86008E086
:1098A0004E480068C0684D4908604C480068002870
:1098B000ECD100BF0020E06000BF012048490870E3
:1098C00000BF207E04280AD10A20207600BF454828
:1098D0000068E0604348046002F084FD03E0214634
:1098E0000220FDF7F3FE00207CBD207E082868D210
:1098F000DFE800F004343F4F5767675F0025608B57
:1099000030B300BF38480068A04205D1364800682F
:10991000C0683549086018E0334800682F4908607E
:109920000EE02E480068C068A04204D12B49E068D0
:109930000968C86008E029480068C06827490860CD
:10994000264800680028ECD100BF0020E06000BF7E
:1099500021460220FDF7BAFE002435E0002521460D
:10996000224801F073F921460320FDF7AFFE0024E1
:109970002AE0002500BF2146174801F067F90120C1
:109980001749087000BF21460220FDF79FFE002402
:109990001AE0204602F024FB05460DB9052020768A
:1099A00012E0204602F01CFB05460DB9052020768A
:1099B0000AE0204602F014FB05460DB90920207686
:1099C00002E00025002400BF00BF1CB115B92046ED
:1099D00000F0F4FE284687E7BC000020C400002009
:1099E000C8000020C0000020B4000020B800002003
:1099F0002DE9F05F04460E469046994600BF207E52
:109A000018B16FF00800BDE8F09F00BF16B13068D4
:109A1000606002E06FF00500F5E7A4F81C800CB16F
:109A2000206868B9201DFCF7ADFD8346BBF1000F2F
:109A300002D16FF00300E6E7DBF80400206000BF0E
:109A4000B4F81AA0608B38B900F02EFE6083608BEA
:109A500010B96FF00100D6E700F05AFE054600206D
:109A600044F8280FA562681E2062606342F2382025
:109A7000A080E0802068A06042F2382020874FF468
:109A80000670E081E089314600F0D8F8E0810120DD
:109A9000A084E08900EB80004FF6FF7101EA4000EE
:109AA000E084C4F85C90283C0221204600F0DEF8F7
:109AB0000746002F3CD102202076BAF1000F26D0B5
:109AC00000BF1C480068A04205D11A480068C06861
:109AD0001849086018E017480068174908600EE048
:109AE00015480068C068A04204D11349E0680968BD
:109AF000C86008E010480068C0680F4908600E4858
:109B000000680028ECD100BF0020E06000BF00BF6B
:109B100000BF0A480068E0600848046002F062FC88
:109B200000BF01200649087000BF204600F046FE35
:109B3000384668E7B4000020C4000020BC000020C4
:109B4000C80000202DE9F05F07460E4691469A4670
:109B5000DDF8288008F0010008B1042000E00020B2
:109B600008F0020109B10C2100E000214518A422EF
:109B700024A10420FDF730FE041E05D13046FEF777
:109B800036FE0020BDE8F09F84F80A8000202060A7
:109B900066603089401B208114213046FEF78BFE21
:109BA00060B12548B0F88C00401C81B22248A0F872
:109BB0008C10204602F0D4F90020E3E7606840688A
:109BC000E060788BFDF739F8E1680880B88BFDF725
:109BD00034F8E16848805046FDF722F8E1684860B3
:109BE000AB46E91705EB91718910491D49EA01312E
:109BF00088B2FDF722F8E16888810020E168488298
:109C00002046BFE72E2E5C2E2E5C5372635C55738C
:109C1000725C4472697665725C55704472697665EF
:109C2000725C6C7769705C636F72655C7463705FA3
:109C30006F75742E6300000060A601202DE9F041CD
:109C400005460E463046FCF79DFC044654B1A08DF7
:109C500040B1A08D283887B2BD4201DA284600E025
:109C6000384605462846BDE8F08100002DE9F84356
:109C700004460D460027B84600BF00BFB4F8680090
:109C8000102805DAB4F868004FF6FC7188420FD945
:109C90004A48B0F88400401C81B24848A0F88410BB
:109CA000A07F40F08000A0774FF0FF30BDE8F88340
:109CB00005F0020000B1012707F0010008B10420FF
:109CC00000E0002007F0020109B10C2100E00021B2
:109CD00000EB0108B4F8660050B93848B0F88400C9
:109CE000401C81B23548A0F884104FF0FF30DDE70A
:109CF000002241461046FEF7AFFBB0F100090ED13D
:109D0000A07F40F08000A0772C48B0F88400401C71
:109D100081B22A48A0F884104FF0FF30C6E700BF98
:109D200000BF00972A4649462046E36DFFF70AFF29
:109D3000061E0DD1A07F40F08000A0771F48B0F82C
:109D40008400401C81B21D48A0F88410701EADE74D
:109D500000BF00BF00BF00BFE06E08B9E66607E0C5
:109D6000E06E00E0006801680029FBD1066000BFDA
:109D70000020A4F86A0005F0020010B905F0010007
:109D800038B1E06D401CE065B4F86600401EA4F8F0
:109D9000660005F0010018B1A07F40F02000A07718
:109DA0007068FEF772FC34F8681F0844208034F8AD
:109DB000680908B100BF00BF002077E760A6012056
:109DC00000BF00BFC0F88C107047000070B51B4882
:109DD0000078401C1949087000BF1948046829E040
:109DE00094F8210015490978884223D01348007857
:109DF00084F82100A07F00F0010060B100BFA07FC7
:109E000040F00200A07700BF204600F0D7FCA07F02
:109E100020F00300A077E568A06F48B10020094951
:109E20000870204601F02AFA0648007800B1D4E70D
:109E30002C4600BF002CD3D170BD0000CA0000200A
:109E4000BC000020C8000020704700002DE9FC473E
:109E500006468A46FB48B0F87A00401C81B2F948B1
:109E6000A0F87A10F84970680860F74871680068CF
:109E7000007800F00F0001EB8000F4490860F24820
:109E8000006800780007800E41423046FEF713FD5F
:109E900010B93089142808D2EA48B0F88200401C72
:109EA00081B2E848A0F882103BE2E94908685146CF
:109EB000FCF7B3F928B9E648007800F0F000E02894
:109EC00008D1E048B0F88800401C81B2DD48A0F815
:109ED000881026E2DD4909688889FCF711FF4FEAFE
:109EE00020394FEA890041423046FEF7E4FC40B198
:109EF000D448B0F88200401C81B2D248A0F8821049
:109F00000FE2D24909680888FCF7FAFECF490968D0
:109F10000880CE4909684888FCF7F2FECB490968F9
:109F20004880CA4909684868FCF7E4FEC7490968DF
:109F30004860C8490860C54909688868FCF7DAFEC6
:109F4000C24909688860C4490860C0490968C8896D
:109F5000FCF7D6FEBD490968C881BC4909688889F3
:109F6000FCF7CEFE00F03F00BC490870308909784C
:109F700001F0030109B1012100E000210844B849C2
:109F800008800027B74804682AE000BF00BF00BF70
:109F900000BF00BF00BFA08BAC4909680988884298
:109FA0001CD1608BA94909684988884216D1AE49FD
:109FB00060680968884211D1A5492068096888420B
:109FC0000CD100BF00BF37B1E068F860A548006859
:109FD000E060A448046000BF00BF03E02746E468D7
:109FE000002CD2D100BF002C4DD1A048046820E045
:109FF00000BF00BFA08B954909680988884217D126
:10A00000608B924909684988884211D196496068F5
:10A01000096888420CD18E4920680968884207D1B6
:10A02000204602F0FBF93046FEF7E1FBBDE8FC8775
:10A03000E468002CDCD100278D48056810E0688BAF
:10A04000824909684988884208D181492868096895
:10A05000884202D00DB1286800B903E02F46ED68B0
:10A06000002DECD100BF75B137B1E868F8608048C9
:10A070000068E8607E480560284600F0E7F9304651
:10A08000FEF7B5FBD2E7002C7ED0002079490860AE
:10A0900030890881084646606C480068C860002026
:10A0A00075490860754908706C48007800F0080030
:10A0B00018B1707B40F001007073A06F98B120461A
:10A0C00001F0DCF80A3028B1A06F60B16448008864
:10A0D000002808DD5B48B0F87E00401C81B259487A
:10A0E000A0F87E10DDE066480460204600F000FE27
:10A0F000804608F10A00002817D06048007800F078
:10A10000080098B100BFD4F88C0028B16FF00A01A4
:10A11000D4F88C202069904700BF2146514800F0B8
:10A1200095FD21460220FDF7D1FAB9E053480078A9
:10A1300000F01000B8B1A07F00F0100050B900BFCF
:10A14000D4F88C0028B16FF00B01D4F88C20206972
:10A15000904700BF2146434800F078FD2146022089
:10A16000FDF7B4FA9CE04FF00008B4F86400002852
:10A1700012DD00BFE06F40B1B4F864202146E36F08
:10A1800020699847804602E09BE04FF0000800BF3E
:10A1900008F10A0000B984E03748006870B300BFD6
:10A1A00000BFA07F00F0100038B133480068FEF710
:10A1B0001EFB2046FFF736FA73E000BFD4F880009C
:10A1C00048B100232C49D4F880C020690A68214690
:10A1D000E047804607E000232748214602681846EA
:10A1E00001F08BFD804600BF08F10A0000B958E07D
:10A1F000B8F1000F02D020480068A0671F4800781F
:10A2000000F02000E8B1A06F30B1A06F407B40F0BB
:10A210002000A16F48733DE0A08D42F238218842B2
:10A2200002D0A08D401CA08500BFD4F8800048B3A8
:10A2300000231A462146D4F880C02069E0478046B2
:10A2400023E027E060A60120D4000020D0000020F9
:10A250000C010020D8000020DC000020E0000020DD
:10A26000E2000020BC00002008010020C000002007
:10A27000B800002084A70120E8000020E4000020AE
:10A28000EC000020FFE74FF0000800BF08F10A00D3
:10A2900000B906E0002029490860204600F08EFA47
:10A2A00000BF00202549086025490860254840680E
:10A2B000A0B324494868FEF79AFA00202149486073
:10A2C0002CE0214909688889FCF71AFD00F0040098
:10A2D00008BB1E48B0F88800401C81B21B48A0F89B
:10A2E0008810B0F87E00401C81B21848A0F87E109B
:10A2F000154800680088144909684988CDE90010AC
:10A3000013480068134A12888118134B134A1448E3
:10A31000006801F0AFFD3046FEF769FA00BF00BFEC
:10A3200084E60A48B0F87E00401C81B20748A0F8D5
:10A330007E103046FEF75BFA00BF77E6EC000020A7
:10A34000E800002084A70120D000002060A60120A2
:10A35000D8000020E2000020080100200C010020AD
:10A36000DC0000202DE9FC410446216D481EFCF76D
:10A3700057FC07463B4600221146204600F0FEFAF5
:10A3800005460DB9BDE8FC816E680B48B0F8780051
:10A39000401C0949A1F8780006200021CDE90010F1
:10A3A000A37A221D21462846FCF762F82846FEF7CC
:10A3B0001EFA00BFE6E7000060A601202DE9F0418B
:10A3C00006464FF07F08002700250F48046813E079
:10A3D000607EB0420FDC607E40450CDC0B49606A59
:10A3E0000968081AB84206D30849606A09680F1A52
:10A3F000254694F81980E468002CE9D115B1284667
:10A40000FFF710F9BDE8F081BC000020B00000208B
:10A4100070B5002600250B4804680BE00A49606A05
:10A420000968081AB04204D30749606A09680E1A1D
:10A430002546E468002CF1D115B12846FFF7F2F863
:10A4400070BD0000C0000020B00000207CB50546B3
:10A450004548007800F0040008B100207CBD424867
:10A46000007800F0100098B14048006800883F492B
:10A4700009684988CDE900103D4800683D4A1288C6
:10A4800081183D4B3D4A3E48006801F0F3FC69E00D
:10A490003548007800F00200002863D0687EFFF79E
:10A4A000CFF8044654B93748B0F88400401C81B254
:10A4B0003448A0F884104FF0FF30CFE72F480068F1
:10A4C0002060688B60832C480068606027480068C3
:10A4D0000088A0830320207625480068401CA062E5
:10A4E000A06A206321480068C089A4F860001F4862
:10A4F0000068C089A4F86200B4F86000A4F84E00B7
:10A500001B480068401E60652869206168696061B9
:10A51000287A00F08C00207200BF00BF1A48006843
:10A52000E0601948046001F05DFF00BF0120174999
:10A53000087000BF204600F0CDFAE08E211DFFF725
:10A540007DFBE08612212046FFF790FB06462EB1E8
:10A5500000212046FFF716F830467FE7204600F03E
:10A560002DF97BE7002079E7E0000020D0000020F3
:10A57000D8000020E2000020080100200C0100208B
:10A58000DC00002060A60120BC000020C8000020E4
:10A5900070B504460E4600BF207E08B1002070BD95
:10A5A00000BF207E012801D12046F8E740F2212299
:10A5B0002AA10320FDF710F905460DB90020EEE7AA
:10A5C00020692861608B688301202876607E687628
:10A5D000207A2872287A40F002002872A07AA872A5
:10A5E000607A687220682860608B30B300BF2748AB
:10A5F0000068A04205D125480068C068234908606A
:10A6000018E022480068224908600EE020480068EF
:10A61000C068A04204D11E49E0680968C86008E02B
:10A620001B480068C0681A4908601948006800287B
:10A63000ECD100BF0020E06000BF21460220FDF702
:10A6400045F81448686100BF13480068E860124884
:10A65000056001F0C7FE00BF2846A0E72E2E5C2E45
:10A660002E5C5372635C5573725C447269766572DA
:10A670005C55704472697665725C6C7769705C6376
:10A680006F72655C7463702E63000000B40000207C
:10A69000C400002037960000B800002010B540200C
:10A6A000FEF7CEFF10BD000030B5002300BF1648F6
:10A6B00004880088401C144D28804FF6FF708442A7
:10A6C00003D14FF440402C462080002117E00F4872
:10A6D00050F8210002680EE0508B0B4C2488A042F9
:10A6E00008D1581C80B20346B0F5804F01DB002032
:10A6F00030BDDCE7D268002AEED1481CC1B2042983
:10A70000E5DB01480088F3E7AC00002060DF0000D3
:10A71000044800680449096808440249086008467A
:10A7200000687047CC000020B000002070B50546DE
:10A730000C46E9688889FCF7E3FA00F0010020B1D3
:10A74000204601F01AFC002433E013E0E168888918
:10A75000FCF7D6FA00F0010038B10120FCF76DFAE1
:10A76000E96889890843E968888126462468304673
:10A7700001F0F6FB4CB1E068406821890844298962
:10A780000D4A12681144081AE0D594B128890A4983
:10A7900009680844E1684968401A002809DDE06852
:10A7A000808805490988401A288129896868FEF748
:10A7B000E5F82C6070BD0000D80000202DE9F047BE
:10A7C000044600BF00BF6C480068A04202D10020D0
:10A7D000BDE8F087B4F86000B4F84C10884202DAA3
:10A7E000B4F8600001E0B4F84C008146E56EA07F4B
:10A7F00000F0020070B14DB1E9684868FCF77AFAE0
:10A80000A16C401A29890844484503D9204601F023
:10A81000C0FBDDE7266F26B100E03668306800280F
:10A82000FBD191E000BFE9688889FCF769FA00BFB5
:10A83000206FA0B1A07F00F0440080B9E06E38B175
:10A84000E06E006858B9E06E0089E18E884206DA51
:10A85000B4F8660018B1B4F86800102801DB0120D4
:10A8600000E0002020B9A07F00F0A00000B977E050
:10A870002868E066207E02280BD01020FCF7DDF966
:10A88000E96889890843E9688881A07F20F003008E
:10A89000A0772146284600F0ADF8E9684868FCF743
:10A8A00029FA0746E9688889FCF72AFA00F00300CC
:10A8B00008B1012000E000202989084407EB0008C6
:10A8C000206DB0EB080001D5C4F85080E968888994
:10A8D000FCF716FA00F0030008B1012000E00020A8
:10A8E0002989084400282BDD00202860206F10B93A
:10A8F00025672E4627E0E9684868FCF7FBF907461C
:10A90000F1684868FCF7F6F9381A16D504F17007B3
:10A9100000E03F68386860B13968C9684868FCF78A
:10A92000E9F98246E9684868FCF7E4F9BAEB000007
:10A93000EFD4386828603D6005E03560366802E095
:10A94000284601F00DFBE56E55B1E9684868FCF753
:10A95000D1F9A16C401A2989084448457FF662AFB5
:10A9600000BFE06E10B90020A4F86A00A07F20F0BC
:10A970008000A07700202BE7EC0000202DE9F047B5
:10A9800005460E469046994606F11400404481B2B1
:10A9900000220120FDF760FD074647B300BF00BF5E
:10A9A0007C68688BFCF749F92080A88BFCF745F997
:10A9B0006080C4F80490A86AFCF732F9A060B2463F
:10A9C000F11706EB91718910491D102242EA0131FD
:10A9D00088B2FCF732F9A081E88DFCF72EF9E0810E
:10A9E000002020826082E98DA86A084428633846E6
:10A9F000BDE8F0872DE9FC4705460C46A06AFCF748
:10AA00000FF9E9688860E08DFCF717F9E968C881FB
:10AA1000E18DA06A08442063E86800F11408A87A70
:10AA200000F0010070B1211D40F2B450FFF706F9AB
:10AA3000814649F00170FCF7F3F8C8F8000008F10E
:10AA4000040800BFB4F93400401C08B90020A086F7
:10AA50000CB1206840B9201DFBF794FD06460EB9E5
:10AA6000BDE8FC8770682060A06B38B917480068A3
:10AA7000A063E9684868FCF73DF9E063A889696864
:10AA80008988401A87B268684089C01B6968488114
:10AA900068680089C01B696808816968E86848605F
:10AAA0000020E96808820A48B0F87800401C08498C
:10AAB000A1F878000621607ACDE90001A37A221D71
:10AAC00021466868FBF7D4FC00BFC9E7B00000204E
:10AAD00060A601202DE9F04780462B48006800F170
:10AAE0001405294909688889FCF70AF90521B1EBA1
:10AAF000203F46DA244909688889FCF701F90521D5
:10AB0000C1EB20304FF6FF7101EA8006002436E0E9
:10AB100015F80490B9F1000F06D0B9F1010F05D076
:10AB2000B9F1020F21D104E0BDE8F087601C84B2C6
:10AB300024E0601C285C042802D1201DB04200DD06
:10AB4000F2E7E01C295CA01C285C41EA002740F2E7
:10AB5000B450874200DC17B940F2B45000E03846E8
:10AB6000A8F83600201D84B208E0601C285C00B9FB
:10AB7000DAE7601C285C204484B200BF00BFB44206
:10AB8000C6DB00BFD0E70000D00000202DE9FF5F4A
:10AB90000C4616469846DDE90FAB0E9FA146B4421F
:10ABA0001BDA0AF0020050B9B87F00F04000A0B9EB
:10ABB000BBF1000F03D0F86E08B9386F68B104F22A
:10ABC000B75020F00300B04201DD304603E004F24C
:10ABD000B75020F003001FFA80F900224946009880
:10ABE000FDF73AFC05461DB9002004B0BDE8F09F12
:10ABF00000BF00BF6889001BA8F800002C816C8191
:10AC00002846F2E710B50446207EF0B1207E0A28DF
:10AC10001BD0207E012818D0A06F20B1A06FFDF7B7
:10AC2000E6FD0020A067606F01F0A7F900206067D3
:10AC3000401EA086E06E01F0A0F9206F01F09DF9A2
:10AC40000020E0662067A4F86A0010BD70B50546D4
:10AC50000C4600BF2868A04203D12868C06828605D
:10AC600017E01E49286808600EE01C480068C068AC
:10AC7000A04204D11949E0680968C86008E0174893
:10AC80000068C06815490860144800680028ECD1C5
:10AC900000BF0020E06000BF2046FFF7B3FF207E2A
:10ACA0000A280DD0207E01280AD0A07F00F00100E4
:10ACB00030B1A07F40F00200A0772046FFF77EFD74
:10ACC000207E012805D000BF00BF00BF00BF00BF2D
:10ACD00000BF0020207600BF00BF70BDC400002070
:10ACE00000BF00BFC0F8881080F820207047000027
:10ACF0002DE9FC4104464FF000080026FE4800788C
:10AD000000F0040070B3207E022807D1FB49206DBB
:10AD10000968884211D14FF001080EE0F849A06A95
:10AD20000968081A09D4A18DA06A0844F449096881
:10AD3000081A002801DC4FF00108B8F1000F0FD00D
:10AD400000BF00BFEF48007840F00800ED490870F0
:10AD5000A07F20F00100A0776FF00A00BDE8FC8121
:10AD60000020FBE7E448007800F0020068B1207E94
:10AD700002280AD0207E032807D000BFA07F40F021
:10AD80000200A07700BF0020E8E7A07F00F01000DD
:10AD900010B9DD4800686062002084F89E002046FB
:10ADA000FFF798FE207E801E082873D2DFE800F0AF
:10ADB000049BF0EFEEEDECEBCF48007800F01000D4
:10ADC000002877D0CC48007800F00200002871D02D
:10ADD000216FC9684868FBF78DFF401CC7490968A7
:10ADE000884267D12834E08F401CE087C44800685F
:10ADF000401C20602068A060C04800682062C348F2
:10AE00000068C0892087C1480068C0896087BC4845
:10AE10000068401EE062042004F8100CE089283C21
:10AE2000211DFEF70BFFE086E08E00EB80004FF661
:10AE3000FF7101EA4000A4F84E00B4F84C0001286C
:10AE400002D1E08E400000E0E08EA4F84C0000BF8C
:10AE500000BFB4F86800401EA4F86800256F286899
:10AE60002067284601F07CF8206F18B94FF0FF30BA
:10AE7000A08603E00020A08684F8460000BFD4F836
:10AE8000840048B100222146D4F8843020699847D4
:10AE9000064602E0E0E10DE0002600BF06F10A00F0
:10AEA00010B96FF0090059E700BFA07F40F0020021
:10AEB000A07717E09048007800F0100090B1934818
:10AEC00000680088914909684988CDE900108C48DC
:10AED00000688F4A128881188E4B8F4A8748006815
:10AEE00000F0C8FFB9E18448007800F010000028A5
:10AEF00063D0A06C401C81490968081A49D47F4975
:10AF0000206D0968081A002843DC0420207600BF61
:10AF100000BF00BF606930B100222146D4E90403BC
:10AF20009847064601E06FF00D0600BF46B106F1F6
:10AF30000A0010B12046FEF775FB6FF009000DE71F
:10AF4000B4F84C70204600F0E1F9B4F8640020B188
:10AF5000B4F86400401EA4F86400012F02D1E08E12
:10AF6000400000E0E08EA4F84C006648007800F055
:10AF7000200038B100BFA07F40F00200A07700BFE2
:10AF80000720207627E053E108E125E0A1E035E045
:10AF900023E05E48006800885C4909684988CDE97B
:10AFA0000010574800685A4A12888118594B5A4A6B
:10AFB0005248006800F05EFF0DE04F48007800F056
:10AFC000020040B1A06A401E4D490968884202D182
:10AFD000204600F0CCFE40E100BF204600F096F98C
:10AFE0004848007800F0200038B100BFA07F40F052
:10AFF0000200A07700BF072020762EE1204600F057
:10B0000085F94048007800F02000E8B33A4800781D
:10B0100000F01000C8B33949206D0968884242D158
:10B0200000BFA07F40F00200A07700BF2046FFF7DE
:10B03000E9FD00BF00BF39480068A04205D137488C
:10B040000068C0683549086018E034480068344931
:10B0500008600EE032480068C068A04204D1304960
:10B06000E0680968C86008E02D480068C0682C499D
:10B0700008602B4800680028ECD100BF0020E06089
:10B0800000BF0120274901E016E00CE0087000BF76
:10B090000A20207600BF24480068E060224804604F
:10B0A00001F0A0F914E000BFA07F40F00200A077FB
:10B0B00000BF082020760BE00F48007800F0100059
:10B0C00030B10E49206D0968884201D106202076F2
:10B0D000C3E0204600F01AF90A48007800F020008A
:10B0E00078B300BFA07F40F00200A07700BF2046E9
:10B0F000FFF788FD00BF19E0E0000020DC00002021
:10B10000D8000020E4000020B0000020D000002083
:10B11000E2000020080100200C010020BC000020FB
:10B12000C4000020C8000020C000002000BF4C4820
:10B130000068A04206D14A480068C06848490860D3
:10B1400019E02AE046480068464908600EE0454894
:10B150000068C068A04204D14249E0680968C8603C
:10B1600008E040480068C0683E4908603D48006803
:10B170000028ECD100BF0020E06000BF01203A4968
:10B18000087000BF0A20207600BF38480068E060E1
:10B190003648046001F026F900BF5EE0204600F06A
:10B1A000B5F83348007800F01000E0B33149206D65
:10B1B000096888423BD12046FFF724FD00BF00BF4D
:10B1C00027480068A04205D125480068C068244986
:10B1D000086018E022480068224908600EE0214813
:10B1E0000068C068A04204D11E49E0680968C860D0
:10B1F00008E01C480068C0681A49086019480068DF
:10B200000028ECD100BF0020E06000BF01201649FB
:10B21000087000BF0A20207600BF14480068E06074
:10B220001248046000E002E001F0DCF800BF14E026
:10B23000204600F06BF80E48007800F0100050B186
:10B240000C49206D0968884205D10B48007840F010
:10B2500010000949087000E000BF00BF00207DE534
:10B26000BC000020C4000020C8000020C000002056
:10B27000E0000020DC000020E40000202DE9F04187
:10B280000446A06F477BA66F0020A06700BFD4F8DC
:10B29000800040B1002332462146D4F880C02069A6
:10B2A000E047054606E0002332462146184600F0F6
:10B2B00024FD054600BF05BB07F0200020B3A08D8C
:10B2C00042F23821884202D0A08D401CA08500BFE8
:10B2D000D4F8800040B100231A462146D4F880C03B
:10B2E0002069E047054600E0002500BF05F10A009F
:10B2F00050B96FF00900BDE8F08105F10A0010B9FE
:10B300006FF00900F7E7A6670020F4E72DE9FE4F8C
:10B3100004460020009000BF00BFFE48007800F007
:10B32000100000287ED0B4F86000A16D084402909F
:10B33000F949606D0968401A15D4F749606D0968CC
:10B34000884204D1F549A06D0968401A0BD4F3492D
:10B35000A06D0968884231D1F1480068C089B4F80D
:10B36000601088422ADDEE480068C089A4F86000B9
:10B37000B4F86200EA490968C989884204DAE848F1
:10B380000068C089A4F86200E34800686065E3488B
:10B390000068A065B4F8600048B994F89D0068B9E9
:10B3A000002084F89C00012084F89D0006E094F8B9
:10B3B0009D00002802DD002084F89D00D749A06C84
:10B3C0000968081A002848DC0020A4F86400D54861
:10B3D000008840BBB4F86010A06D0144029881421F
:10B3E00035D1B4F93400002831DBCC49A06C0968B0
:10B3F00088422CD10120009094F84700401CC0B234
:10B4000094F84710884204DD94F84700401C84F803
:10B41000470094F84700032812DDB4F84C00E18E91
:10B42000084401E04AE10AE080B2B4F84C108842D6
:10B430000DDDB4F84C00E18E0844A4F84C0006E0A1
:10B4400094F84700032802D1204600F0BDFC009884
:10B45000002801D184F84700ADE0A06C401CAF4942
:10B460000968081A7ED4AD49206D0968081A0028B9
:10B4700078DCA07F00F0040038B1A07F20F0040049
:10B48000A077B4F84E00A4F84C0000202834A07730
:10B49000608BB4F9181000EBE10000B2A083208C9F
:10B4A0009E490988081AA087E08FA18F0844E08789
:10B4B0000020E07799480068206214F8100C283CBE
:10B4C000042824DBB4F84C00B4F84E1088420FDA9C
:10B4D000B4F84C00E18E084480B2B4F84C108842B5
:10B4E00015DDB4F84C00E18E0844A4F84C000EE0E1
:10B4F00034F8361F4943E28A91FBF2F1114488B2D5
:10B50000E18A363C814201DAA4F84C0000BF26E013
:10B51000256F206F0068206700BF6868FDF7B5F8E9
:10B5200000BFB4F8640058B1E9688889FBF7E8FB0C
:10B5300000F0010020B1B4F86400401EA4F86400DB
:10B540006868FDF7A2F834F8681F081A20802846BA
:10B5500000F006FD34F8680908B100BF00BF206F95
:10B56000D8B100E024E0216FC9684868FBF7C2FB4E
:10B570008346216FC9688889FBF7C2FB00F003008E
:10B5800008B1012000E00020216F098908445844D7
:10B5900062490968401A0028BADD206F18B94FF0D7
:10B5A000FF30A08601E00020A0860020E07702E0C6
:10B5B0000020A4F864002BE0E56EE06E0068E06611
:10B5C000E06E10B90020A4F86A0000BF6868FDF7BB
:10B5D0005CF800BFB4F8640058B1E9688889FBF7EB
:10B5E0008FFB00F0010020B1B4F86400401EA4F805
:10B5F00064006868FDF749F834F8681F081A20806D
:10B60000284600F0ADFC34F8680908B100BF00BF5F
:10B61000E06EF0B1E16EC9684868FBF76BFB8346EA
:10B62000E16EC9688889FBF76BFB00F0030008B185
:10B63000012000E00020E16E0989084458443749A0
:10B640000968081A05D43549206D0968081A0028C8
:10B65000B2DDA06B90B33149E06B0968401A2DD57B
:10B6600034F8380F30490988081A0FFA80FAB4F90B
:10B670000800AAEBE0000FFA80FA2089504400B2DB
:10B680002081383CBAF1000F03DACAF100000FFA4A
:10B6900080FA3834B4F90A00AAEBA0000FFA80FA55
:10B6A0006089504400B260816089B4F9081000EBF1
:10B6B000E10000B2A081002044F838091948008850
:10B6C00000286EDD207E07286BDA1348A16A006827
:10B6D000401C081A66D41048A16A0068114A1288F2
:10B6E0001044401E081A00285CDC0B49A06A096857
:10B6F000A0EB01090D48D0F8048000BF00BF00BFD7
:10B7000000BF40684089484531DA00BF00BF0748A4
:10B7100040680DE0E0000020D8000020DC000020A0
:10B72000D0000020E2000020B000002084A701200B
:10B730000089A0EB090080B201900BE0B8F80A0084
:10B74000A9EB00090198A8F808000020A8F80A0051
:10B75000D8F80080B8F80A004845EFDBC9F10000CE
:10B7600001B24046FDF7A7F858B100BF09E0F8491B
:10B770004868C9F1000109B2FDF79DF808B100BFA2
:10B7800000BFF3480089218DF24A1288891A401AB5
:10B79000EF490881EF49A06A0860ED49C96848602F
:10B7A0000BE089E2EB49A06A0968081A05D500BFD9
:10B7B000A07F40F00200A07700BFE649A06A0968B8
:10B7C000081A6FD4A18DA06A0844401EE149096897
:10B7D000081A002866DCDF49A06A096888426FD130
:10B7E000DB49C9688889FBF78BFA00F0030008B1D0
:10B7F000012000E00020D64909890844D649088084
:10B80000A08D0988884241DAD149C9688889FBF747
:10B8100077FA00F0010098B1CD49C9688889FBF733
:10B820006FFA00F03E0B5846FBF707FAC849C968A3
:10B8300089894CF2FF0211400843C549C9688881D3
:10B84000A08DC3490881C9688889FBF759FA00F0BF
:10B85000020020B1BE480089401EBD490881BC4A93
:10B8600011895068FDF78AF8B949C9688889FBF7DA
:10B8700047FA00F0030008B1012000E00020B449BD
:10B8800009890844B449088000BF00BF606F0028E0
:10B8900015D0AF49C9688889FBF732FA00F001007A
:10B8A00078B109E004E2D4F874B0606F00686067B2
:10B8B000584600F055FB00BF606F0028F3D172E0DE
:10B8C0000DE1656F2DE0E9688889FBF719FA00F052
:10B8D000010008B39E49C9688889FBF711FA00F096
:10B8E0000200C8B90120FBF7A8F99949C9688989FC
:10B8F00008439749C96888819549C9688889FBF7D1
:10B90000FFF900F0030008B1012000E00020904999
:10B9100009890844904908802F462D68384600F070
:10B920001FFB55B1E86840682989014489480068CF
:10B93000894A12881044401AC5D59DB385480068CD
:10B94000854909880844E9684968401A002829DDC2
:10B95000E86880887F490988401A7D490881C9685C
:10B960008889FBF7CDF900F0020020B17848008902
:10B97000401E77490881764A11895068FCF7FEFF1E
:10B980007349C9688889FBF7BBF900F0030008B167
:10B99000012000E000206E49098908446E490880B2
:10B9A00000BF00BF65676B4800686B4909880844A1
:10B9B000A06200BF00BFA08D67490988401AA0851A
:10B9C000204600F093FD624840680089002806DDAB
:10B9D0005F4840686149086000205D4948605C49F3
:10B9E000C9688889FBF78CF900F0010028B15C4830
:10B9F000007840F020005A49087055E0666F606F8B
:10BA0000C068406853490860F1688889FBF778F995
:10BA100000F0030008B1012000E000203189084453
:10BA2000A16A0844A06200BFF1688889FBF768F941
:10BA300000BFF1688889FBF763F900F0030008B1E3
:10BA4000012000E0002031890844A18D081AA0855A
:10BA5000204600F04BFD7068008900280DDD3F484E
:10BA6000006828B13D4871680068FCF7E7FD02E016
:10BA70003A497068086000207060F1688889FBF7B7
:10BA80003FF900F0010050B13548007840F0200047
:10BA900033490870207E042801D1072020763068C1
:10BAA0006067304600F05CFA606F28B1606FC06874
:10BAB0004068A16A8842A1D000BFA07F00F00100C9
:10BAC00040B1A07F20F00100A077A07F40F00200ED
:10BAD000A07703E0A07F40F00100A07700E12046BE
:10BAE00000F057FA606F20B9194800F00BFA606750
:10BAF000F6E00027656FD7E0E868406815490968F7
:10BB0000884213D112480089298988420DDD1048E6
:10BB100000F0F8F906463EB10FB13E6000E06667FE
:10BB200029463046FEF702FEC1E0C0E0D7B9E8681A
:10BB3000406808490968081A41D5054800F0E2F94B
:10BB4000064626B1666729463046FEF7EFFDAEE0B1
:10BB500084A70120D8000020E2000020E800002097
:10BB6000E4000020F8684068401C5E490968081A33
:10BB700025D4E8684068401E5A490968081A002818
:10BB80001DDC594800F0BEF90646BEB1F8684068B1
:10BB90003989084453490968401A002809DDF868C2
:10BBA000808850490988081A388139897868FCF7F3
:10BBB000E5FE3E6029463046FEF7B8FD77E028688E
:10BBC000E8BBE868406847490968081A002869DD49
:10BBD000E9688889FBF794F800F0010000B166E09D
:10BBE000414800F08FF92860286848B3E868406849
:10BBF000298908443B490968401A002809DDE8689A
:10BC0000808838490988081A288129896868FCF7DA
:10BC1000B5FEA18DA06A014434480088314A1268FB
:10BC2000104481423DD22968C9688889FBF768F8C9
:10BC300000F00100B0B12968C968888901E031E0ED
:10BC40002FE0FBF75DF800F03E0B5846FAF7F5FFE2
:10BC50002968C96889894CF2FF02114008432968A4
:10BC6000C9688881208DA18D08441E490988401A21
:10BC7000296808812A6811895068FCF77FFE2968C5
:10BC8000C9688889FBF73CF800F0030008B101207F
:10BC900000E000202968098908441449088000BF91
:10BCA00000BF04E02F462D68002D7FF425AF17E07C
:10BCB000204600F06EF913E00A49A06A0968081AE4
:10BCC00008D4A18DA06A0844401E06490968081AD4
:10BCD000002805DD00BFA07F40F00200A07700BF74
:10BCE000BDE8FE8FD800002084A70120E2000020DC
:10BCF00000BF00BFC0F8801070472DE9F041074633
:10BD00000D4614461E463CB12189284600F00CF829
:10BD10002046FCF76CFD05E026B92846FDF776FDC8
:10BD2000BDE8F0810020FBE770B504460E4600BF79
:10BD300000BF00BF00BFA08D3044A085A08D42F29F
:10BD40003821884201DD0846A085204600F0CEFB60
:10BD5000054640F68E00854208DB00BFA07F40F01C
:10BD60000200A07700BF2046FEF728FD70BD2DE938
:10BD7000F0410446206F08B9BDE8F081256F2868BE
:10BD8000206704F16C0600E03668306858B131680D
:10BD9000C9684868FAF7AEFF0746E9684868FAF7E5
:10BDA000A9FF381AF0D4306828603560286810B9C7
:10BDB0000020A4F86A0094F84600401C84F846006D
:10BDC0000020A06300BFD7E710B50446206F90B3F2
:10BDD000A07F00F0040070BB2046FFF7C8FFB4F856
:10BDE0004C00B4F86010884207DDB4F8600000EB46
:10BDF000D0714910A4F84E1006E0B4F84C0000EBE6
:10BE0000D0714910A4F84E10B4F84E00E18E4900EC
:10BE1000884204DAE08E4004000CA4F84E00B4F826
:10BE20004E00E18E032202FB0100A4F84C00A07F2B
:10BE300040F00400A07710BD70B50446206F00B933
:10BE400070BD256F00E02D6828680028FBD1E06EEA
:10BE50002860206FE0660020206794F84600401CB0
:10BE600084F846000020A0632046FEF7A7FC00BF30
:10BE7000E6E700002DE9FC5F81460E46174698462E
:10BE8000DDE90CAB002214210120FCF7E5FA0546A0
:10BE90000DB9BDE8FC9F00BF00BF6C685046FAF7C3
:10BEA000CCFE20805846FAF7C8FE60804846FAF774
:10BEB000B7FE60603046FAF7B3FEA06045F21400AA
:10BEC000FAF7BBFEA08143F62200E0810020208229
:10BED00060820B48B0F87800401C0949A1F878004E
:10BEE00006200021FF234246CDE9001039462846AE
:10BEF000FAF7BEFA2846FCF77AFC00BFC9E7000053
:10BF000060A6012070B5054640F29D4208A10420BC
:10BF1000FBF762FC04460CB9002070BD95E80F00E9
:10BF200084E80F006068FCF765FD2046F5E7000037
:10BF30002E2E5C2E2E5C5372635C5573725C4472C1
:10BF4000697665725C55704472697665725C6C776F
:10BF500069705C636F72655C7463702E63000000CF
:10BF600010B5044644B1606810B16068FCF73FFC4E
:10BF700021460420FBF7AAFB10BD70B5044605E07E
:10BF800025682046FFF7ECFF2C4600BF002CF7D1B8
:10BF900070BD2DE9FC4104460027206DFAF740FEF4
:10BFA00080464346002239462046FEF7E7FC054618
:10BFB00015B9B81EBDE8FC816E68A07F20F00300B3
:10BFC000A0770621607ACDE90001A37A221D2146DF
:10BFD0002846FAF74DFA2846FCF709FC0020E9E765
:10BFE00070B50446E06ED8B1E56E00E02D682868B3
:10BFF0000028FBD1E9688889FAF782FE00F0070083
:10C0000068B90120FAF719FEE96889890843E968E7
:10C010008881A07F40F02000A077002070BD00BF85
:10C0200001212046FDF722FEF8E700BF00BFC167EF
:10C03000704770B504460D461646207E012802D191
:10C040006FF00C0070BD85B1A07F40F01000A077AC
:10C0500026B101212046FDF7E7FBF3E7A06F20B1F1
:10C06000A06FFCF7C4FB0020A0678EB1207E0328E0
:10C0700004D0042803D0072807D101E000BF00BF87
:10C08000E9B22046FDF7D0FBDCE76FF00C00D9E702
:10C090000020D7E72DE9FE4F00200290CA48006833
:10C0A000401CC9490860C9480078401CC74908704D
:10C0B00000BF0025C648046858E100BF00BF00BFAC
:10C0C00000BF00BF00BF94F82100C0490978884232
:10C0D00001D1E4684AE1BD48007884F821000026D7
:10C0E000B146207E022806D194F84600062802D1E7
:10C0F000701CC6B26BE094F846000C2802D1701C8C
:10C10000C6B264E094F89D0000281BDD14F89C0F73
:10C11000401C2070217860789C3C401EAD4A105C29
:10C12000814254DB002084F89C0094F89D0007288D
:10C1300004D294F89D00401C84F89D00204600F035
:10C140000BFC44E0B4F93400002803DBA08E401C53
:10C1500000B2A086206FD0B3B4F93400B4F9441013
:10C16000884234DB207E02280CD040346088B4F949
:10C17000001000EBE100A179974A515C884000B2C1
:10C18000A080403C0020A086B4F84C00B4F86010B9
:10C19000884202DAB4F84C0001E0B4F8600082464C
:10C1A0004FEA6A00A4F84E00B4F84E00E18EB0EBFE
:10C1B000410F06DAE08E4FF6FF7101EA4000A4F865
:10C1C0004E00E08EA4F84C002046FFF735FE207E9E
:10C1D00006280BD1A07F00F0100038B17A49606AC0
:10C1E0000968081A282801D9701CC6B2207A00F004
:10C1F0000800A8B3207E042802D0207E07282FD173
:10C200002434D4E91C21E06E01FB02004FF4FA71E2
:10C21000B0FBF1F054F824196B4A1268511A8842A5
:10C2200006D2701CC6B209F1010000F0FF0917E048
:10C2300094F89E10D4E9240201FB02004FF4FA7135
:10C24000B0FBF1F0604A616A1268511A884207D265
:10C250002046FEF787F894F89E00401C84F89E0064
:10C26000606F78B15849606A0968081AB4F94410D7
:10C2700001EB4101B0EB410F04D3606FFFF77DFE8E
:10C2800000206067207E032807D14F49606A096853
:10C29000081A282801D9701CC6B2207E092807D1A7
:10C2A0004949606A0968081AF02801D9701CC6B2A9
:10C2B000A6B32046FEF7A6FC25B100BF00BFE0688C
:10C2C000E86004E000BF00BF4149E0680860B9F1E0
:10C2D000000F09D0A08B618BCDE90010231D2246F1
:10C2E000A16A206DFFF7C6FDD4F88C80D4F810B099
:10C2F0002746E46839460220FBF7E8F90020374971
:10C30000087000BFB8F1000F03D06FF00901584664
:10C31000C04700BF3148007808B1CAE600E024E019
:10C320002546E468E87F401CE877E87F95F8201010
:10C3300088421ADB0020E8772849087000BFD5F84A
:10C34000880030B12946D5F88820286990470290A6
:10C3500001E00020029000BF2048007800B1A8E66C
:10C36000029810B92846FEF729FA00BF002C7FF486
:10C37000A4AE00251A48046822E000BF00BF0026D2
:10C380001149606A0968081AF02801D9701CC6B200
:10C39000A6B12046FEF736FC25B100BF00BFE0681D
:10C3A000E86004E000BF00BF0D49E0680860274670
:10C3B000E46839460220FBF789F901E02546E46884
:10C3C000002CDAD1BDE8FE8FB0000020CA000020AA
:10C3D000BC00002059DF00004CDF0000C800002036
:10C3E000C000002010B50948006868B90848006816
:10C3F00010B90848006838B10120044908600022DB
:10C400000549FA20FCF7CAFF10BD0000F400002027
:10C41000BC000020C0000020EDCB00001CB504468D
:10C420002148007800F0040008B100201CBD1E481F
:10C43000007800F0020008B31C49A06A0968081AD5
:10C4400024D4A18DA06A084418490968081A002854
:10C450001CDC174800680088154909684988CDE93F
:10C46000001012480068134A12888118124B134AB0
:10C4700013480068FFF7FEFC0020D7E70A48007861
:10C4800000F0010010B10F480068606209480088A0
:10C49000002807DDA07F40F00200A0772046FEF7CD
:10C4A0008DF9C3E70020C1E7E0000020D80000209C
:10C4B000D0000020E2000020080100200C01002034
:10C4C000DC000020B000002010B5FDF77FFC06481E
:10C4D0000078401CC0B20449087000F0010008B1A7
:10C4E000FFF7D8FD10BD0000C900002010B50146BF
:10C4F0008B8D886AC218C88E41F21C140B6BA04247
:10C5000001DD204600E0C88E1844101A04D4888D3E
:10C51000C885086B101A10BD0B6B886AC01A0028FA
:10C5200002DD0020C88506E08C6A0B6B181B00BF7B
:10C5300000BFC88500BF0020EDE700002DE9FF4FD8
:10C540008FB0044617464FF0000A0025AB46002086
:10C550000E900D9000260B900A9009908146B4F839
:10C56000621001EBD1725210E38E9A4201DDE28E2D
:10C5700004E0B4F8620000EBD072521092B207925D
:10C5800000BF109820B96FF00D0013B0BDE8F08F18
:10C5900000BF3946204600F09DF90890089808B180
:10C5A0000898F2E7B4F868000C90E06E002873D0A9
:10C5B000E56E00E02D6828680028FBD1A87A00F01D
:10C5C000010008B1042000E00020A97A01F0020176
:10C5D00009B10C2100E00021084406902989069841
:10C5E00001440798401A1FFA80F8B4F86A000990CD
:10C5F000BDF82400002818DD00BF00BFAB46BDF821
:10C600002400B84202DABDF8240000E03846814632
:10C6100006EB090086B2BDF82400A0EB090080B249
:10C620000990A8EB09001FFA80F800BF00BFBE42C6
:10C6300042DAB8F1000F3FDD288900283CDDB81B45
:10C64000404501DD404600E0B81B80B20590AB4696
:10C65000129800F00100B0B10121129809AB4246D6
:10C66000CDE90040029103200599FEF78FFAB0F161
:10C67000000A00D10DE1109A9119DAF80400059A28
:10C68000F3F788FE0DE0012203200599FBF7E4FE95
:10C69000B0F1000A01D1FCE00FE010983044CAF874
:10C6A00004000598304486B25046FBF7EEFF0C9923
:10C6B000084480B20C9000BF01E000BF00BF84E0DE
:10C6C000B81B80B206900B990798401A80B205906B
:10C6D000DDE90510884201DD059800E00698049028
:10C6E000129800F0010008B30D9808B9012100E08C
:10C6F00000211298CDE9004002910B9A0498104451
:10C7000081B209AB0020079AFEF740FAB0F10008A9
:10C7100000D1BEE000BF00BF109A9119D8F80430D4
:10C720000B9A9818049AF3F735FE1EE000BF00BF7D
:10C73000012200200499FBF78FFE039000B9A8E0C6
:10C740001098811903984160002210460B99FBF75D
:10C7500083FEB0F1000803D10398FCF748F898E095
:10C7600040460399FBF76AFF00BF4046FBF78DFF89
:10C770000C99084480B20C900C98102804DC4FF6F9
:10C78000FC710C98884203D94046FCF730F880E0F1
:10C790000A980090E06D8319002241462046FDF77B
:10C7A000D1F9B0F1000B00D173E00D9810B9CDF8BC
:10C7B00034B004E000BF00BF0E98C0F800B0CDF860
:10C7C00038B00498304486B200BFBE42FFF678AF5E
:10C7D000B9F1000F21DDD5F8048017E0B8F80800A2
:10C7E0004844A8F80800D8F8000068B9B8F80A204A
:10C7F000D8F8041088184A461099F3F7CBFDB8F81A
:10C800000A004844A8F80A00D8F80080B8F1000FE0
:10C81000E4D128894844288100BFBDF82400A4F849
:10C820006A00BAF1000F0AD000BF00BF5146686825
:10C83000FBF704FF2889BAF808100844288115B9C5
:10C840000D98E06601E00D98286054F85C0F3844BC
:10C8500020606089C01B60810C98A081A0895C3C2D
:10C8600008B100BF00BFBBF1000F10D0DBF80C0017
:10C8700068B1129800F0020048B90820FAF7DDF913
:10C88000DBF80C1089890843DBF80C108881002044
:10C890007BE6A07F40F08000A0770D48B0F88400D0
:10C8A000401C81B20A48A0F88410BAF1000F02D0EF
:10C8B0005046FBF79CFF0D9810B10D98FFF75DFBFC
:10C8C000B4F8680008B100BF00BF4FF0FF305CE66D
:10C8D00060A601200246107E04280BD0107E072897
:10C8E00008D0107E022805D0107E032802D06FF0F9
:10C8F0000C00704709B90020FBE7B2F866008842D7
:10C9000006DA907F40F0800090774FF0FF30F0E73C
:10C91000B2F86800102805DAB2F868004FF6FC7328
:10C9200098420ED90B48B0F88400401C83B20948E5
:10C93000A0F88430907F40F0800090774FF0FF3077
:10C94000D7E7B2F8680008B100BF01E000BF00BF40
:10C950000020CEE760A601202DE9FC4705462C6F9C
:10C9600004B9EC6E0CB9BDE8FC87E1688889FAF778
:10C97000C7F900F0010018B1208908B9012000E0D2
:10C9800000208046B8F1000F01D1012000E0002016
:10C990008146E06843684A4600212846FDF7EEFFDD
:10C9A000064606B9DFE77768B8F1000F09D0112015
:10C9B000FAF743F9B9894CF2FF0211400843B881F4
:10C9C0000DE0706800F1140A616809892289891AEA
:10C9D0008BB2012251466068FBF7C0FE00BF0B48D6
:10C9E000B0F87800401C0949A1F878000620002121
:10C9F000CDE90010AB7A2A1D29463046F9F738FDFB
:10CA00003046FBF7F4FE00BFADE7000060A6012052
:10CA100010B586B004460C48FCF720FC88B1002015
:10CA20008DF80400039401A90748FCF7EFFB616847
:10CA300001F10C000021FCF766FB94F9080006B038
:10CA400010BD6FF00500FAE78400002010B5044621
:10CA500000210648FCF757FB201D21688847034842
:10CA6000FCF751FC94F9080010BD0000880000207C
:10CA70002DE9F04105460E4617461548FCF7EEFB3A
:10CA8000002822D0E12213A10720FAF7A5FE0446D0
:10CA90001CB94FF0FF30BDE8F08105202070A56083
:10CAA000E66027B121460A48FCF7B0FB0BE02146BF
:10CAB0000748FCF7BFFB30B121460720FAF706FE16
:10CAC0004FF0FF30E7E70020E5E76FF00500E2E711
:10CAD000840000202E2E5C2E2E5C5372635C5573F6
:10CAE000725C4472697665725C55704472697665F1
:10CAF000725C6C7769705C6170695C74637069709A
:10CB00002E63000038B504460D46FAF79CF80E482F
:10CB100004600E480560C8210D48FCF751FB08B1C0
:10CB200000BF00BF01210B48FCF7D0FB08B100BFDC
:10CB300000BF05204FF4006300220749009007A0C2
:10CB4000FCF7F2FB38BD00007C00002080000020D4
:10CB5000840000208800002025CC000074637069E8
:10CB6000705F7468726561640000000070B505460E
:10CB70000E461148FCF772FB10B96FF0050070BD4E
:10CB8000C0220EA10820FAF727FE044614B94FF080
:10CB9000FF30F4E701202070A560E66021460648DA
:10CBA000FCF748FB30B121460820FAF78FFD4FF023
:10CBB000FF30E4E70020E2E7840000202E2E5C2E08
:10CBC0002E5C5372635C5573725C44726976657255
:10CBD0005C55704472697665725C6C7769705C61F3
:10CBE00070695C74637069702E63000010B5044650
:10CBF000FFF76AFC0748006810B90748006828B1C9
:10CC000000220649FA20FCF7C9FB02E00020044993
:10CC1000086010BDBC000020C0000020EDCB00006B
:10CC2000F400002008B53A48006820B1394800688F
:10CC30003749096888474FF4FA70F6F7E1FB00219D
:10CC40003548FCF760FA61E03348FCF75CFB694665
:10CC50003248FCF719FC00212F48FCF754FA0098E1
:10CC6000007807284ED2DFE800F0040C232B353F74
:10CC70004800009A9268101D009A926811688847CF
:10CC800043E00098C06890F8350000F0600028B1DB
:10CC9000009AD2E90201F8F7F1FF04E0009AD2E924
:10CCA0000201F9F7E1FA08200099FAF70FFD2CE0EC
:10CCB000009A9268101D009A92681168884724E0D3
:10CCC000009B083307CBFCF769FB07200099FAF7B4
:10CCD000FDFC1AE0009AD2E90301FCF723FC0720CF
:10CCE0000099FAF7F3FC10E0009AD2E902108847A5
:10CCF00007200099FAF7EAFC07E0009AD2E902104F
:10CD0000884702E000BF00BF00BF00BF9CE70000F3
:10CD10007C0000208000002088000020840000208B
:10CD200070B505462C4600BF6068B0F1005F03D3C4
:10CD30000F496068884215D3298903221046FBF702
:10CD40008BFB04464CB129462046FBF7A7FC064660
:10CD50001EB12046FBF74BFD00242846FBF747FD9C
:10CD6000204670BD2468002CDED12846F9E700007B
:10CD70000000072070B504463748F7F7D5FA374862
:10CD8000F5F730F83648F5F72DF860213548F5F716
:10CD900051F8062084F82E0004F12F0200213248B9
:10CDA000F4F784FD40F2DC50A085322084F8350091
:10CDB000F5F7E4F8122200212B48F4F7CBFE0546E4
:10CDC000132200212848F4F7C5FE05461122002150
:10CDD0002548F4F7BFFE054645F003052B46112212
:10CDE00000212148F4F7CFFE3C23122200211E48E7
:10CDF000F4F7C9FE122200211B48F4F7ABFE0546EA
:10CE00004FF482611848F4F7BBFD00211648F4F78F
:10CE100051FE064631461448F4F70EFE1248F4F768
:10CE2000F6FE1148F4F7DDFE10490F48F4F721FE35
:10CE30003820F5F749F9F5F781F90D492820F3F77E
:10CE40006DFE2820F3F700FC4FF4905300221146AA
:10CE50000548F4F798FE70BD090800F005180900B0
:10CE6000051409000010064000C00E40C3010080F8
:10CE70004567000010B5044600BF00BF0A48A06225
:10CE8000742084F836006921372001550748606115
:10CE90000748A06104F12F00034908602046FFF70E
:10CEA00069FF002010BD000040010020C5560000B1
:10CEB00075D2000070B505460C46AE6A04F48030A9
:10CEC00020B110480068401C0E49086004F400407E
:10CED00020B10D480068401C0B49086004F0004078
:10CEE00010B1284600F012F804F0010010B13046ED
:10CEF00000F068F804F4E07010B1284600F0A6F8DD
:10CF000070BD00004C01002050010020FEB5054618
:10CF1000122200212748F4F71DFE064610220021A8
:10CF20002448F4F717FE0446012200212148F4F7B3
:10CF300011FE074600BF06F4005098B104F001004E
:10CF400040B101201C490870012229461B48FFF707
:10CF50008FFD07E000201849087001222946184873
:10CF6000FFF786FD06F4A05018B36B4601AA02A98C
:10CF70001048F4F7CBFC04F0020020B1029820F432
:10CF80008040029003E0029840F48040029004F058
:10CF9000040020B1029840F40060029003E002987F
:10CFA00020F4006002900348DDE900320299F4F7B2
:10CFB000CDFCFEBD00C00E4054010020C383000024
:10CFC0009983000070B505466C68002639E0A168B9
:10CFD00001EBC101206850F8210000F0004000B1D1
:10CFE00032E0A16801EBC101206800EB8100006A1A
:10CFF000E0B1A16801EBC101206800EB810090F86D
:10D00000200000F0010040B9A26802EBC2022168D2
:10D0100001EB8201086AFBF7EAFB0020A26802EB41
:10D02000C202216801EB8201086200E00CE0A06806
:10D03000401CA060D4E90110884201D10020A0600A
:10D04000761C6068B042C2D800BF70BD2DE9F041C7
:10D050000546AE6AB468A06810B1A068401E01E041
:10D060006068401E0746FAE0A16801EBC101206834
:10D0700000EB8100006A002870D0A16801EBC101BB
:10D08000206850F8210000F0004000B1EBE0A168FA
:10D0900001EBC101206850F8210000F48070F8B164
:10D0A000A16801EBC101206850F82100C0F30D40D8
:10D0B000A26802EBC202216801EB8201096A488181
:10D0C000A16801EBC101206800EB8100006A408982
:10D0D000A26802EBC202216801EB8201096A0881A1
:10D0E0006248006898B1A26802EBC202206800EBB7
:10D0F0008200016A5D480068FBF7A0FA5B4800689F
:10D10000A26802EBC202216801EB82010862A168F9
:10D1100001EBC101206800EB8100006A53490860FF
:10D12000A16801EBC101206850F8210000F4807073
:10D13000A0B1A16801EBC101206850F8210000F402
:10D14000004060B149480068FBF751FB4848C0887F
:10D15000401C4749C8800020444908601AE0444800
:10D160004088401C42494880294640480068FFF7F3
:10D17000FDFC60B13D480068FBF739FB3C48808905
:10D18000401C3B4988810846C088401CC88000205C
:10D1900036490860032240F2EC511046FBF75CF977
:10D1A000A26802EBC202216801EB820108624FF41F
:10D1B0008040A26802EBC202216801EB8201486054
:10D1C000A16801EBC101206800EB8100006A70B327
:10D1D000A16801EBC101206800EB8100006A406892
:10D1E000A26802EBC202216801EB82018860A1689B
:10D1F00001EBC101206800EB81004068A26802EBEE
:10D20000C202216801EB8201096A49890843A268C8
:10D2100002EBC202216801EB820148604FF000403E
:10D22000A26802EBC202216841F822000EE0FFE78B
:10D230000020A26802EBC202216801EB8201886033
:10D240000B488089401C0A4988810CE0A068401C7A
:10D25000A060D4E90110884201D10020A060A0683C
:10D26000B8427FF401AF00BFBDE8F0815801002053
:10D2700060A601202DE9F84F81460E46002000905F
:10D28000FBF73DFF00903046FBF7B4FB3046FFF75D
:10D2900047FD06465EB94E488089401C4C4988814E
:10D2A0000098FBF762FF4FF0FF30BDE8F88FD9F828
:10D2B0002840606800686168C96801EBC10100EB43
:10D2C0008105286A68B13046FBF791FA40488089A9
:10D2D000401C3F4988810098FBF747FF4FF0FF3023
:10D2E000E3E73046FBF7D1F907466068806861687C
:10D2F000C968884205D9606880686168C968401A51
:10D3000006E06068C068C0F1180061688968084478
:10D310008346BB450DD23046FBF769FA2C4880891D
:10D32000401C2B4988810098FBF71FFF4FF0FF300E
:10D33000BBE74FF0010A4FF080502860B04638E05C
:10D34000606800686168C96801EBC10100EB810594
:10D35000B8F80A006860D8F80400A860BAF1000FB5
:10D3600005D04FF0000A4FF08050286001E0002007
:10D370002860286840F4500028607F1ED8F800809C
:10D380006068C068401C6168C8606068C068182830
:10D3900002D100206168C8602FB9286840F0C04001
:10D3A00028602E6201E0701C2862286840F000406E
:10D3B0002860002FC4D10748F4F725FC04480088F2
:10D3C000401C034908800098FBF7CFFE00206CE763
:10D3D00060A6012000C00E402DE9F04105460E4632
:10D3E00017464FF000081B48046818E0A54204D116
:10D3F00000BF00BF4FF0010810E0608AB8420DD1B5
:10D4000044B1206830B12EB1306818B1206831685D
:10D41000884203D16FF00700BDE8F081E468002C7A
:10D42000E4D10EB9002000E03068286037B900F080
:10D430007DF9074617B96FF00700EDE76F82B8F185
:10D44000000F04D103480068E8600248056000202E
:10D45000E2E70000FC0000202DE9F04104460E4602
:10D460001746608A60B9628A21462046FFF7B4FFFA
:10D470008046B8F1000F02D04046BDE8F08100BF01
:10D480000EB9002000E030686060A782207C40F088
:10D49000040020740848056804E0AC4201D1002073
:10D4A000EBE7ED68002DF8D103480068E060024822
:10D4B00004600020E1E70000FC0000200021416042
:10D4C0008182017C21F004010174704770470000E3
:10D4D0002DE9FF5F05460E467B48B0F86200401C10
:10D4E00081B27948A0F86210D5F804B029899BF878
:10D4F000000000F00F00082202EB8000814208DBF0
:10D500009BF800000007800E41422846FBF7D3F944
:10D5100090B16D48B0F86A00401C81B26A48A0F82A
:10D520006A10B0F86600401C81B26748A0F8661027
:10D530002846FBF75CF9C4E0D5F804906349086815
:10D540003146F8F76AFE8046B9F80000F9F7D8FBD3
:10D550000390B9F80200F9F7D3FB029000270020EE
:10D56000019082465A4804684CE000200190618A8C
:10D570000298814223D1B8F1000F02D1ACB12068EA
:10D5800098B152492068096888420ED0B8F1000F5E
:10D5900015D054B1206840B12168B06801404B48B3
:10D5A0000068B2681040814209D101200190BAF1AF
:10D5B000000F04D1207C00F0040000B9A2460198BD
:10D5C000F0B1A18A039881421AD1201D30B1606860
:10D5D00020B1404960680968884211D13FB1E068D4
:10D5E000F8603B480068E0603948046007E036486E
:10D5F000B0F87600401C81B23348A0F8761003E002
:10D600002746E468002CB0D100BF04B9544624B9C1
:10D610002E497068096888424FD16FF0070128468B
:10D62000FBF749F968B100BF00BF2748B0F86600B2
:10D63000401C81B22448A0F866102846FBF7D7F8B2
:10D640003FE074B1A06940B103980090214B2A4695
:10D650002146D4E906C0E04732E02846FBF7C7F888
:10D660002FE0B8F1000F15D11848007800F0F00055
:10D67000E0280FD09BF8000000F00F00082202EB1A
:10D6800080012846FBF717F900BF00BF0321284699
:10D69000F8F752FC0C48B0F87000401C81B20A4800
:10D6A000A0F87010B0F86600401C81B20648A0F8DF
:10D6B00066102846FBF79BF802E02846FBF797F830
:10D6C00000BFBDE8FF9F000060A601200C01002004
:10D6D000FC0000200801002010B54FF4757207A16E
:10D6E0000120FAF779F804462CB120212046F2F700
:10D6F0006AFEFF20A072204610BD00002E2E5C2E78
:10D700002E5C5372635C5573725C44726976657209
:10D710005C55704472697665725C6C7769705C63A5
:10D720006F72655C7564702E6300000010B5002296
:10D7300000BF124803880088401C104C20804FF620
:10D74000FF70834203D14FF44040234618800C48B9
:10D7500001680EE0488A094B1B88984208D1501C8A
:10D7600080B20246B0F5804F01DB002010BDE0E73B
:10D77000C9680029EED101480088F7E7F8000020C9
:10D78000FC0000208161C2617047000070B5054651
:10D790000D480068A84205D10B480068C0680A49D6
:10D7A00008600CE00848046807E0E06820B1E06821
:10D7B000A84201D1E868E060E468002CF5D1294670
:10D7C0000120F9F783FF70BDFC0000202DE9F8432C
:10D7D00006460F46144698462046F8F7D3FE0546FF
:10D7E0005DB90A48B0F86E00401C81B20748A0F845
:10D7F0006E106FF00300BDE8F883434622463946B9
:10D800003046009500F004F8F5E7000060A601201E
:10D810002DE9FF4F83B004460E469B46DDF840805D
:10D82000608A60B9628A21462046FFF7D5FD8246AC
:10D83000BAF1000F03D0504607B0BDE8F08F0821C1
:10D840003046FBF738F880B1002208210120FAF7B2
:10D8500003FE054615B94FF0FF30EDE7308928B1DA
:10D8600031462846FAF706FF00E0354600BF00BF04
:10D870006F68608AF9F7E1F938805846F9F7DDF901
:10D8800078800020F8800CB1206810B908F10409F4
:10D890000EE02068D8F80410884208D0B54203D0C2
:10D8A0002846FAF7A4FF00256FF00500C4E7A1465B
:10D8B0002889F9F7C2F9B8801121607A8DE803014F
:10D8C000A37A49462846059AF8F7F6FD8246B542FE
:10D8D00003D02846FAF78BFF00250448B0F8600013
:10D8E000401C0249A1F860005046A5E760A601204F
:10D8F0000090D0030C00000000EA32060000000097
:10D9000080D1F0080400000000400040100000003A
:10D910000080054010000000005000401100000091
:10D92000009005401100000000600040120000005F
:10D9300000A005401200000000700040130000002D
:10D9400000B0054013000000004002401400000039
:10D9500000C0054014000000005002402E000000EE
:10D9600000D005402E000000006002402F000000A3
:10D9700000E005402F000000007002403000000071
:10D9800000F005403000000000D0034046000000D9
:10D99000000006404600000000100640470000005E
:10D9A0000020064048000000003006407F000000D4
:10D9B0000040064080000000005006408400000047
:10D9C000006006408C000000004000401000000095
:10D9D00000800540100000000050004011000000D1
:10D9E000009005401100000000600040120000009F
:10D9F00000A005401200000000700040130000006D
:10DA000000B0054013000000004002401400000078
:10DA100000C0054014000000005002402E0000002D
:10DA200000D005402E000000006002402F000000E2
:10DA300000E005402F0000000070024030000000B0
:10DA400000F005403000000000D00340430000001B
:10DA500000000640430000000010064044000000A3
:10DA6000002006404500000000300640580000003D
:10DA70000040064059000000005006405C000000D5
:10DA80000060064064000000007006406C0000006A
:10DA9000008006406D000000009006407F000000FE
:10DAA00000400040008005400050004000900540CC
:10DAB0000060004000A005400070004000B005403C
:10DAC0000040024000C005400050024000D0054028
:10DAD0000060024000E005400070024000F0054098
:10DAE00000D0034000000640001006400010064031
:10DAF000002006400020064000300640003006406E
:10DB000000400640004006400050064000500640DD
:10DB1000006006400060064000700640007006404D
:10DB200000800640008006400090064000900640BD
:10DB300000070000000600000005000000040000CF
:10DB400000030000000200000001000000000000CF
:10DB50000000000018ED00E01CED00E020ED00E00A
:10DB600000E400E004E400E008E400E00CE400E08D
:10DB700010E400E014E400E018E400E01CE400E03D
:10DB800020E400E024E400E028E400E02CE400E0ED
:10DB900030E400E034E400E038E400E03CE400E09D
:10DBA00040E400E044E400E048E400E04CE400E04D
:10DBB00050E400E054E400E058E400E05CE400E0FD
:10DBC00060E400E064E400E068E400E06CE400E0AD
:10DBD00070E400E074E400E078E400E07CE400E05D
:10DBE00080E400E084E400E088E400E000E100E09C
:10DBF00004E100E008E100E00CE100E010E100E0F9
:10DC000080E100E084E100E088E100E08CE100E0F8
:10DC100090E100E000E200E004E200E008E200E061
:10DC20000CE200E010E200E080E200E084E200E0CC
:10DC300088E200E08CE200E090E200E000000100F9
:10DC400002000100030001000200010004000100C5
:10DC500002000100030001000200010005000100B4
:10DC600002000100030001000200010004000100A5
:10DC70000200010003000100020001000600010093
:10DC80000200010003000100020001000400010085
:10DC90000200010003000100020001000500010074
:10DCA0000200010003000100020001000400010065
:10DCB0000200010003000100020001000700010052
:10DCC0000200010003000100020001000400010045
:10DCD0000200010003000100020001000500010034
:10DCE0000200010003000100020001000400010025
:10DCF0000200010003000100020001000600010013
:10DD00000200010003000100020001000400010004
:10DD100002000100030001000200010005000100F3
:10DD200002000100030001000200010004000100E4
:10DD300002000100030001000200010001000000D8
:10DD4000785634120100400001001800000601005E
:10DD500001001000140002000A0001003F00010051
:10DD60000100050001001800780001000400010016
:10DD70000400180008000100040001000100010077
:10DD80008000010016000100010080000100010078
:10DD9000010040005800E80301001A720100100061
:10DDA00001000800E8032800800208004000221952
:10DDB000000000000C000000690000000B000000E3
:10DDC0007100000073000000160000000B0000004E
:10DDD00062000000720000006700000068000000A0
:10DDE0006B0000006B00000005000000FFFFFFFF5C
:10DDF0001C002000A0001C001000100030001400C7
:10DE00001400100030001C0604000400060004008A
:10DE100014000A0008000800100010003000300054
:10DE20006465746563746564206D656D70206F76DC
:10DE30006572666C6F7720696E20706F6F6C200062
:10DE400000000000000000000000000000000000D2
:10DE500000000000000000000000000000000000C2
:10DE600000000000000000000000000000000000B2
:10DE700000000000000000000000000000000000A2
:10DE80000000000000000000000000000000000092
:10DE90000000000000000000000000000000000082
:10DEA0006465746563746564206D656D7020756E5E
:10DEB000646572666C6F7720696E20706F6F6C207E
:10DEC0000000000000000000000000000000000052
:10DED0000000000000000000000000000000000042
:10DEE0000000000000000000000000000000000032
:10DEF0000000000000000000000000000000000022
:10DF00000000000000000000000000000000000011
:10DF10000000000000000000000000000000000001
:10DF2000A0DF0000C8DF0000E8DF0000A8DF00007D
:10DF300094DF00007CDF000088DF0000DCDF0000F1
:10DF4000B4DF0000BCDF0000D0DF000001020304EA
:10DF500005060707070707070703060C1830607850
:10DF6000B8000020B4000020BC000020C000002049
:10DF7000FFFFFFFFFFFF00000000000046494E5F6B
:10DF8000574149545F31000046494E5F574149545B
:10DF90005F32000045535441424C495348454400C8
:10DFA000434C4F534544000053594E5F524356442F
:10DFB00000000000434C4F53494E47004C4153541E
:10DFC0005F41434B000000004C495354454E000054
:10DFD00054494D455F57414954000000434C4F534D
:10DFE000455F57414954000053594E5F53454E54C5
:10DFF0000000000014E0000000000020D801000034
:10E00000A804000048E00000D801002000F801004A
:10E010001446000001AD021EC00B486E194C1AFFD9
:10E0200001131801B72018CF012018F678D201206B
:10E03000081A20281A300401741DC0A80164AB29F5
:08E0400008427063BA0B0000F6
:0400000500000201F4
:00000001FF
